:020000040800F2
:1080000050DE002019130108198300081B830008A3
:108010001D8300081F830008218300080000000062
:10802000000000000000000000000000598200086D
:1080300025830008000000008D8200085D9501087E
:1080400033130108331301083313010833130108F4
:1080500033130108331301083313010833130108E4
:1080600033130108331301083313010833130108D4
:1080700033130108331301083313010833130108C4
:1080800033130108331301083313010833130108B4
:1080900033130108331301083313010833130108A4
:1080A0003313010833130108331301083313010894
:1080B0003313010833130108331301083313010884
:1080C0003313010833130108331301083313010874
:1080D00033130108AF99010833130108379C0108D5
:1080E0003313010833130108331301083313010854
:1080F0003313010833130108331301083313010844
:108100003313010833130108331301083313010833
:10811000CF9B010833130108313C010833130108D8
:108120003313010833130108331301083313010813
:1081300000F002F800F080F80AA090E8000C8244F9
:108140008344AAF10107DA4501D100F075F8AFF2D6
:10815000090EBAE80F0013F0010F18BFFB1A43F025
:1081600001031847B8BD0300D8BD03000A444FF00F
:10817000000C10F8013B13F0070408BF10F8014B86
:108180001D1108BF10F8015B641E05D010F8016BCB
:10819000641E01F8016BF9D113F0080F1EBF10F82F
:1081A000014BAD1C0C1B09D16D1E58BF01F801CB52
:1081B000FAD505E014F8016B01F8016B6D1EF9D5D5
:1081C0009142D6D3704700000023002400250026EA
:1081D000103A28BF78C1FBD8520728BF30C148BF2A
:1081E0000B607047642925F0B387782925F0EC8768
:1081F000732926F054830020704710B510BD7047D6
:1082000054656D636F54535441543800000000703E
:10821000000000671FB526F04EF926F02FFC040081
:108220000020002128F060FA401C6060002000213E
:1082300028F070FAE0601FBD26F0E8FD1146FFF758
:10824000E9FF02F0BDFB27F083F803B4FFF7D5FF89
:1082500003BC11F013FA00001A4B19680868B0E863
:10826000F00F80F309884FF0000080F311884EF082
:108270000D0E70470000000003480068006880F39E
:10828000088862B600DF00BF08ED00E0EFF3098068
:108290000C4B1A6820E9F00F106008B54FF0BF00D2
:1082A00080F3118810F01DFF4FF0000080F311885B
:1082B000BDE8084019680868B0E8F00F80F3098845
:1082C000704700BFBC02002001B44FF0BF0080F334
:1082D000118801BC704701B44FF0000080F3118891
:1082E00001BC70470B49D1F800C04A685CF8043BF8
:1082F0001068184442F8040B8C4528BFA1F1DC0C2F
:108300008A4228BFA1F1DC02C1F800C04A6020F017
:1083100000407047E8D700207047FEE7FEE7FEE721
:10832000FEE7704770477047704700000CB50022A9
:10833000019200925248016841F4803101604FF48B
:10834000A063016801F4003100910199491C019179
:10835000009911B901999942F3D10168890302D5B5
:108360000121009100E000920099012930D1454996
:108370000A6842F010020A600A6822F003020A60EA
:108380000A6842F002020A60416841604168416047
:10839000416841F480614160416821F47C11416091
:1083A000416841F4E8114160016841F08071016069
:1083B00001688901FCD5416821F0030141604168F1
:1083C00041F0020141604168C1F381010229FAD103
:1083D0000CBDABE710B52A48016841F0010101600E
:1083E0004168294A114041600168284A11400160F2
:1083F000016821F480210160416821F4FE0141609F
:108400004FF41F018160FFF7E4FF21494FF0006046
:10841000086010BD10B51A4A506800F00C011D4BE1
:108420001D4800290ED004290ED008290ED0036063
:108430005168194AC1F30311121D515C0268CA4008
:10844000026010BD0360F3E70360F1E7516801F4D7
:108450007011536803F48033022404EB914133B16B
:1084600053689B0307D50D4B59430160E0E70B4B65
:1084700059430160DCE7074B59430160D8E700002E
:1084800000100240002002400000FFF8FFFFF6FE4F
:1084900008ED00E000127A001C00002000093D00F9
:1084A0009A48994941609A494160704797480169E3
:1084B00041F08001016170479448C068C10701D054
:1084C00001207047410701D502207047C00601D541
:1084D000032070470020704770B50446FFF7ECFF9B
:1084E0000546012D05D111F0FDF9641EA4B2002C42
:1084F000F4D104B9FF25284670BD70B5054645F690
:10850000FF763046FFF7E8FF002812D17F4C206944
:1085100040F0020020616561206940F04000206168
:108520003046FFF7D9FF012803D0216921F002016D
:10853000216170BD70B506460D46FF20FFF7CCFFE8
:1085400000280ED1714C206940F001002061358077
:10855000FF20FFF7C1FF012803D0216921F00101AD
:10856000216170BD008870472DE9F04105460E4637
:108570001746002407E036F814102846FFF7DAFF04
:10858000AD1C641CA4B2BC42F5D3BDE8F081C107A8
:1085900003D030F8010C000A70470088C0B2704761
:1085A00010B50446002307E02046FFF7DBFF21F863
:1085B0001300A41C5B1C9BB29342F5D310BD2DE9A4
:1085C000F05F82460F461546AAF10062B2F5002F11
:1085D00038D272B6FFF764FF4FEAD228C2F34906D9
:1085E000C6F58064A54200D82C46DFF828B139E0F2
:1085F00032183BF812208A4203D1401C80B2A042BC
:10860000F6D3A04214D24846FFF777FF002006E0D9
:10861000821937F810102BF81210401C80B2A042BB
:10862000F6D348464FF480623A49FFF79DFF04E0D5
:10863000224639465046FFF797FFA54204D1FFF77F
:1086400035FF62B6BDE8F09F08F10108002607EB90
:1086500044070AEB440A281B85B24FF48064A54204
:1086600000D82C464FF0006000EBC829421429497D
:108670004846FFF795FF00204FF6FF71BFE730B582
:1086800004460D46002306E02046FFF780FFE8542D
:10869000641C5B1C9BB29342F6D330BD70472DE93E
:1086A000F047ADF5006D0D46904600240746A0F159
:1086B0000060B0F5002F23D200264FF48069EA460F
:1086C00015E06878000215F8021B08442146641C76
:1086D000A4B22AF811004A46944206D10024694601
:1086E0003846FFF741FF07F50067B61CB6B24645AE
:1086F000E7D3002C04D0224669463846FFF734FF02
:108700000DF5006DBDE8F0872301674500200240AC
:10871000AB89EFCDB00900202A4908432A490860F7
:10872000704770B50F23C27801260178002A1ED049
:10873000254A126802F4E062C2F5E062120AC2F150
:108740000404D3404578A54082781A402A43120198
:1087500001F1E02181F80024007800F01F018E4033
:108760004009800000F1E020C0F8006170BD01F018
:108770001F0086404809800000F1E020C0F88061B9
:1087800070BD124A114001430F48001F016070473D
:108790000D4A121D002903D0116801431160704772
:1087A00011688143116070474FF0E021042804D024
:1087B000086920F0040008617047086940F004006F
:1087C000086170470000FA050CED00E080FFFF1F14
:1087D00010B5DB4988420AD144150121204607F033
:1087E00034FC2046BDE81040002107F02EBCD549DE
:1087F00088420AD104150121204607F026FC2046B4
:10880000BDE81040002107F020BCCF4988420AD1C2
:108810000121CC03204607F018FC2046BDE810409B
:10882000002107F012BC10BD10B54268C74B1A40BA
:108830000C790B6842EA0422134343608268C44BFC
:108840001A40D1E9024323434C7942EA44021343DC
:108850008360C26A22F47002097C491EC9B242EAEE
:108860000151C16210BD002101600171417181603F
:10887000C160012101747047002904D0816841F072
:10888000010181607047816821F0010181607047BA
:10889000002904D0816841F480718160704781684B
:1088A00021F4807181607047C9B2002A03D0426808
:1088B0000A434260704742688A4342607047816859
:1088C00041F008018160704701460020896809076E
:1088D00000D501207047816841F004018160704734
:1088E000014600208968490700D50120704700290A
:1088F00004D0816841F4A00181607047816821F44F
:10890000A00181607047014600208968490200D5B6
:1089100001207047426822F46042491E42EA413118
:1089200041607047002904D0416841F40061416012
:108930007047416821F400614160704770B50726B7
:1089400009290AD9C568A1F10A0404EB4404A64028
:10895000B543A3401D43C56007E0056901EB410431
:10896000A640B543A3401D4305611F23072A09D232
:10897000446B521E02EB820293409C4391400C4395
:10898000446370BD0D2A09D2046BD21F02EB820230
:1089900093409C4391400C43046370BDC46A0D3AFC
:1089A00002EB820293409C4391400C43C46270BD31
:1089B000002904D0816841F480118160704781688A
:1089C00021F4801181607047C06C80B270475C48B0
:1089D0004C3000687047002904D0416841F4806140
:1089E00041607047416821F480614160704700290F
:1089F00004D0416841F4805141607047416821F4DE
:108A0000805141607047826822F4E0420A438260EC
:108A10007047002904D0816841F4004181607047AB
:108A2000816821F4004181607047002904D0816889
:108A300041F4021181607047816821F40211816064
:108A40007047014600208968890200D501207047DF
:108A500070B5072609290AD9C568A1F10A0404EBF3
:108A60004404A640B543A3401D43C56007E0056923
:108A700001EB4104A640B543A3401D430561836B50
:108A8000C3F30154121B921C02EB82021F24944078
:108A9000A34391400B43836370BD826B22F4401269
:108AA000491E42EA01518163704708B50090009861
:108AB000084400900098026008BD08B50090009836
:108AC0000844283000900098006880B208BD4268D1
:108AD000204B1A400A4342607047416282627047ED
:108AE000426822F01F020A4342607047144908316D
:108AF000002804D0086840F4000008607047086847
:108B000020F40000086070470246002012680A4204
:108B100000D001207047C9430160704710B502467C
:108B200000200B0A5468C9B20C401168194202D0E7
:108B3000002C00D0012010BD090AC9430160704714
:108B40000024014000280140003C0140FFFEF0FFEE
:108B5000FDF7F1FFFFFD3FFF01684FF6FE72114088
:108B600001600021016041608160C1607249724A08
:108B70000839904204D1486840F00F0048607047BF
:108B80006D4A1432904204D1486840F0F0004860C9
:108B90007047694A2832904204D1486840F47060B6
:108BA00048607047644A3C32904204D1486840F4BF
:108BB000704048607047604A5032904204D1486823
:108BC00040F47020486070475B4A6432904204D1A0
:108BD000486840F4700048607047574A78329042C5
:108BE00004D1486840F0706048607047534A111FD4
:108BF000904204D1086840F00F00086070474F4A67
:108C00001432904204D1086840F0F00008607047C8
:108C10004A4A2832904204D1086840F470600860E3
:108C20007047464A3C32904204D1086840F4704094
:108C300008607047414A50329042FAD1086840F4C7
:108C400070200860704730B5026847F6F0739A43A9
:108C50000C6A8B682343D1E904452C4323438C6978
:108C60002343CC6923434C6A23438C6A2343134335
:108C70000360CA6842600A6882604968C16030BDAA
:108C80000021016041608160C160016141618161D9
:108C9000C1610162416281627047002904D00168AC
:108CA00041F001010160704701684FF6FE7211400A
:108CB00001607047002A03D002680A4302607047CF
:108CC00002688A430260704741607047406880B222
:108CD000704702460020D10003D5184908390968B9
:108CE00002E0154908390968114200D00120704797
:108CF000C10003D51149091F086070470E490839A2
:108D00004860704702460020D10003D50B4908395E
:108D1000096802E0084908390968114200D00120B9
:108D20007047C10003D50549091F08607047024913
:108D300008394860704700000800024008040240FB
:108D400010B59C49884209D10121042007F07DF922
:108D50000021BDE81040042007F077B99649884209
:108D600009D10121082007F070F90021BDE8104069
:108D7000082007F06AB99149884209D101211020E1
:108D800007F063F90021BDE81040102007F05DB93D
:108D90008B49884209D10121202007F056F9002192
:108DA000BDE81040202007F050B98649884209D11B
:108DB0000121402007F049F90021BDE81040402082
:108DC00007F043B98049884209D10121802007F08A
:108DD0003CF90021BDE81040802007F036B97B49FE
:108DE00088420AD184150121204607F02EF9204639
:108DF000BDE81040002107F028B910BD10B50121D1
:108E0000084607F022F90021BDE81040012007F0D4
:108E10001CB92DE9F0410022CC7804F00F03E406E0
:108E200001D58C7823430C784FF00F0714F0FF0F17
:108E30004FF0010C1CD005680CFA02F40E88264095
:108E4000A64211D1960007FA06F825EA080503FAAA
:108E500006F848EA0505CE78282E02D0482E02D022
:108E600002E0446100E00461521C082AE4D305607A
:108E70000A88FF2A1ED94568002202F108060CFA6A
:108E800006F40E882640A64210D1960007FA06F88E
:108E900025EA080503FA06F848EA0505CE78282EE3
:108EA00000D14461CE78482E00D10461521C082ABA
:108EB000E3D34560BDE8F0814FF6FF7101800221E8
:108EC00081700421C17070470246002092680A42F6
:108ED00000D001207047806880B2704702460020B1
:108EE000D2680A4200D001207047C06880B2704743
:108EF0000161704741617047002A01D001617047EC
:108F000041617047C160704741F480328261816184
:108F1000826181698069704710B52D4B1A684FF6E0
:108F20008074224042EA00100843186010BD2949AD
:108F3000C8617047F0B5264C002801DAE36900E00B
:108F40006368C0F30346420D120185B2C0F30157B6
:108F50009540032F07D0C2020CD50322B2409343A1
:108F600043F0706209E023F07062636823F070637D
:108F7000636002E0AB4343F0706201B12A43002812
:108F800001DAE261F0BD6260F0BD10B58A07120F30
:108F90000F23934021F003040D4921448C689C4326
:108FA0008C608B68904003438B6010BD0949DC31B5
:108FB0000860704700080140000C014000100140AB
:108FC0000014014000180140001C01400020014035
:108FD00000000140000020420FB41CB5074B06AA58
:108FE0007B4469460090059825F02FFC00206946D7
:108FF00025F03EFC1CBC5DF814FB00008D580200FF
:109000000000000000000000000000000000000060
:109010000000000000000000000000000000000050
:10902000FD4A01211160FD490870012011F02AB8A4
:1090300010B5FB48012404701BF0EEFEF948C0682F
:109040001BF0F1FEF84902200870F848047010BDCA
:10905000012080F31388F6480168F64A01F4E061C4
:1090600011430160BFF34F8FFEE7F0B587B00121D8
:10907000202006F0D4FF0121042006F0D0FF0121BA
:10908000102006F0CCFF0121082006F0C8FF0121C6
:10909000402006F0C4FFE84810250224007AE74E7D
:1090A00004280BD34020ADF818008DF81B508DF824
:1090B0001A4006A9E248FFF7ACFE0AE00420ADF82A
:1090C00018008DF81B508DF81A4006A93046FFF79E
:1090D000A0FE4FF40040ADF814008DF817508DF845
:1090E0001640374605A93846FFF793FEADF8104005
:1090F0008DF813508DF8124004A93846FFF789FE09
:109100000820ADF80C008DF80F508DF80E4003A923
:109110003846FFF77EFE0126ADF808608DF80B504B
:109120008DF80A4002A93846FFF773FEADF80460D7
:109130008DF807508DF8064001A9C248FFF769FE77
:1091400007B0F0BD10B545F2555006F027FE0520DA
:1091500006F027FE4FF47A6006F026FE06F02CFE9D
:10916000BDE8104006F023BE06F021BE2DE9F84F01
:1091700040F2053008F097FCB349087040F2F6253C
:10918000284608F090FC6C1EFF2807D100212846D5
:1091900008F08AFC6421204608F086FC204608F08E
:1091A00082FC0446284608F07EFCA84904EB002017
:1091B0000880A14F012697F8F302012806D987F805
:1091C000F362012140F2F32008F06EFCA0495E201A
:1091D00008800021942008F067FC40F2D32008F0BA
:1091E00062FC04464FF4357008F05DFC994904EBCD
:1091F00000200881072008F056FCFF2804D0082032
:1092000008F051FCFF2803D10921072008F04CFC8D
:1092100040F2625008F047FC044640F2645008F007
:1092200042FC8D4904EB0020088040F26354204644
:1092300008F039FC89490870012804D90E70012111
:10924000204608F031FC78790025FF282ED102F065
:1092500061FB0021052008F027FC7021042008F0A4
:1092600023FC01F01AFE87F8DA50787A00F03F010B
:109270007972092008F018FC0024002104F5A1707F
:1092800008F012FC641CE4B2072CF6D30024002181
:1092900004F2491008F008FC641CE4B2072CF6D371
:1092A00097F86E00012801D987F86E5040F29C446F
:1092B000204608F0F8FB6A4908704FF0FE0AFF28C4
:1092C00001D0012805D881F800A05146204608F0B9
:1092D000EBFB97F85902FF2808D197F85A02FF28AC
:1092E00004D1C82087F8590287F85A5297F87800B5
:1092F000DFF8708138B10421012812D0022820D073
:1093000003282AD124E0294687F89B509B2008F0A7
:10931000CBFB314688F8006040F2673008F0C4FBB0
:109320001BE097F89B0020B987F89B109B2008F062
:10933000BBFB294688F8005040F2673008F0B4FBC8
:109340000BE040F2673008F0AEFB88F8000004E064
:1093500087F89B109B2008F0A7FB43480570434902
:1093600097F89B0008704249087008B141480670A0
:10937000DFF8049199F8000018F077FB3F49088066
:1093800099F800203E483F4932B197F86C2002809E
:1093900097F86D00088005E097F87120028097F833
:1093A000700008804FF0000B002404F1B900009019
:1093B00008F079FB30B1009808F075FB032801D262
:1093C0004FF0010B641CE4B2052CEED32E48BBF128
:1093D000010F05D0057097F8CC002C4910B10AE0B8
:1093E0000670F8E797F8CB0028B997F8CE0010B9C7
:1093F00097F8CD0078B12648057017F8CD0F7A7828
:1094000000EB0220234A80B21080BA7BCD3F032AB2
:1094100047D00E7040E049E0A0012142867B002049
:10942000B006002000000020BE060020BC06002080
:109430000CED00E00400FA05947F002000140140C8
:10944000000C014000080140D70300206C00002000
:109450005000002050120020EA0300202D030020BD
:109460008004002083000020D60300207600002026
:109470004300002070000020420000205C0000201B
:10948000D8030020DA03002080000020860000209E
:10949000940000209E00002097F8D310012204F0D1
:1094A0007FFEB879FF2803D010B111E00D70F8E706
:1094B00087F806A087F8F352FE48A0F800A00146FE
:1094C0000122FD48FFF77BF8B979062008F0ECFA95
:1094D0004FF42E7B584608F0E6FA87F8B8020C28BD
:1094E00005D987F8B8520021584608F0DDFA97F8F8
:1094F000D902012806D987F8D952002140F2D92093
:1095000008F0D2FA97F8DC02012806D987F8DC5275
:1095100000214FF4377008F0C7FA00244FF0030A17
:10952000381990F8F710FF2906D180F8F7A0032129
:1095300004F1F70008F0B8FA641CE4B2082CEFD389
:1095400097F8B802192805D987F8B852002158466B
:1095500008F0AAFA012008E0391891F8BA22FF2A87
:1095600001D181F8BA52401CC0B297F8B812491C18
:109570008142F1D8D1490D8097F80201FF2803D12B
:1095800097F80121FF2A1CD02843000297F80121F7
:1095900002430A801B2008F086FA04461C2008F0CB
:1095A00082FA04EB002A2F2008F07DFA04463020CE
:1095B00008F079FA04EB0020C14C824503D22670F2
:1095C00002E00D80E6E72570312008F06CFA824653
:1095D000322008F068FA0AEB002B452008F063FA05
:1095E0008246462008F05FFA0AEB0020834501D24C
:1095F000667000E0657040F2673008F054FA88F851
:109600000000012801D988F8006097F86103B8B913
:1096100097F8E10097F87E10884203D397F87D1001
:1096200088420DD9C8203C4687F8E100C821E120D6
:1096300008F03AFA94F8591294F85A0218F01DFA00
:10964000F62008F030FA87F8F6009E48017841F0DD
:10965000070101709C48007810B3787A40F001004F
:10966000787289F80060787A00F0FB01797209203D
:1096700008F01AFA7B2024F009FF40F25324204618
:1096800008F011FA022803D90021204608F00CFA4C
:1096900040F2EF24204608F006FAFF2807D00AE03F
:1096A000787A00F0FE00787289F80050DBE700213C
:1096B000204608F0F9F908F043FA8448808820B978
:1096C00040F2E171842001F0A9FF0C2008F0EBF9D1
:1096D0007F490870BDE8F88F10B501210D2006F014
:1096E0009EFCBDE8104001217A48FFF723BC2DE91C
:1096F000F0410024784800260682784D724995F89A
:109700009B000870764F012139706E4B07221A704A
:1097100085F87A63C82285F87B2395F87F20012A93
:1097200001D9704A117095F8B9326F4A0BB980B1FE
:109730001170107818F099F96C4908803A786C48E3
:109740006C494AB195F86C20028095F86D0008804C
:1097500008E004201070ECE795F87120028095F87D
:109760007000088095F892106348012905D0032104
:10977000817195F8D80010B103E08671F9E75F4870
:10978000067017F045FD5E48291991F8B210015591
:10979000641CE4B2072CF7D3BDE8F08110B501F0EA
:1097A0007CFBFFF7E1FCBDE81040A0E75548002432
:1097B0000470554804704FF4FA6010F0B3F8FFF7E6
:1097C0008BFF07F0C9FD5148047007F038FE1420E4
:1097D00010F0A8F8F9E74E4DDFF83891DFF838813E
:1097E0004E4EDFF83CA1DFF83CB14F4F00247C71B6
:1097F000B8F800207979CA40D00702D0685C401CD4
:109800006854685C06280FD36C5419F8010010B135
:10981000401E09F8010019F8010028B9D00703D04B
:1098200000223D4801F0B1FA7879401CC0B278714D
:109830000328DDD37C71BBF800207979CA40D007BA
:1098400002D0705C401C7054705C06280FD37454B6
:109850001AF8010010B1401E0AF801001AF80100C0
:1098600028B9D00703D000222E4801F08EFA78796B
:10987000401CC0B278710328DDD342F2107010F0A2
:1098800051F8B4E786B0FFF7D3FB00201CF070F866
:1098900000201DF043FA254816F0D8FE2449142074
:1098A000087024490B200870234902200870052005
:1098B000224945E058000020007700087A02002085
:1098C0007E0200204100002043000020B011002053
:1098D0002B0300200004300028120020947F002079
:1098E000420000203C0000203F0000205C000020DF
:1098F000D8030020DA030020BA16002062000020FE
:10990000CC00002004010020FB000020FF0000200C
:10991000DD000020A60000208E000020DA000020DC
:10992000A30000209000002000000020DC82002026
:10993000A10400209E0400209F040020A204002017
:109940000870FD4CFD4E002520780C2802D1FFF751
:109950006FFB25702078132808D1FFF769FB0020E2
:109960001CF006F800201DF0D9F92570B07978B9FF
:10997000757000234FF41672F14901A800951BF091
:109980000CFA024622B10023ED4901A81DF057F957
:1099900005200FF0C7FFD7E70026EA48012404702E
:1099A000E94F97F8D800002804D0C0EB00108100E0
:1099B000E6480180DFF898B30025DFF89883FFF7C9
:1099C000D3FBE549087808B1401E0870087808B94B
:1099D000E2480570DFF8609399F800000D280AD17D
:1099E0003878ABF800007878ABF802000222D8494A
:1099F000DB48FEF7E4FD99F800000E280BD1B8789B
:109A0000ABF80000F878ABF80200D5480222D04944
:109A10001030FEF7D4FDD34A1078012803D1D24983
:109A20000878401C0870D0480178052901D91570C4
:109A30000570CE490878012806D1887918B1CD7112
:109A4000401E887100E0CC71C9490878012806D110
:109A5000887918B1CD71401E887100E0CC71C5497C
:109A60000878012806D1887918B1CD71401E887117
:109A700000E0CC71C0490878012806D1887918B176
:109A8000CD71401E887100E0CC71BC490878012876
:109A900006D1887918B1CD71401E887100E0CC7173
:109AA00097F8D80050B1A949088808B1401E08802D
:109AB000B34809880278114300D10470761CF6B2CD
:109AC0003C2E07D397F85C0318B1AE480178491EC5
:109AD00001700026AB48007830B997F85C0318B1E4
:109AE00087F85C53A848847099F80000102803D1C7
:109AF00089F8005001F00EFF99F80000112809D0F4
:109B000003F07BFFA1490880DFF884A2DAF80000A7
:109B1000B8B121E08848057014244FF45A7640F219
:109B20006C75B44205D0652C03D0FF21204607F0A8
:109B3000BBFF641CA4B2AC42F3D301F0EBFEFFF711
:109B400087FA97F8B90238B104F060F888F8044051
:109B500088F8024088F801408E4A107801280CD11C
:109B60008D490878401CC0B20870052805D11570D1
:109B70000D7002F099FF84488470DAF8000098B103
:109B800097F8631081B1401ECAF8000060B99B20AD
:109B900007F089FF8149087087F89B0080490870A9
:109BA00088F80240784845707E490888012801D924
:109BB000401E08807C49088808B1401E088008883B
:109BC00038B997F8ED00FF2803D001217748FFF757
:109BD00091F997F8ED00FF2803D101217348FFF7B1
:109BE00087F97349087818B188F80140401E087059
:109BF0007049087818B188F80240401E087008784B
:109C000058B96D480470DFF8B4A19AF80000012833
:109C100001D102F0AAFB8AF800506949087818B10E
:109C2000401E087088F803406649087808B1401E55
:109C30000870087878B96448017801290BD105705B
:109C40000F2089F8000088F8014088F8024088F861
:109C500005405E4805705E490888401E80B2088055
:109C600008B95C480470DFF8709199F8000010B1F1
:109C7000401E89F8000099F8000020B90022012157
:109C8000564801F082F899F8010010B1401E89F899
:109C9000010099F8010020B9002203214F4801F08A
:109CA00074F899F8020010B1401E89F8020099F882
:109CB000020020B900220521484801F066F899F811
:109CC000030010B1401E89F8030099F8030020B981
:109CD00000220721414801F058F899F8040010B11A
:109CE000401E89F8040099F8040020B900220921D7
:109CF0003A4801F04AF899F8050010B1401E89F879
:109D0000050099F8050020B900220B21334801F025
:109D10003CF899F8060010B1401E89F8060099F841
:109D2000060020B900220D212C4801F02EF84FF436
:109D30007A700FF0F7FD42E61F030020BA160020EC
:109D40001407002030000020947F002064000020D1
:109D500058000020BA110020190300201803002029
:109D6000107700082303002024030020D2110020D4
:109D7000DC110020E6110020FA110020F011002073
:109D8000620000201E030020000000204C00002084
:109D900054000020710000206E00002043000020CD
:109DA0003400002034030020460000200008014059
:109DB000380000203900002072000020350000200B
:109DC0003A000020F6000020F7000020F8000020F4
:109DD000680000206A000020A6020020A4020020E3
:109DE0000EB5FC484FF0010880F8008080F8018033
:109DF00080F8028080F8038080F8048080F8068074
:109E00000121F548FFF774F8F549F4480860F54872
:109E10000178F54801704FF6FF76ED21CDE9001687
:109E200047F61760002302901A462421F02008F01C
:109E300053FA47F61965CDE9016538200E210090E7
:109E4000C823EA4A084608F02BFA6921662009F07F
:109E5000A1F99421662009F09DF9BF21662009F03F
:109E600099F9CDE90065E2A36C220A21012008F0EE
:109E7000FDF9CDE90065DFA397220A21012008F052
:109E8000F5F9CDE90065DCA3C2220A21012008F022
:109E9000EDF9DA4F0024DFF868A39AF80600401CB9
:109EA000C0B28AF80600052801D98AF80640DFF812
:109EB000549399F8000001285BD0022868D0042848
:109EC0007FD0052877D00728FCD0062874D0082832
:109ED000FCD00B2871D00F2870D0CB49087800280F
:109EE0006DD000200870C9490978012968D09AF816
:109EF000020080B308F09BFFB64880F8018080F82C
:109F0000028080F8038080F804806921662009F0CF
:109F100041F99421662009F03DF9BF21662009F03E
:109F200039F9CDE90065B2A36C220A21012008F0BD
:109F30009DF9CDE90065AFA397220A21012008F021
:109F400095F9CDE90065ACA3C2220A21012008F0F1
:109F50008DF98AF80240AE490878002870D00020B8
:109F60000870AC4880F800809AF80600052868D090
:109F7000DFE0284607F0BFFFCDE900651E22A6A35B
:109F80001146012008F072F90FF0ECFCFFF760F8C1
:109F900089F80040284607F0AEFFCDE900651E2293
:109FA000A0A31146012008F061F901F0B3FC02F012
:109FB00079FD1BE205E06AE076E082E086E0A0E061
:109FC000A1E089F80040994890F8650001280FD079
:109FD000B0B102281CD0032822D0042828D005289C
:109FE00030D0062836D007283CD0082842D048E098
:109FF0004FF4964948460FF051FBC7F8029040E0F5
:10A000004FF4165948460FF049FBC7F8029038E064
:10A010004FF4164948460FF041FBC7F8029030E074
:10A020004FF4614948460FF039FBC7F8029028E029
:10A030004FF4E13948460FF031FBC7F8029020E0B9
:10A040006EE06FE04FF4963948460FF027FBC7F8F3
:10A05000029016E04FF4966948460FF01FFBC7F8D0
:10A0600002900EE04FF4965948460FF017FBC7F8E0
:10A07000029006E04FF4615948460FF00FFBC7F815
:10A080000290B879032894D10FF06CFCAEE16848D7
:10A090000088C1B2C0F3072017F095FD002002F040
:10A0A0004DF889F80040A1E161480088C1B2C0F3D1
:10A0B000072017F0E2FC012002F040F889F8004088
:10A0C00094E117F0A5F889F800408FE1CDE900652B
:10A0D00047A36C220A21012008F0C8F8CDE90065E9
:10A0E00044A397220A21012008F0C0F8CDE90065B9
:10A0F00041A3C2220A21012008F0B8F889F80040E3
:10A1000074E10120EEE640B94A48008884380F28FF
:10A1100003D3022008F06CFE64E103F0CBF861E1A8
:10A1200001201DE744480022B0F90010104609F054
:10A130004FFCDFF8F89099F85C03F8B1DFF8FCA069
:10A140009AF8000018B908F072FE8AF80080CDE98C
:10A1500000653BA36C220021012008F087F8CDE9BF
:10A16000006539A397220021012008F07FF899F8B3
:10A1700006102022002008F07BFEB9E099F80800C4
:10A18000042873D931480078012804D09AF80710C0
:10A1900001296DD06DE008F04AFE4FF4784BCDE90F
:10A1A00000B52BA367220021012008F05FF8CDE95C
:10A1B00000B529A392220021012008F057F8CDE92B
:10A1C00000B527A3BD220021012008F04FF88AF82E
:10A1D00007808DE0BA110020000801401001002026
:10A1E0000C0100204300002034000020FC0F040874
:10A1F0005345540046414E0053595300BA160020AF
:10A20000000000201F0300203D02002071000020FC
:10A210003B0000203C0200205570646174696E6749
:10A22000000000005265737461727400947F002016
:10A230004A00002050000020680200201D0300207A
:10A240004D4F44425553000049440000470200204E
:10A250004869676800000000566F6C7461676500AC
:10A260006F6E2052533438350000000035E0FFE7B0
:10A2700058B1FE48B0F9000008F04AF8FC480078F0
:10A2800008F029FA08F071FA32E08AF8074008F07D
:10A29000CEFDF84880F8018080F8028080F80380C5
:10A2A00080F8058080F804806921662008F072FF3C
:10A2B0009421662008F06EFFBF21662008F06AFF37
:10A2C000ED21CDE9001647F61760002302901A46EB
:10A2D0002D21EF2008F000F80AE0E448B0F9000072
:10A2E00008F016F8E248007808F0F5F908F03DFAB1
:10A2F0004FF0000A504603F014FF0AF1010A0AF079
:10A30000FF0ABAF1090FF5D308F051FB08F064FA1F
:10A3100099F80800042811D9D7480078012806D0F8
:10A32000D648007838B1012009F0DFFA0FE00020AC
:10A3300009F0DBFA0BE009F06BFA08E0CF4800788F
:10A3400018B1012009F0D1FA01E009F061FADFF853
:10A35000249399F8070048B1CDE901650023C84A64
:10A360001A210D20009407F09BFF08E0CDE901655C
:10A3700000231A461A210D20009407F0ADFF99F82A
:10A38000080048B1CDE901650D23BE4A1A211846DF
:10A39000009407F085FF08E0CDE901650D23002258
:10A3A0001A211846009407F097FF99F8070010B19A
:10A3B000401E89F8070099F8080010B1401E89F87E
:10A3C0000800B1498879022815D0052842D006280E
:10A3D00040D0CDE901651A21D223AC4A0846009449
:10A3E00007F05EFFAA48007803F0F0F84FF496708B
:10A3F0000FF098FA4FE5087A462809D2CDE90165B1
:10A400001A21D223A34A0846009407F049FFE9E73E
:10A41000502809D2CDE901651A21D2239E4A084667
:10A42000009407F03DFFDDE75A2809D2CDE9016528
:10A430001A21D223994A0846009407F031FFD1E748
:10A44000CDE901651A21D223954A0846009407F008
:10A4500027FFC7E7CDE901651A21D223914A0846B3
:10A46000009407F01DFFBDE700258F4C0FF01CFE88
:10A470008E4F4FF4964697F86510092932D2DFE8DF
:10A4800001F0050A0E13181D22272C004FF4165058
:10A490000FF004F929E030460FF000F925E04FF401
:10A4A00016400FF0FBF820E04FF461400FF0F6F893
:10A4B0001BE04FF4E1300FF0F1F816E04FF4963066
:10A4C0000FF0ECF811E04FF496600FF0E7F80CE0B5
:10A4D0004FF496500FF0E2F807E04FF461500FF0A0
:10A4E000DDF802E030460FF0D9F8714A4FF4C87138
:10A4F0001180704801804FF496400FF02BF96E48A0
:10A500000121017000208146391881F8A991401C71
:10A51000C0B20828F8D3DFF8A4816949087830B1BF
:10A52000401EC0B20870012801D115F019FA654823
:10A53000017831B10178491E0170007808B90FF037
:10A5400011FA61494889322802D2401C488114E03E
:10A55000A1F80A9007F0F4FA5C4882885C490A8006
:10A5600082798A70C279CA70027A0A71027859496E
:10A570000A7042784A7080788870C82D74D100259E
:10A58000554E3178491C3170544A98F80000D080FB
:10A5900050EAC17101D0012826D151490978142906
:10A5A0000BD015290BD0404C4E4922680A606268D6
:10A5B0004A60227A0A7220B107E04B4CF4E74B4C18
:10A5C000F2E74FF416500FF0C5F809200FF063FDC5
:10A5D000474897F8602201788A4205D087F86012D0
:10A5E0004FF4187007F060FA98F8000010B931784D
:10A5F000C90701D1022837D12F480078012808D097
:10A60000022808D0032809D004280AD007280BD034
:10A6100022E0384C20E0374C08341DE0354C083C33
:10A620001AE0344C103417E015F02AFA0024264EB4
:10A63000DFF8C4A0DFF8C4B01036305D15F025FA9D
:10A640009AF80000B0719BF80000F071641CE4B24D
:10A65000062CF2D31C4C103498F8000018B94FF4B3
:10A6600096400FF077F84BE052E000005C000020CD
:10A6700034000020BA1100204702002018030020F7
:10A680008411040828140408AB220020CC16040806
:10A6900000010020141C04085C210408A4260408FE
:10A6A000EC2B040834310408BE190308947F002001
:10A6B00064020020620200202903002044020020DE
:10A6C000310300202F03002000000020B0110020E3
:10A6D000F4030020EC030020940200206088002096
:10A6E0001F030020CA030020C7190308D01903085C
:10A6F0009A02002094190308E5030020E4030020D7
:10A70000FE48216801606168416008200FF0C3FCC9
:10A710006D1CADB20A200FF005F9FEE608B50AF08F
:10A72000CAFAF74D2878697800EB0121F5480180D5
:10A73000A978EA7801EB0221418029796A7901EB55
:10A7400002218180A979EA7901EB0221C180297A6D
:10A750006A7A01EB02210181A97AEA7A01EB0221EE
:10A760004181297B6A7B01EB02218181A97BEA7B04
:10A7700001EB0221C1810421E348FEF7BBFB4FF44A
:10A780000071E248FEF7B4FB0DF06AFE45200BF0C5
:10A7900098FADF4C0027E770DE4E4FF032084FF09A
:10A7A000010901230022DC49DC48CDF800800BF0D0
:10A7B000F8FB08B986F80090E078401CC0B2E07061
:10A7C0000A28EED33078012800D03770DFF850A384
:10A7D000D44ED54FDFF85483DFF854B30425D54861
:10A7E0000178491C017009F0B9FE0AF075F80DF006
:10A7F00050FEFEF7B9FC4FF0000C84F804C00020B6
:10A80000BF4A473A131893F89E12022901D004292F
:10A8100042D1DFF824E33EF810E0BEF1010F02D090
:10A820002379C3B133E09AF8001031BB357087F853
:10A83000009088F8005082F89B5093F89E120229ED
:10A8400006D192F86310C1EB01118900CBF800101A
:10A8500084F804901BE092F8B93213B104290DD0AA
:10A8600015E0DBF8001041B986F800C03D7088F8AB
:10A8700000C082F89BC08AF800C008E086F800C0DB
:10A880003D7088F800C082F89BC08AF800C0AB49D0
:10A8900081F8049081F80290401CC0B20828AFD320
:10A8A0000AF007FB9648473890F8EF12012935D196
:10A8B000A34A90F8F1121288511A00D5494290F833
:10A8C000B42391422ADD84F8009084F8019090F836
:10A8D0006310FF2902D13C2180F8631090F86310C7
:10A8E000A9B1C1EB01118900CBF80010954981F89D
:10A8F0000090357088F80050417A41F001014172B2
:10A90000092007F0D1F887F80090022060708B488A
:10A9100080F8029080F8019080F804904FF49670CF
:10A920000FF000F85BE7002400258749002008703D
:10A93000864908708649FF2008708649087040F6ED
:10A94000B8300EF0EFFFDFF8B881DFF8DC91824E0F
:10A950006F4FA8F1470899F8000017F086F830808B
:10A96000B7F90810884203D0388174490120487033
:10A970006D1CADB298F8800100EB8000A84204D2B3
:10A98000012017F0E7FA002502E0002017F0E2FAB4
:10A99000641CE4B2052C09D998F8DB0003280BD01D
:10A9A000012003F0BCFC002404F01FFD0AF0A7FD09
:10A9B000C8200EF0B7FFCEE7022003F0B0FCF2E7AC
:10A9C0002DE9FF41002465490803FDF7DAFEFEF793
:10A9D00083FE4FF4A060FDF79FFEFEF7C5FB482005
:10A9E0000EF06CFF40F2CF21642009F03FF906F031
:10A9F000AFFFFEF7A7FB00F050FAFEF736FB0AF0B8
:10AA0000DDFA002101200AF03BFC002102200AF0BF
:10AA100037FC002103200AF033FC002104200AF057
:10AA20002FFC002105200AF02BFC35484C49473803
:10AA300090F86A000870FEF799FBFEF795FBFEF7A9
:10AA400093FB01214748FEF753FA07F0A3FBFEF7FB
:10AA50004EFEFEF789FB0125FEF786FB142C0AD279
:10AA600007F0D6F8012806D0641CE4B264200EF08A
:10AA700059FF002DF0D100240620CDE900044FF449
:10AA8000617802942346424637A13B4803940EF076
:10AA900040F90220CDE900044FF4C8760294002367
:10AAA000324636A1374803940EF033F90525CDE937
:10AAB000005402940023324633A1354803940EF02B
:10AAC00028F90326CDE9006402940023642231A111
:10AAD000344803940EF01DF90127CDE90074029467
:10AAE0000023642230A1344803940EF012F9CDE91A
:10AAF000005402940023424660E00000CA03002094
:10AB0000DB7F00200412002000180140000C0140EF
:10AB100000000020460200208C0200208802002055
:10AB200031000020430000203F00002034000020BE
:10AB3000540000204D0200203C120020BA110020D9
:10AB40005C020020420000207B0000209E020020CA
:10AB50009F020020A00200205C000020008000086E
:10AB60007F00002000080140436F6E74726F6C4CD0
:10AB70006F6769630000000027A90008496E7075BF
:10AB8000740000001DA70008434F4D4D0000000059
:10AB900069A4000844697370616C795265667265D6
:10ABA00073680000E19D0008536F667477617265F9
:10ABB00074696D65720000009999000850A15248AF
:10ABC00003940EF0A6F8CDE90074029400236422E9
:10ABD0004EA1524803940EF09CF8CDE90054029423
:10ABE00000234FF416724EA1504803940EF091F8D2
:10ABF000CDE900640294002364224DA150480394DF
:10AC00000EF087F80EF062FB04B00020BDE8F08182
:10AC10002DE9F041002500F07F004FF6FF7404EAB3
:10AC200040000C0602D540F0010701E000F0FE07ED
:10AC300001F07F00000440EA02261E4300244FF08A
:10AC40007E5826FA04F000F0010060B1C4F117014B
:10AC5000884026F087FC0146404626F039FB29460D
:10AC600026F0C8FA0546641CE4B2172CE9D37F3FEE
:10AC70000124BC404146284626F0BCFA0546204641
:10AC800026F070FC2946BDE8F04126F0B3BC2D4DFE
:10AC900000264FF47A77287870B1401EC1B229702F
:10ACA00051B9002400222146274800F06EF8641CA8
:10ACB000E4B2032CF6D32E7038460EF033FEEAE7EA
:10ACC00070B51546214B188021480078002815D111
:10ACD000084626F047FC1F4904460860284626F02F
:10ACE00041FC1D4905460860204626F0E7FB1B494C
:10ACF0000880284626F0E2FB1949088270BD000052
:10AD00004D5354500000000085980008436F6F6C4D
:10AD1000696E674C6F636B4F75740000D7970008BE
:10AD2000576966697461736B00000000C57801089B
:10AD30004B65797061647348616E646C65000000F6
:10AD4000AD9700087A0000208800002064020020EF
:10AD500046020020880200208C0200207C02002095
:10AD60002812002048437047C84000F00100704797
:10AD700001238B40DBB20178002A02D01943017015
:10AD80007047DA4311400170704701238B409BB23A
:10AD90000188002A02D0194301807047DA4311402C
:10ADA0000180704701228A40D1B20078084201D167
:10ADB000002070470120704770B540F27A4006F0DD
:10ADC00072FEFE4D287040F27C4006F06CFE4FF69D
:10ADD000FF7404EA0020688040F27B4006F063FEC6
:10ADE00069880844688040F27D4006F05CFEF44DBE
:10ADF000287040F27F4006F056FE04EA002068808A
:10AE000040F27E4006F04FFE6988084468804FF4A7
:10AE1000906006F048FEEB4D287040F2824006F04C
:10AE200042FE04EA0020688040F2814006F03BFECA
:10AE300069880844688040F2894006F034FEE24D9B
:10AE4000287040F28B4006F02EFE04EA0020688055
:10AE500040F28A4006F027FE69880844688040F284
:10AE6000834006F020FED94D287040F2854006F060
:10AE70001AFE04EA0020688040F2844006F013FEC7
:10AE800069880844688070BD01EB002109B27F2801
:10AE900001D908B27047084670472DE9F84F6E2077
:10AEA00006F001FEDFF8288388F86E0000240128F0
:10AEB00005D988F86E4000216E2006F0F5FD0025CA
:10AEC000C44E4FF48F67284606F0EDFDA5F15F02F2
:10AED000A42A1FD298F86E1001EBC10303EB4111B5
:10AEE00006EBC10313F812C0844507D803EB4202F6
:10AEF0005278824202D308F805000DE0B64800EB14
:10AF00008100284410F85F1C08F80510284606F058
:10AF1000CBFD01E008F805006D1CADB2BD42D2D9F1
:10AF200098F85D00FF2801D188F85D40AB4998F89A
:10AF30005D000870AB4D0222A9492846FDF730FBA1
:10AF4000A74E327898F80610FF291BD0D1B1914254
:10AF500005D03180012231462846FDF730FB00251F
:10AF60006F46284606F09FFD78556D1CADB2042D46
:10AF7000F7D39C4B9B4D9DF8001010332035FF29D3
:10AF800010D01BE0022296492846FDF709FB3078D5
:10AF900088F80600FF2801D00028E0D1FE2088F8BC
:10AFA0000600DCE79DF80100FF2807D19DF80200AC
:10AFB000FF2803D19DF80300FF282ED0F1B398F8A5
:10AFC0000000814224D09DF8010098F801209042B1
:10AFD0001ED09DF8022098F80250AA4218D09DF881
:10AFE000032098F80350AA4212D0318070801D4689
:10AFF00002227B492846FDF7E2FA9DF802103180D3
:10B000009DF803107180022275492846FDF7D7FA92
:10B0100098F8D902FF2830D036E00222704918464D
:10B02000FDF7BEFA307888F80000B07888F80100A3
:10B0300002226B492846FDF7B3FA00E006E03078BB
:10B0400088F80200B07888F80300E1E7022264493A
:10B050001846FDF7A5FA307888F80000B07888F82F
:10B06000010002225E492846FDF79AFA307888F8F6
:10B070000200B07888F80300CAE788F8D9420021B6
:10B0800040F2D92006F010FD98F87E03FF280DD17C
:10B0900088F87E4388F87D43002140F27D3006F039
:10B0A00003FD002140F27E3006F0FEFC98F87E039E
:10B0B0004B4D0002283D98F87D130143298398F8F1
:10B0C0001B1098F81C00012601EB002298F82F00B5
:10B0D000454900EB0020824201D20E7000E00C7066
:10B0E00098F8310098F8322000EB022298F84500D9
:10B0F00000EB0020824201D24E7000E04C704FF411
:10B100005A77384606F0CFFC38490870FF2804D13A
:10B110000C702146384606F0C7FC98F85C00344BAA
:10B12000FF2803D198F85B10FF290AD098F85B102C
:10B13000FFF7AAFE188098F881132020FF290AD073
:10B140001BE01C8000215B2006F0AEFC00215C208F
:10B1500006F0AAFCEFE74F2188F88113662188F8F2
:10B16000821388F8831388F8844388F8850388F865
:10B17000860388F8870388F8880398F889236F2165
:10B18000FF2A11D14C2288F8892388F88A13772264
:10B1900088F88B2388F88C4388F88D0388F88E0311
:10B1A00088F88F0388F8900398F891236427FF2A82
:10B1B0002ED14D2288F8912365221BE0D211002068
:10B1C000DC110020E6110020F0110020FA1100200F
:10B1D000947F0020701F030800220308450200200E
:10B1E00058000020007700087E0200202203002083
:10B1F0006E02002088F8922388F8937388F89443AD
:10B2000088F8950388F8960388F8970388F89803D8
:10B2100098F89923FF2A11D1482288F899236922A6
:10B2200088F89A2388F89B4388F89C0388F89D0344
:10B2300088F89E0388F89F0388F8A00398F8A12354
:10B24000FF2A12D1412288F8A123752288F8A2236F
:10B25000742288F8A32388F8A41388F8A54388F8F3
:10B26000A60388F8A70388F8A80398F889034C2850
:10B2700000D0EE7198F8ED00FF2806D0C0EB00106A
:10B280004FF6FF7101EA8000E88298F8A903FF28D1
:10B2900001D188F8A94398F89702FF2811D198F8AE
:10B2A0009602FF280DD1002140F2972006F0FCFB0A
:10B2B00088F89742012140F2962006F0F5FB88F8C5
:10B2C000966298F82D04FF280ED1002505F22D4036
:10B2D00080B2002106F0E8FB08EB050080F82D4461
:10B2E0006D1CADB22E2DF1D315F00EFE98F8820034
:10B2F0004546022801D985F8824095F89200DFF88A
:10B300002CB4012804D985F8924003208BF806005C
:10B3100095F8B403FF2806D11E2185F8B4134FF425
:10B320006D7006F0C1FB40F28C4006F0BCFB00EBF8
:10B3300080004000FE4908804FF47A72904201D9A3
:10B340000A8005E0B0F5FA7F02D24FF42F70088032
:10B3500040F28D4006F0A7FBF6490870FFF72CFD80
:10B3600095F8F102FF2800D010B9A02085F8F1026D
:10B37000F149A879087040F28F4A504606F093FBD5
:10B38000DFF8B8934FF49268FF2804D1404606F0E6
:10B390008AFBFF283AD0504606F085FBC9F800002A
:10B3A000404606F080FBD9F8001041EA0020C9F8B9
:10B3B000000040F2914006F076FBD9F8001041EA17
:10B3C0000040C9F8000040F2924006F06CFBD9F84A
:10B3D000001041EA0060C9F800000021DFF8609326
:10B3E000002001EB41024FEA820801EB410209EB28
:10B3F000C20208EB40032B4493F8B5C3BCF1180F0D
:10B4000011D902EB400C8CF8014010E028786978E3
:10B4100040EA0120A97840EA0140E97840EA016069
:10B42000C9F80000D9E702EB400A8AF801C093F896
:10B43000B6333B2B02D902F8104001E002F810307D
:10B44000401C80B20628D4D3491C89B20829C7D32E
:10B450000020BC492A1892F82D240A54401C80B2BE
:10B460002E28F7D395F878043238652801D385F86B
:10B47000787440F2954006F016FBB34F0002388016
:10B4800040F2944006F00FFB39880843388040F2C0
:10B49000974006F008FBAD4F0002388040F296401E
:10B4A00006F001FB3988084338800027A046E819D8
:10B4B00090F86712FF2907D180F8678207F26720AA
:10B4C00080B2002106F0F0FA7F1CBFB2092FEED344
:10B4D00095F88101FF2806D185F88181002140F28D
:10B4E000811006F0E1FA95F88001FF2806D185F871
:10B4F000808100214FF4C07006F0D6FA0021944AF2
:10B50000944F002007EB811343F82020401C80B2A9
:10B510001028F9D3491C89B20729F2D39BF80600F9
:10B52000032838D10024DFF830A20AF266390AF184
:10B53000D60AE1B25046FFF735FC40B1E1B24846C9
:10B54000FFF730FC26F00EF807EB8411C861641C8D
:10B55000A4B2052CEDD305215046FFF723FC50B1D2
:10B5600095F8620395F86313000200B2084425F0D1
:10B57000E1FFC7F85C0106215046FFF713FC50B10C
:10B5800095F8640395F86513000200B2084425F0AD
:10B59000D1FFC7F89C0195F85F03FF2812D195F8F9
:10B5A00060132846FF290DD180F85F8380F86083FF
:10B5B000002140F25F3006F077FA00214FF4587016
:10B5C00006F072FAE879092803D00921072006F06D
:10B5D0006BFA95F85F0040F26134152805D13146C9
:10B5E00085F86163204606F05FFA95F8A2001528F9
:10B5F00005D1314685F86163204606F055FA4FF4CF
:10B60000187006F050FA5549087095F82903FF287C
:10B6100002D1052085F82903BDE8F88F1CB5024644
:10B620000846843A4E4CC1B2072A0ED2DFE802F037
:10B63000040E190D242F3900A1786278CDE900217C
:10B640002378E279A17906F03AFB1CBDA1786278F3
:10B65000CDE900212378E279C1B2A08806F02FFB62
:10B660001CBDA1786278CDE900212378A179C2B20E
:10B67000A08806F024FB1CBDA1786278CDE90021EA
:10B68000E279C3B2A179A08806F019FB1CBDA078AD
:10B69000CDE900102378E279A179A08806F00FFBAC
:10B6A0001CBD6078CDE900012378E279A179A088FA
:10B6B00006F005FB1CBD10B501210F2006F0F4F9C2
:10B6C0000021102006F0F0F90121112006F0ECF91C
:10B6D0000021BDE81040122006F0E6B970B5002444
:10B6E000204D04F5B070295D06F0DEF9641CE4B26B
:10B6F000072CF6D370BD70B500241B4D24F001005B
:10B70000295C04F11B0006F0CFF9A41CE4B2152C4F
:10B71000F4D3012424F00100285A010A04F11B008B
:10B7200006F0C2F9A41CE4B2162C1FE0BA160020E1
:10B73000A20200201C030020280300200C0000208F
:10B740006A8600203C8600207402002072020020DD
:10B7500000007F437C840020947F00209A02002018
:10B76000B01100201B1A0308DA190308D2D30024F1
:10B77000FE4D24F00100295C04F1310006F094F93B
:10B78000A41CE4B2152CF4D3012424F00100285A9F
:10B79000010A04F1310006F087F9A41CE4B2162C6A
:10B7A000F3D370BD2DE9F0410025DFF8C4830024F8
:10B7B000C5EBC50000EB080605EB85073819315DC0
:10B7C00000F5A17006F070F9641CE4B2052CF5D305
:10B7D0006D1CEDB2022DEAD3BDE8F08170B50024F6
:10B7E000E44D04F22D10295D06F05EF9641CE4B20C
:10B7F000152CF6D370BD2DE9F04107460024DE4D2F
:10B800000126062F21D2DFE807F07F037F21446263
:10B81000DA48015D04F2031006F046F9012C07D165
:10B820000321A02006F040F90321A12006F03CF9F5
:10B83000072C04D2002104F1B20006F035F90121F1
:10B840006F2006F031F985F86F605DE0CC48015D4E
:10B8500004F2031006F028F9012C07D10221A020E0
:10B8600006F022F90221A12006F01EF9072C04D2CD
:10B87000002104F1B20006F017F904219B2006F024
:10B8800013F903216F2006F00FF9032085F86F00EC
:10B890003AE0BC48015D04F2031006F005F9012C02
:10B8A00007D10221A02006F0FFF80221A12006F016
:10B8B000FBF8072C04D2002104F1B20006F0F4F8E2
:10B8C00001216F2006F0F0F885F86F601CE0AE48AB
:10B8D000015D04F2031006F0E7F8012C07D1022104
:10B8E000A02006F0E1F80221A12006F0DDF8072CE7
:10B8F00004D2002104F1B20006F0D6F801216F2035
:10B9000006F0D2F885F86F60641CE4B22A2CFFF4CC
:10B9100078AF61E72DE9F0415F249C4D964E4FF4DE
:10B920008177652C19D096F86E0000EBC00101EB11
:10B93000401005EB8000204410F85F1C204606F004
:10B94000B3F896F86E0000EBC00101EB401005EB78
:10B950008000204410F85F0C3055641CA4B2BC4237
:10B96000DFD996F86E1040F259256C1C11B10129EF
:10B9700013D024E0C821284606F096F8002120467E
:10B9800006F092F8284606F08EF886F8590220460E
:10B9900006F089F886F85A0211E0A821284606F038
:10B9A00083F80221204606F07FF8284606F07BF84F
:10B9B00086F85902204606F076F886F85A0274484E
:10B9C0000078FFF718FFFFF709FFFFF7EBFEFFF71F
:10B9D00092FEFFF783FEFFF76EFE4F2140F28130AB
:10B9E00006F062F8662140F2823006F05DF86621CA
:10B9F00040F2833006F058F800214FF4617006F0F1
:10BA000053F8202140F2853006F04EF8202140F214
:10BA1000863006F049F8202140F2873006F044F8DD
:10BA200020214FF4627006F03FF84C2140F289303B
:10BA300006F03AF86F2140F28A3006F035F87721A7
:10BA400040F28B3006F030F800214FF4637006F0BE
:10BA50002BF8202140F28D3006F026F8202140F20C
:10BA60008E3006F021F8202140F28F3006F01CF8CD
:10BA700020214FF4647006F017F84D2140F2913008
:10BA800006F012F8652140F2923006F00DF86421BC
:10BA900040F2933006F008F800214FF4657006F08C
:10BAA00003F8202140F2953005F0FEFF202140F2FE
:10BAB000963005F0F9FF202140F2973005F0F4FFB1
:10BAC00020214FF4667005F0EFFF482140F29930D5
:10BAD00005F0EAFF692140F29A3005F0E5FF002108
:10BAE00040F29B3005F0E0FF20214FF4677005F035
:10BAF000DBFF202140F29D3005F0D6FF202140F2EF
:10BB00009E3005F0D1FF202140F29F3005F0CCFFA0
:10BB100020214FF4687005F0C7FF412140F2A130A9
:10BB200005F0C2FF752140F2A23005F0BDFF74217F
:10BB300040F2A33005F0B8FF6F214FF4697005F0B3
:10BB4000B3FF002140F2A53005F0AEFF202140F206
:10BB5000A63005F0A9FF202140F2A73005F0A4FF90
:10BB600020214FF46A7005F09FFF13E0F0190308DD
:10BB7000F0230308061A0308947F002048230308D3
:10BB8000722303089C230308C6230308002203082A
:10BB90007F0000200021922005F086FF0024482726
:10BBA0004FF0470807EB4405A8B205F07CFFFF28DB
:10BBB00009D108EB440080B2002105F075FFA8B25E
:10BBC000002105F071FF641CA4B2082CEAD3012007
:10BBD00086F8B80201214FF42E7005F065FF0E21A2
:10BBE00040F2BA2005F060FF0E2086F8BA0296F8FF
:10BBF00048030025FF2873D106F552765420307093
:10BC000053217170B0704121F17030713820707122
:10BC1000B571F571A6F5527654214FF4527005F0C6
:10BC200043FF532140F2493005F03EFF542140F2DA
:10BC30004A3005F039FF412140F24B3005F034FF26
:10BC400054214FF4537005F02FFF382140F24D304E
:10BC500005F02AFF002140F24E3005F025FF0021BB
:10BC600040F24F3005F020FF00214FF4547005F0F2
:10BC70001BFF002140F2513005F016FF002140F279
:10BC8000523005F011FF002140F2533005F00CFF57
:10BC900000214FF4557005F007FF002140F25530A8
:10BCA00005F002FF002140F2563005F0FDFE0021B4
:10BCB00040F2573005F0F8FE00214FF4567005F0C1
:10BCC000F3FE002140F2593005F0EEFE002140F273
:10BCD0005A3005F0E9FE002140F25B3005F0E4FE49
:10BCE000C82140F2AA3005F0DFFE002140F2AB305F
:10BCF00005F0DAFEC8214FF46B7005F0D5FE002187
:10BD000040F2AD3005F0D0FE282140F2AE3005F013
:10BD1000CBFE102140F2AF3005F0C6FE1E214FF4DD
:10BD20006C7005F0C1FE0F2140F2B13005F0BCFE91
:10BD3000322140F2B23005F0B7FE052140F2B330B7
:10BD400005F0B2FE06214FF4A87005F0ADFE1E21ED
:10BD500040F2511005F0A8FE08214FF4A97005F03B
:10BD6000A3FE1E2140F2531005F09EFE12214FF457
:10BD7000AA7005F099FE1E2140F2551005F094FEC0
:10BD800016214FF4AB7005F08FFE1E2140F25710C4
:10BD900005F08AFE002140F2B92005F085FE96F8F4
:10BDA0009702FF280DD196F89602FF2809D10021AD
:10BDB00040F2972005F078FE012140F2962005F030
:10BDC00073FE40F2E1718420FFF728FC0024301953
:10BDD00090F86712FF2907D180F8675204F26720B4
:10BDE00080B2002105F060FE641CA4B2092CEED3E1
:10BDF000002404F5A17080B2002105F055FE641CFA
:10BE0000A4B2072CF5D3002404F2491080B200211B
:10BE100005F04AFE641CA4B2072CF5D3DCE42DE93E
:10BE2000F041FE4C40F25A26204694F86E10771EE0
:10BE300090F87E0000297DD000EBC0000525B0FB06
:10BE4000F5F020307B34C1B2E1707E2005F02CFE8D
:10BE5000A07800EBC000B0FBF5F02030C1B2A170BB
:10BE60007D2005F021FE14F8040C00EBC000B0FBAF
:10BE7000F5F02030C1B204F8041C772005F014FE60
:10BE800094F8660000EBC000B0FBF5F02030C1B2C2
:10BE900084F86610E12005F007FE94F8DE0194F8BE
:10BEA000DF1100EB012080B200EBC000B0FBF5F029
:10BEB00000F5A07082B2110A84F8DF1184F8DE2147
:10BEC000304605F0F1FD94F8DE11384605F0ECFD42
:10BED000A07EE17E00EB012080B200EBC000B0FB51
:10BEE000F5F000F5A07080B2010AE176A076962008
:10BEF00005F0DAFDA17E952005F0D6FD207F617F5B
:10BF000000EB012080B200EBC000B0FBF5F000F5C3
:10BF1000A07080B2010A61772077982005F0C4FDF7
:10BF2000217F972005F0C0FDA07FE17F00EB01207D
:10BF300080B200E041E000EBC000B0FBF5F000F59E
:10BF4000A07080B2010AE177A0779A2005F0ACFDDD
:10BF5000A17F992005F0A8FD14F8070D617800EB8A
:10BF6000012080B200EBC000B0FBF5F000F5A0703E
:10BF700080B2010A61702070752005F095FD14F8FB
:10BF8000071B742005F090FD14F8090D617800EB93
:10BF9000012080B200EBC000B0FBF5F000F5A0700E
:10BFA00080B2010A61702070732005F07DFD217858
:10BFB000BDE8F041722005F077BD2038C0B20925F8
:10BFC00000EB8000B0FBF5F07B34C1B2E1707E2065
:10BFD00005F06AFDA0782038C0B200EB8000B0FB0D
:10BFE000F5F0C1B2A1707D2005F05EFD14F8040CDF
:10BFF0002038C0B200EB8000B0FBF5F0C1B204F80D
:10C00000041C772005F050FD94F866002038C0B27B
:10C0100000EB8000B0FBF5F0C1B284F86610E120BF
:10C0200005F042FD94F8DE0194F8DF1100EB0120E9
:10C03000A0F5A07080B200EB8000B0FBF5F082B2FA
:10C04000110A84F8DF1184F8DE21304605F02CFD5A
:10C0500094F8DE11384605F027FDA07EE17E00EB66
:10C060000120A0F5A07080B200EB8000B0FBF5F0DD
:10C0700080B2010AE176A076962005F015FDA17E3A
:10C08000952005F011FD207F617F00EB0120A0F5D8
:10C09000A07080B200EB8000B0FBF5F080B2010A26
:10C0A00061772077982005F0FFFC217F972005F02D
:10C0B000FBFCE17F5A4EA07F06EB0121084480B2D1
:10C0C00000EB8000B0FBF5F080B2010AE177A077C9
:10C0D0009A2005F0E9FCA17F992005F0E5FC14F811
:10C0E000070D617806EB0121084480B200EB800067
:10C0F000B0FBF5F080B2010A61702070752005F088
:10C10000D3FC14F8071B742005F0CEFC14F8090DBD
:10C11000617806EB0121084480B200EB8000B0FB9F
:10C12000F5F080B2010A61702070732005F0BCFC4C
:10C130002178BDE8F041722005F0B6BC10B5374C4F
:10C14000012823D09A2005F0AEFC703484F82A0030
:10C15000992005F0A8FC84F82900702005F0A3FCC4
:10C160002070712005F09FFC6070752005F09BFC2D
:10C170006071742005F097FC2071732005F093FC2A
:10C18000E070722005F08FFCA07010BD40F25A20C4
:10C1900005F089FC793484F8E10140F2592005F07A
:10C1A00082FC84F8E0016C2005F07DFC04F80D0CA5
:10C1B0006D2005F078FC04F80C0C962005F073FC5B
:10C1C0006077952005F06FFC2077982005F06BFCD8
:10C1D000E077972005F067FCA07710BD2DE9F043CC
:10C1E000DFF838800F4E414698F8B99291F87D00FB
:10C1F00091F8615300EB800300EB800044000A4F8C
:10C2000091F8C5104FF0050CA6F12C02B9F1000F02
:10C2100001D1D07C98B198F8590207E0947F0020B2
:10C22000C0FEFFFF5C0000201F03002098F85A8228
:10C2300000EB0820084400B250834DB32CE098F87E
:10C24000990098F89A8000EB082000B250830A29E0
:10C2500003D00844508385B115E00A2190FBF1F822
:10C2600001FB1808B8F1000FF5D090FBF1F801FBC5
:10C270001801401A0A305083EDE7B2F91A00B0EB0A
:10C28000430F00DD5483508B308087F800C007E0F7
:10C29000B0EB430F00DD5483508B308006203870A4
:10C2A0000020D07282F808C0BDE8F0832DE9F0418B
:10C2B000DFF8FCC3FF4A9CF8B700907361469CF816
:10C2C000B98291F87E0091F8615300EB800300EB96
:10C2D00080004400F84F91F8C51002F12C06B8F127
:10C2E000000F01D1D07C50B19CF859029CF85AC281
:10C2F00000EB0C20401A00B250834DB32CE09CF8A8
:10C3000099009CF89AC000EB0C2000B250830A29D7
:10C3100003D0401A508385B115E00A2190FBF1FC4F
:10C3200001FB1C0CBCF1000FF5D090FBF1FC01FBF4
:10C330001C01401A0A385083EDE7B2F91A00B0EB3D
:10C34000430F00DA5483508B30800720387007E0A9
:10C35000B0EB430F00DA5483508B308008203870E4
:10C360000020D0720520107258E52DE9F041D14C23
:10C37000CF4D01262179687A002914D040F00101BF
:10C380006972A674092005F08FFB95F86300C0EB75
:10C390000010800060622179E17485F89B1095F8A7
:10C3A000B902C8B11BE000F0FE0169720027A77452
:10C3B000092005F079FBC148077067622179E174B3
:10C3C00085F89B1095F8B90210B99B2005F06CFB1D
:10C3D000A7710420E07303E09B2005F065FBE67382
:10C3E000E07CE070B648067118E530B5B14A01232B
:10C3F00053711079042801D2401C10711079AC4C93
:10C40000002504280DD90020211891F89E12022938
:10C4100001D0042900D15370401CC0B20828F3D3C6
:10C42000157194F86F1013790420994200D210719D
:10C43000D5725072A348057030BD9E4901204871E5
:10C440000879002801D0401E087199480A7990F8AF
:10C450006F00904200D208710020C87204224A7214
:10C4600098490870704710B59149002491F86B0005
:10C47000002825D191F8A903022802D2401C81F896
:10C48000A90391F8A00028B991F8A903022801D1C5
:10C4900081F8A94391F8A10030B991F8A9030128C6
:10C4A00002D1022081F8A90391F8A903022801D939
:10C4B00081F8A94391F8A91340F2A93005F0F4FAE4
:10C4C0007C48C4720421817210BD10B578490024E3
:10C4D00091F86B0000281DD191F8A90310B1401EFE
:10C4E00081F8A90391F8A00028B991F8A9030228BE
:10C4F00001D181F8A94391F8A10028B991F8A903C5
:10C50000012801D181F8A94391F8A91340F2A9307B
:10C5100005F0CAFA6748C4720421817210BD7CB567
:10C52000694843F6EF464FF6FF75007847F6196401
:10C5300001281CD0022833D0032817D1CDE900549C
:10C5400062A36C220A21012005F090FECDE900547F
:10C550005FA397220A21012005F088FECDE900564D
:10C560005CA3C2220A21012005F080FE7CBDCDE93A
:10C57000005656A36C220A21012005F077FECDE972
:10C58000005453A397220A21012005F06FFECDE944
:10C59000005450A3C2220A21012005F067FE7CBD91
:10C5A000CDE9005449A36C220A21012005F05EFE6A
:10C5B000CDE9005646A397220A21012005F056FE38
:10C5C000CDE9005443A3C2220A21012005F04EFE0A
:10C5D0007CBD7CB53C4843F6EF464FF6FF750078CE
:10C5E00047F6196401281CD0022833D0032817D13C
:10C5F000CDE9005435A36C220A21012005F036FE56
:10C60000CDE9005432A397220A21012005F02EFE25
:10C61000CDE900562FA3C2220A21012005F026FEF3
:10C620007CBDCDE9005629A36C220A21012005F02A
:10C630001DFECDE9005426A397220A21012005F012
:10C6400015FECDE9005423A3C2220A21012005F0E2
:10C650000DFE7CBDCDE900541CA36C220A210120F3
:10C6600005F004FECDE9005619A397220A21012006
:10C6700005F0FCFDCDE9005416A3C2220A210120D9
:10C6800005F0F4FD7CBD2DE9F041022006F0B0FB81
:10C69000084E114B064D308C06F11E04772825D02C
:10C6A0007D2823D070285AD0712861D0822815E0C7
:10C6B000947F0020300000201F030020E0000020B5
:10C6C000BA11002018000020F80000205345540043
:10C6D00046414E0053595300701F030851D00021AA
:10C6E00001226B2854D05E2871D07FE0772819D0C2
:10C6F00095F8610301282ED095F87E00B4F900105A
:10C70000401C81420DDD95F86E0000EBC00202EB8B
:10C71000401003EBC00090F83C00814201DD491E4F
:10C720002180C8E095F86103012813D1B4F9001005
:10C7300095F87E0081420DDD95F86E0000EBC00299
:10C7400002EB401003EBC00090F83000814201DDA5
:10C75000491E2180AFE02088401E2080ABE0218868
:10C760000A392180C9B285F8701005F09DF9A2E060
:10C7700021880A392180C9B285F8711005F094F931
:10C7800099E0B4F90000002801DD401E208092E00D
:10C79000B4F90000032802DB401E20808BE0022851
:10C7A00002D001280AD086E095F87900032801D04C
:10C7B000012801D821807EE022807CE095F8790074
:10C7C000032801D0012876D8218074E0FFE7377D67
:10C7D00067B1B4F9000095F8CF10884202DD401E21
:10C7E000208068E095F8D100208064E05D2801D1C8
:10C7F000377DD7B1572818D072281AD0652821D094
:10C8000095F86E1001EBC10707EB411103EBC10373
:10C81000A0F15F0113F81130B4F900108B424AD037
:10C82000491E2180E5283CD040E02088401E208021
:10C8300041E02088401E2080010A85F89A1085F882
:10C84000990038E0B4F9000090B1072813D001280E
:10C8500014D0082815D0042815D0052816D0032890
:10C8600017D0022818D0062818D0401E208022E0B9
:10C87000072020801FE0062020801CE00820208068
:10C8800019E0218017E00520208014E0032020809B
:10C8900011E0022020800EE022800CE004202080A5
:10C8A00009E095F85F10012900D122805F2802D1AC
:10C8B000208800B92280308C642802D1207885F845
:10C8C000640051E570B5022006F092FAFD4BFE4C73
:10C8D000FE4A188C03F11E01772804D07E2802D06E
:10C8E0005E2834D042E092F861331BB10888401CC6
:10C8F000088070BD772815D092F87D00B1F900301E
:10C90000401E8342F5DA92F86E0000EBC00202EBA3
:10C91000401004EBC00090F83F008342E9DA5B1C52
:10C920000B8070BDB1F9003092F87D008342F8DAD7
:10C9300092F86E0000EBC00202EB401004EBC00066
:10C9400090F831008342ECDA5B1C0B8070BD1D7DDA
:10C9500065B1B1F9000092F8D130984202DA401C7A
:10C96000088070BD92F8CF00088070BD02256B284A
:10C9700002D05E2819D01AE0B1F900303BB992F824
:10C980007900032801D0012801D80D8070BD92F8EC
:10C990006E0000EBC00202EB401004EBC000407ED2
:10C9A0009842F3DD5B1C0B8070BD1B7D13B37028B8
:10C9B00024D071282CD0722834D082283AD065280F
:10C9C0003FD092F86E3003EBC30505EB431304EB45
:10C9D000C304A0F15F0304EB43035C78B1F90030BA
:10C9E0009C4201D05B1C0B806428DDD1087882F862
:10C9F000640070BD0888401C088070BD0B880A3335
:10CA00000B80D9B282F87010BDE8704005F04CB8C8
:10CA10000B880A330B80D9B282F87110BDE87040E0
:10CA200005F042B80888401C0880010A993251700C
:10CA3000107070BDB1F900000228FADA401C0880BD
:10CA400070BDB1F90000062811D0072812D0A0B19E
:10CA5000082815D0012816D0022816D0032817D090
:10CA6000052818D00428EBD10620088070BD0720C7
:10CA7000088070BD0020088070BD0820088070BD4F
:10CA80000120088070BD0D8070BD0320088070BD3E
:10CA90000520088070BD0420088070BD4FF47A70B6
:10CAA0000CF040BFFCF7D4BA2DE9F05FDFF814B208
:10CAB000874E0BF11E05BBF820000127DFF814A2FA
:10CAC000824CB5F900104FF00208942806D0642873
:10CAD00009D05A465E28127D0ED00EE0C80701D15B
:10CAE0008AF8008080E094F86410642004F0DCFF91
:10CAF000287884F8640077E012B15E2820D034E012
:10CB000094F85F00022801D013286DD17248DFF835
:10CB1000CC910088081AA9F80000C1B25B2004F08B
:10CB2000C3FFB9F80000C0F307215C2004F0BCFF8C
:10CB3000B9F8000084F85B00000A84F85C0053E058
:10CB40009AB1C9B2062004F0AFFF2878A0715D4900
:10CB50002831088001226248FBF731FD6149A07944
:10CB600008700C208AF800003EE083280DD0554A5A
:10CB70001E32B2F9002002EB82025200952814D036
:10CB80009B281BD0722826D02EE0C80706D0012192
:10CB9000832004F089FF8BF8107025E002218320A8
:10CBA00004F082FF8BF810801EE0D1B2C2F30720A0
:10CBB00014F063FF0120FFF7C1FA15E0C9B28BF84A
:10CBC000131084F89B108BF804109B2004F06CFF6A
:10CBD000B770377108E02A80D1B2C2F3072014F091
:10CBE000F2FF0020FFF7AAFABBF82000B5F9001009
:10CBF000225C8A427AD021545E2802D0C9B204F065
:10CC000053FFBBF820006A2807D1297804F04CFFB5
:10CC10002878FEF7F0FDFFF745FFBBF820006E28EF
:10CC200007D1297884F86E1004F03EFF3770FFF7C3
:10CC3000F6F8BBF82000792803D1FFF733FFFFF7A0
:10CC40002DFFBBF820005F2804D1297884F85F10FD
:10CC500004F02AFFBBF820006B281AD1288804288A
:10CC600009D194F8E500012805D0394684F8E5702B
:10CC7000E52004F019FF288805280AD194F8E60079
:10CC8000012806D084F8E67094F86210E62004F0DB
:10CC90000BFFBBF82000144E4FF00009652871D13E
:10CCA000297804F001FFB5F9000030B301282FD036
:10CCB000022838D0032841D004284BD0052855D06D
:10CCC000062814E030000020701F0308947F002025
:10CCD000BA1100201F030020820200206E020020F3
:10CCE0000077000828030020BA1600200DE14AD082
:10CCF000072854D008285ED068E084F865904FF487
:10CD000016500CF0CBFC4FF41650C6F802005DE054
:10CD100084F865704FF496400CF0C0FC4FF49640D8
:10CD2000C6F8020052E084F865804FF416400CF01B
:10CD3000B5FC4FF41640C6F8020047E0032084F823
:10CD400065004FF461400CF0A9FC4FF46140C6F857
:10CD500002003BE0042084F865004FF4E1300CF061
:10CD60009DFC4FF4E130C6F802002FE0052084F866
:10CD700065004FF496300CF091FC4FF49630C6F8F5
:10CD8000020023E024E0062084F865004FF496605A
:10CD90000CF084FC4FF49660C6F8020016E0072001
:10CDA00084F865004FF496500CF078FC4FF49650E0
:10CDB000C6F802000AE0082084F865004FF46150CC
:10CDC0000CF06CFC4FF46150C6F802000CF0CAFD88
:10CDD000BBF8200083280FD12878C00706D0012196
:10CDE000832004F061FE8BF8107005E0022183209F
:10CDF00004F05AFE8BF81080BBF820006C2801D09C
:10CE00006D2825D10A216C2827D094F86D20B5F91A
:10CE1000000002EB8202B0EB420F0DDB90FBF1F061
:10CE2000401CC1B284F86D106D2004F03DFE94F8F2
:10CE30006D10022015F023F80120FFF77FF99BF811
:10CE4000110040F001008BF81100F84880F80090C4
:10CE5000BBF82000602818D01DE094F86C20B5F9CC
:10CE6000000002EB8202B0EB420FE5DB90FBF1F039
:10CE7000401CC1B284F86C106C2004F015FE94F8CC
:10CE80006C10012014F0FBFFD6E7297884F86010BD
:10CE9000602004F009FEBBF820006F280DD194F843
:10CEA0006F009BF81310884207D204218BF81310EF
:10CEB00084F89B109B2004F0F7FDBBF8200092281B
:10CEC00010D1B5F90000DA49084001281FD003202D
:10CED000B07184F892900021922004F0E5FD0420C6
:10CEE0008AF80000BBF8200082280ED1B5F90000B6
:10CEF00001281ED0022823D00021822004F0D4FD76
:10CF000084F8829009208AF80000BDE8F09F86F836
:10CF1000069084F8927013F0F7FF002019F0FEFEDF
:10CF20000121922004F0C0FD0021822004F0BCFD0C
:10CF3000D8E70121822004F0B7FD84F88270E1E790
:10CF40000221822004F0B0FD84F88280DAE770B517
:10CF500086B005F06CFFB74CB74D03AA218C6B4629
:10CF60005E2902D1207D012820D095292BD09B2934
:10CF700036D000205E3901EB810105EB81010D5CAB
:10CF800015540D18AD7A1D54401CC0B20A28F6D3B2
:10CF9000012005F02DFF694603A806F0E4F8A54935
:10CFA000208CA64A1E315E2827D037E000202918A1
:10CFB00091F84C64165491F856141954401CC0B2A0
:10CFC0000A28F4D3E4E70020291891F86064165485
:10CFD00091F86A141954401CC0B20A28F4D3D7E758
:10CFE0000020291891F87464165491F87E1419548D
:10CFF000401CC0B20A28F4D3CAE7237D73B19379E9
:10D0000092F8D150AB4201D9957104E092F8CF501B
:10D01000AB4200D2957192790A800CE0832814D03B
:10D020000A23722814D095281CD0822825D0922853
:10D0300027D0125C0A805E2805D1207D002802D10D
:10D040007F480088088006B070BD227C0A80F2E725
:10D0500012F8995F527805EB022212B292FBF3F2BA
:10D060000A80E8E792F8595292F85A2205EB022218
:10D0700012B292FBF3F20A80DDE792F882200A8076
:10D08000D9E7704A927912B100220A80D3E70122CF
:10D090000A80D0E767485E21027B002A0AD001841B
:10D0A000664991F87F10032901D19521018400215F
:10D0B000017502E001840121017548E770B5012086
:10D0C00005F096FE022005F093FE5A49088C94283C
:10D0D00001D10A7B42B10D7B00246323574A012D05
:10D0E00007D05E2816D019E05E200884012008755C
:10D0F00025E092F87F20032A02D00B840C751EE0F5
:10D10000952804D09B28F9D195200884F6E79B2028
:10D110000884F3E70D7D0DB10C7510E092F87F40A7
:10D12000042C0FD0602831D09223822830D083285D
:10D1300036D0722836D0922837D0401C0884BDE8FB
:10D14000704004E75E2806D0A0F16802022A05D2EA
:10D15000401C0884F3E769200884F0E76A2806D0B9
:10D16000A0F16C02022A05D2401C0884E7E76C207B
:10D170000884E4E7822801D10A7C22B16E28DED13E
:10D1800094200884DBE784200884D8E70B84D6E762
:10D1900092F8830010B183200884D0E70B84CEE797
:10D1A0000B84CCE776200884C9E793200884C6E77F
:10D1B0002DE9F041012005F01BFE022005F018FECC
:10D1C0001C491E4E5E22087B88B196F87F0003281A
:10D1D00001D00A8427E0088C952802D09B2803D030
:10D1E00021E09B2008841EE0952008841BE0088C29
:10D1F00000235E2805D10C7D1CB1942008840B759A
:10D2000011E05E2801D10C7DF4B196F87F70822484
:10D210008325042F1BD063283ED092283FD0762848
:10D2200045D0401E0884BDE8F04190E67B00002018
:10D230000100008030000020D41A0308947F0020F1
:10D2400068020020BA16002001200875EBE7682864
:10D2500006D0A0F16902012A05D8401E0884E2E741
:10D260000A840B75DFE76C2806D0A0F16D02012A55
:10D2700005D8401E0884D6E76A200884D3E794289E
:10D2800005D09228CFD1087C20B10D84CBE76E2049
:10D290000884C8E70C84C6E760200884C3E796F8D2
:10D2A0008300012801D00C84BDE70D84BBE7742006
:10D2B0000884B8E77CB5FB4A47F6196402F11E0101
:10D2C000108CB1F900104FF6FF75772867D012DC8B
:10D2D000A0F15E0019282DD2DFE800F03361612C47
:10D2E0002C6193F761612C2C61612C2C4E61686874
:10D2F000612C612C6100802851D009DCA0F17800FC
:10D30000082817D2DFE800F04B5D4B4B4B4B4BF935
:10D3100094285FD008DC822870D0832835D09228EA
:10D320006DD0932806D155E09B2873D0E52836D0E0
:10D33000E62834D002B02022BDE87040002005F07D
:10D3400097BD107D30B102B02022BDE870400020B2
:10D3500005F08EBDD44890F86E0030B102B0462280
:10D36000BDE87040002005F083BD02B04322BDE857
:10D370007040002005F07CBD41B1CDE90054CBA345
:10D38000C2220021012004F071FF7CBDCDE90054D0
:10D39000C8A3C2220021012004F068FF7CBD02B0B6
:10D3A0002022BDE87040002005F062BD0A2091FBFC
:10D3B000F0F002B001B2BDE870402022002005F07C
:10D3C00057BDCDE90054BDA3C2220021012004F0C5
:10D3D0004DFF7CBDC80708D0CDE90054B8A3C222D8
:10D3E0000021012004F042FF7CBDCDE90054B5A32B
:10D3F000C2220021012004F039FF7CBD46E065E037
:10D4000008E0CDE90054B0A3C2220021012004F0BD
:10D410002DFFF2E70529F0D2DFE801F0030C151E1D
:10D420002700CDE90054AAA3C2220021012004F064
:10D430001DFFE2E7CDE90054A6A3C222002101208E
:10D4400004F014FFD9E7CDE90054A4A3C2220021BF
:10D45000012004F00BFFD0E7CDE90054A1A3C222C4
:10D460000021012004F002FFC7E7CDE900549FA38B
:10D47000C2220021012004F0F9FECDE900549BA353
:10D48000C2220021012004F0F1FEB6E701290AD0F2
:10D49000022911D0CDE9005496A3C2220021012017
:10D4A00004F0E4FEA9E7CDE9005494A3C2220021D0
:10D4B000012004F0DBFEA0E7CDE9005491A3C222D5
:10D4C0000021012004F0D2FE97E71DE08F480140C3
:10D4D000012909D0CDE900548DA3C22200210120E9
:10D4E00004F0C4FE89E708E0CDE900548AA3C22213
:10D4F0000021012004F0BAFE7FE702B02022BDE83F
:10D5000070405A2005F0B4BCC1B101291FD00229D6
:10D5100026D003292DD0042934D005293BD0062953
:10D5200042D0072949D008298CD1CDE900547CA3E9
:10D53000C2220021012004F099FE5EE7CDE90054EB
:10D5400079A3C2220021012004F090FE55E7CDE925
:10D55000005477A3C2220021012004F087FE4CE78B
:10D56000CDE9005474A3C2220021012004F07EFE04
:10D5700043E7CDE9005472A3C2220021012004F048
:10D5800075FE3AE7CDE900546FA3C22200210120C5
:10D5900004F06CFE31E7CDE900546DA3C2220021F6
:10D5A000012004F063FE28E7CDE900546AA3C222FB
:10D5B0000021012004F05AFE1FE7CDE9005468A3C2
:10D5C000C2220021012004F051FE16E770B5664D1D
:10D5D000354C0026297894F87F000939122951D258
:10D5E000DFE801F0090C505015180F1B12202550D0
:10D5F0003F4245484B4EFEF7F1FD43E0FEF756FE35
:10D6000040E0FEF7F2FE3DE0FEF717FF3AE0FEF7DE
:10D6100086FF37E0FEF7DDFF34E0052832D0FEF765
:10D6200022FF2FE005282DD0FEF74FFF2AE005F05E
:10D63000FEFBFFF72FFD94F87F001A4C40B1042841
:10D6400006D0022808D0032806D0052804D019E007
:10D650002673FFF71FFD15E0FFF71CFD0120207367
:10D6600010E0FFF72BFD0DE0FFF7A2FD0AE0FFF74A
:10D6700029F907E0FFF707F804E0FFF715FA01E0E2
:10D68000FFF712FA2E7070BD00218438374A072840
:10D6900079D2DFE800F0046D716F737577009188BF
:10D6A00071E0000030000020947F00202D462D20E6
:10D6B000000000002D432D20000000003441000038
:10D6C0004E4F0000594553003130302020000000FB
:10D6D0004F6666004D6F6465310000004D6F6465F4
:10D6E000320000004D6F6465330000004175746FB7
:10D6F0000000000052533438350000005A494742B8
:10D7000045450000204155544F00000001000080B5
:10D710004D4F4442555300004241434E4554000092
:10D7200031343430302000003936303020200000D1
:10D7300031393230302000003338343030200000AE
:10D74000353736303020000031313532303020006E
:10D7500037363830302000003132303020000000C1
:10D76000343830302000000000010020B0110020CB
:10D77000917908E0117A06E0D17904E0117802E0AD
:10D78000517800E0917808B2704710B503F0EFFFD0
:10D79000802004F066F804F017F808B1002010BDEE
:10D7A000FE2004F05EF804F00FF808B1002010BD70
:10D7B00003F0F3FF012010BD10B5044603F0D7FFBE
:10D7C000802004F04EF803F0FFFF08B1002010BDE8
:10D7D0003CB1F52004F045F803F0F6FF28B1002035
:10D7E00010BDF32004F03DF8F6E703F0D6FF01206A
:10D7F00010BD70B50E4603F0BAFF812004F031F879
:10D8000003F0E2FF012004F04DF84FF6FF7101EA4A
:10D810000025012004F046F840EA0504002004F049
:10D8200041F803F0BAFF3480012070BD01F002031B
:10D83000834201D00020704721F0030150B140F233
:10D84000E2404143C81701EB104000143C381080FF
:10D850000120704744F2A4404143C81701EB104037
:10D860000014A0F590504D3800B20A2190FBF1F061
:10D870001080EDE770B5054603F079FF812003F0D5
:10D88000F0FF03F0A1FF08B1002070BD012004F0FB
:10D8900009F84FF6FF7101EA0024012004F002F8B4
:10D8A000204484B2002003F0FDFF03F076FF022D38
:10D8B0000AD044F2A4404443FA480A2100EB244031
:10D8C00090FBF1F080B270BD40F2E24044436FF053
:10D8D0003B0000EB2440F5E710B503F048FF802043
:10D8E00003F0BFFF03F070FF08B1002010BDE72078
:10D8F00003F0B7FF03F068FF08B1002010BD03F08C
:10D9000036FF812003F0ADFF03F05EFF08B1002079
:10D9100010BD002003F0C6FF044603F03EFFE0B256
:10D9200010BD70B50646C1F1FA0023F0BAF94FF008
:10D930003332DD4B23F008FA04460D46304623F01F
:10D94000B0F922462B4622F02DFF23F07BF900B2DE
:10D9500070BD2DE9F0470446084623F0EBFDD3499E
:10D9600023F0B6FC23F01AFC22F002FD22F0E8FEC0
:10D970000646204623F095F9CD4F0D460446002279
:10D980003B4623F0E1F922F0DBFE8146DFF82483F9
:10D99000DFF824A3204629464246534622F002FFE0
:10D9A00004460D46484623F0F9FB22462B4622F05A
:10D9B000B5FF22F0C5FE0146304623F01BFC23F0E4
:10D9C000EDFB8946064600223B4623F0F1FA044669
:10D9D0000D46304649464246534623F0B5F92246A5
:10D9E0002B4622F09BFF23F02DF900B2BDE8F08713
:10D9F00063214FF4607004F057B8B0498A889207E9
:10DA00000BD08A790D2A15D2DFE802F014393B3E9B
:10DA10004144474A4D5053575B008A790D2A09D239
:10DA2000DFE802F00807090C0F1215181B1E21254C
:10DA30002900C8797047C8791F307047C8793B30D2
:10DA40007047C8795A307047C87978307047C879BC
:10DA500097307047C879B5307047C879D43070476F
:10DA6000C879F3307047C87900F211107047C8794F
:10DA700000F598707047C87900F5A7707047C879AD
:10DA80007047C8791F307047C8793C307047C879F3
:10DA90005B307047C87979307047C87998307047E3
:10DAA000C879B6307047C879D5307047C879F43036
:10DAB0007047C87900F589707047C87900F2311055
:10DAC0007047C87900F24F10704700B5FFF795FF17
:10DAD0007B498883C0F3C70200F0070179481044EE
:10DAE00000F22D40FDF75EF908B1012000BD0020D5
:10DAF00000BD2DE9F043734D714901266A7A724FDA
:10DB0000CB7C4FF0040C02F0FE044FF00008052817
:10DB10000FD2DFE800F00E03101E2100CE7342F09A
:10DB2000010068728E7481F813C081F804C0BE7160
:10DB3000BE70BDE8F08381F80FC06C7281F812806E
:10DB4000002BF6D081F8138081F80480BE71BE707E
:10DB5000EFE70A20C873ECE70C20C8736C7281F8F9
:10DB60001280002BE5D081F8138081F80480BE710B
:10DB7000BE70DEE710B5514A147A002C03D0127A39
:10DB8000012902D002E00722FAE708224D490728BE
:10DB90003AD2DFE800F039040D161F283100521E7A
:10DBA00002EB4200084490F8150400F007032BE054
:10DBB000521E02EB4200084490F81504C0F3C20361
:10DBC00022E0521E02EB4200084490F8160400F0D6
:10DBD000070319E0521E02EB4200084490F81604B5
:10DBE000C0F3C20310E0521E02EB4200084490F85A
:10DBF000170400F0070307E0521E02EB420008443E
:10DC000090F81704C0F3C20358B210BD2DE9FC5FB1
:10DC1000002613F079F92948007AE0B32748007A02
:10DC2000401E00F0FF09FFF750FF2849284ADFF89F
:10DC300094E000287ED00EF2094003784478C3EBCC
:10DC4000031304EB83030B808378C478C3EB0313C3
:10DC500004EB83034B8003794479C3EB031304EB98
:10DC600083038B808379C479C3EB031304EB8303B1
:10DC7000CB80037A447AC3EB031304EB83030B8159
:10DC8000C37A807AC0EB001003EB80004881002447
:10DC900009EB490800E01DE002EB4807385DFF286A
:10DCA0001BD051E0B3EDFFFF3333C3BF00007A4414
:10DCB00000A03140CDCCCCCCCCFCA240B011002097
:10DCC00030000020947F0020BA1100206C09002051
:10DCD0001C8400204FF00609A5E7FF484FF6FF71AE
:10DCE00020F8141008EB5400FC4A019010440090F6
:10DCF00090F81504E10741D0C10801F0030119B300
:10DD0000E1073ED000F0C70AFF2109EB490080007F
:10DD100000EB440B0BEB020080F8B51380F8B61350
:10DD20000BF2B53003F0C0FE0BF2B630FF2103F06A
:10DD3000BBFE00E0D9E0009880F815A40198514698
:10DD400000F2154003F0B0FE641CE4B2062CA5D32B
:10DD5000DFF88C9399F80000E8B30020DE4901F168
:10DD60000E0231F8103022F81030401CC0B20628E4
:10DD7000F7D305244FF0000C00201FE000F0030152
:10DD8000BDE700F0F80ABFE7411C32F8103032F866
:10DD900011A0534511D90126938132F8113022F890
:10DDA0001030938922F8113017F800A03B1893F82F
:10DDB00001B007F800B083F801A0C8B2A042E3D3D5
:10DDC000641EE4B20CF1010C0CF0FF0CBCF1060F68
:10DDD000D2D3002000E001E089F80000CEB3002497
:10DDE000BE4E08EB5402931993F81514E00706D0C1
:10DDF000385D012817D0D8B1FF281ED01FE0385D4C
:10DE0000012803D038B1FF280AD018E001F0F8004B
:10DE100040F0010113E001F0F80040F002010EE0D3
:10DE200001F0F8010BE001F0C70040F0080106E046
:10DE300001F0C70040F0100101E001F0C70183F8D4
:10DE4000151402F2154003F02FFE641CE4B2062CF8
:10DE5000C7D3A44841780078C0EB001001EB8004E0
:10DE60009D4E0E363088A04207D87088A04204D953
:10DE700001210846FFF77EFEC5B27088A04207D890
:10DE8000B088A04204D901210220FFF773FEC5B279
:10DE9000B088A04207D8F088A04204D9012103200D
:10DEA000FFF768FEC5B2F088A04207D83089A042CB
:10DEB00004D901210420FFF75DFEC5B23089A042DC
:10DEC00007D87089A04204D901210520FFF752FE2E
:10DED000C5B27089A04204D801210620FFF74AFE8E
:10DEE000C5B22846BDE8FC5F03E609EB49070EEB27
:10DEF000870000F2B53003784478C3EB031304EBDA
:10DF000083030B808378C478C3EB031304EB830390
:10DF10004B8003794479C3EB031304EB83038B80B9
:10DF20008379C479C3EB031304EB8303CB80037AB7
:10DF3000447AC3EB031304EB83030B81C37A807A27
:10DF4000C0EB001003EB80004881002002EB470487
:10DF5000225CFF2A19D0401CC0B20628F8D3DFF893
:10DF6000808198F80000E0B30020DFF86CB10BF17D
:10DF70000E0B31F810202BF81020401CC0B20628E0
:10DF8000F7D305220023002121E05548807CBDE81D
:10DF9000FC5FAEE5481C3BF811C03BF81090CC4547
:10DFA00014D90126ABF80CC03BF810C02BF811C0F7
:10DFB000BBF80CC02BF810C014F8019004EB010C56
:10DFC0009CF801A004F801A08CF80190C1B2914224
:10DFD000E0D3521ED2B25B1CDBB2062BD3D300209F
:10DFE00000E001E088F80000D6B30026F14607EB18
:10DFF000560202EB090393F81514F00706D0A05D52
:10E00000012817D0D8B1FF281ED01FE0A05D01283D
:10E0100003D038B1FF280AD018E001F0F80040F032
:10E02000010113E001F0F80040F002010EE001F000
:10E03000F8010BE001F0C70040F0080106E001F034
:10E04000C70040F0100101E001F0C70183F815148A
:10E0500002F2154003F028FD761CF6B2062EC6D358
:10E06000204841780078C0EB001001EB80041A4E84
:10E070000E363088A04207D87088A04204D900210B
:10E080000120FFF777FDC5B27088A04207D8B0889D
:10E09000A04204D900210220FFF76CFDC5B2B08870
:10E0A000A04207D8F088A04204D900210320FFF73E
:10E0B00061FDC5B2F088A04207D83089A04204D9DA
:10E0C00000210420FFF756FDC5B23089A04210D8C8
:10E0D0007089A0420DD907E06C090020947F0020D0
:10E0E00030000020B011002000210520FFF742FD84
:10E0F000C5B27089A04204D800210620FFF73AFD7E
:10E10000C5B22846FFF7F5FC98F80200854204D016
:10E110001E49012008718870487088F80250BDE8D7
:10E12000FC9FF0B503461A481A4CC51895F86702CB
:10E13000FF2824D0002658B1411E012705290BD203
:10E14000C9B21548FCF72EFE012803D0E65416E0AC
:10E15000E65414E0E75412E01049062806D1B1F95C
:10E160000020002A01DDE75400E0E654072806D12C
:10E17000B1F90200002801DDE75400E0E65495F80B
:10E180006702002801D16420E054F0BDBA110020DC
:10E19000947F0020880900209E020020C6000020F5
:10E1A0002DE9F041FC4C0023A370E370FC4D3C24AE
:10E1B000FA4F182605EB8203002904D0012939D033
:10E1C000022968D157E0B0FBF4F104FB110197F884
:10E1D00002C06144C9B2B1FBF4FCB1FBF4F804FB2A
:10E1E0001811D970B0FBF4F104FB1101401A80B290
:10E1F000B0FBF4F0B0FBF4F104FB1101614497F8BB
:10E2000001C06144C9B2B1FBF4FCB1FBF4F804FBFA
:10E2100018119970B0FBF4F0397860440844C0B22A
:10E22000B0FBF6F1B0FBF6F406FB1400587005F8ED
:10E23000221030E0B978D970B0FBF4F104FB110181
:10E2400097F801C06144C9B2B1FBF4FCB1FBF4F82A
:10E2500004FB18119970B0FBF4F03978604408445D
:10E26000C0B2B0FBF6F1B0FBF6F406FB1400587038
:10E2700005F822100FE0B978D9707978997039785B
:10E280000844C0B2B0FBF6F1B0FBF6F406FB140094
:10E29000587005F82210D8783B2801D13A20D87060
:10E2A000BDE8F08110B5BC4BBD49BC4A002814D074
:10E2B00011F82040DB789C422FD101EB80001378CD
:10E2C0004178994227D181785378994221D1C078F9
:10E2D000917888421BD8012010BD08789B7898421D
:10E2E00013D14878137898420DD1887853789842A2
:10E2F00007D1C8789178884201D8012010BD00204C
:10E3000010BD002010BD002010BD002010BD002059
:10E3100010BD002010BD002010BD002010BD2DE953
:10E32000F14FDFF8748298F80C0001285AD10024CC
:10E33000814608F13E0B4FF0000A08F11A06994F8A
:10E340004DE0651CE8B2FFF7ADFF012801D1315D5A
:10E3500011B101282CD041E097F8DB00032813D03D
:10E3600017F8CB0F797800EB012080B2A8F82400D1
:10E3700006F80490397ACB3F0122FFF711FF97F896
:10E38000DB0002280DD029E006F80490EAB23BF841
:10E3900014000021FFF704FF7F483B3000F8049091
:10E3A000EDE706F804A088F80AA088F80CA015E0AC
:10E3B000305D012812D197F8DB00032814D017F83C
:10E3C000CD0F797800EB012080B2A8F8240006F880
:10E3D00004A0B979CD3F0122FFF7E2FEECB200982C
:10E3E0008442AED3BDE8F88F6B48423030F8140059
:10E3F00030B106F804A0EAB20021FFF7D1FEEDE744
:10E4000006F80490EAB23BF814000021FFF7C8FEBA
:10E41000E4E7D21C884205D1D1B25F48002218300F
:10E42000FCF7B3BCD1B25C4801221830FCF7ADBC9C
:10E4300010B50446002903D0574900203231085551
:10E440005548012221461830FCF79FFCE41CE1B23C
:10E4500051480022BDE810401830FCF796BC10B5BA
:10E4600004464D482630015D4F48005D821C9142B4
:10E470000DD94948002221461030FCF786FC214680
:10E4800045480122BDE810401230FCF77EBC801EDA
:10E4900081420DDA4048012221461030FCF775FC1C
:10E4A00021463D480022BDE810401230FCF76DBC0B
:10E4B0003948002221461030FCF767FC21463648D7
:10E4C0000022BDE810401230FCF75FBC2DE9F04F90
:10E4D00089B00446334EDFF8C09096F86B000028F0
:10E4E00007D0012844D0314F02287ED0032810D114
:10E4F000AAE099F8050006280CD096F8A90302288E
:10E5000015D0012813D02046FFF7A9FF0120FFF7FF
:10E51000A6FFC1E02048012200211030FCF735FCA5
:10E520001D48002211461230FCF72FFCB4E00120F8
:10E53000FFF795FF96F8A90302280CD01648012290
:10E5400000211030FCF721FC134800221146123044
:10E55000FCF71BFCDAE71048002211461030FCF7EC
:10E5600014FC0D48012200211230FCF70EFCCDE70F
:10E570000120FFF774FF99F80400C8B10648002293
:10E5800011461030FCF701FC034801220021123033
:10E59000FCF7FBFB17E028E07A000020B011002018
:10E5A00091090020947F0020D3030020DC03002089
:10E5B00001220021FE48FCF7E8FBFD48002211463D
:10E5C000801CFCF7E2FB99F80B0070B3401E89F841
:10E5D0000B0000221146F648FCF7D7FBF448002256
:10E5E0001146801CFCF7D1FB56E096F89F020528E7
:10E5F00004D096F89E02052807D00AE07888012802
:10E6000001D0002505E0012503E0388801280DD060
:10E6100000256DB100221146E548FCF7B6FBE44841
:10E6200001220021801CFCF7B0FB35E00125F0E75A
:10E6300001220021DE48FCF7A8FBDD48002211463C
:10E64000801CFCF7A2FB27E00221DA48FCF7AAFBBA
:10E6500010B9012089F8070096F89F02052804D018
:10E6600096F89E02052807D00AE07888012801D094
:10E67000002505E0012503E0388801285DD000254C
:10E68000F5B301220021CA48FCF77FFBC8480022ED
:10E690001146801CFCF779FBA020A0EB4407C5487D
:10E6A000C349D438C44AC05D253104EB440B02EBA6
:10E6B0004B08002628B3062856D010F80800085545
:10E6C000C81C12F81B200255DFF8E4A20AF1160A52
:10E6D0000AF10F011AF80400095D0AF109058842E0
:10E6E00004D305F10901095D884224D9B148D43821
:10E6F00090F87900022801D004283DD8214601E095
:10E700001DE028E0B9F81200FCF72EFB30B1A84854
:10E710001AF804102830005D81420CD32146B9F864
:10E720001000FCF721FB38B3A1481AF8041025307B
:10E73000005D814220D92E5569E10125A0E7002224
:10E7400011469B48FCF721FB994801220021801CBF
:10E75000FCF71BFBA0E79648642228300255964838
:10E7600010F81B000855AFE70E55934810F81B2012
:10E770008F4828300255A7E72146B9F81000FCF76A
:10E78000F3FAD0B30021A1208A4AA0EB4400D43A86
:10E79000DFF824E2105C05AB08E0D25D01EB4B0C26
:10E7A000724412F80C205A54491CC9B2814AD43A16
:10E7B0008842F2D80022C0F1060C06E003EB020BFF
:10E7C000022100F80B10521CD2B29445F6DC1AF864
:10E7D00004004FF0030E032802D802460AF804E0B2
:10E7E0001AF804009DF819C0CDF820C0ACF1020C55
:10E7F000604503DA062129551BE06FE09DF81410EF
:10E80000884201D92E5514E0002103EB010B9BF83F
:10E8100001B0584509D913F801B0ABF1020B5845C6
:10E8200003DA01F1010B05F804B0491CC9B204294F
:10E83000EBD39DF814108B1E984207DB884205D855
:10E84000295D012902D009B1012129559DF8151032
:10E850008B1E984208DB884206D8295D012903D027
:10E86000022901D0022129559DF816108B1E9842CD
:10E8700008DB884206D8295D022903D0032901D08C
:10E8800005F804E09DF817108B1E984208DB8842BB
:10E8900006D8295D032903D0042901D00421295574
:10E8A0009DF818108B1E984208DB884206D8295D17
:10E8B000042903D0052901D005212955604509DB2C
:10E8C0000899884206D8295D052903D0062901D078
:10E8D00006212955032801D10AF804202146B9F858
:10E8E0001200FCF741FAE8B30020324905AAD439F6
:10E8F000C95D04E018F800301354401CC0B28142D6
:10E90000F8D800206623C1F1060705E002EB000CF1
:10E9100001F80C30401CC0B28742F7DC9DF819703A
:10E920001AF8040007F1020C604502D90C212955A0
:10E9300014E09DF81410884201D22E550EE00021FB
:10E9400053185B78984205D2535C9B1C984201D9BE
:10E95000CB1D2B55491CC9B20429F1D39DF81410C5
:10E96000884200E053E008D3891C884205D8295D1D
:10E97000072902D009B1072129559DF815108842B1
:10E9800009D3891C884206D8295D072903D00829A4
:10E9900001D0082129559DF81610884210D3891CF2
:10E9A00088420DD8295D08290AD0092908D005E038
:10E9B0008A000020688000209D0900200921295537
:10E9C0009DF81710884209D3891C884206D8295D12
:10E9D000092903D00A2901D00A2129559DF81810C8
:10E9E000884209D3891C884206D8295D0A2903D0A8
:10E9F0000B2901D00B212955B84208D3604506D810
:10EA0000285D0B2803D00C2801D00C202855FE4F80
:10EA10000DF11C0A385D0AF804002146B9F8180007
:10EA2000FCF7A2F978B12146B9F80E00FCF79CF981
:10EA300048B9385DB8B1401C3855F348002221462A
:10EA40001A38FCF7A2F904F1030808F0FF01B9F83D
:10EA50001800FCF789F970B32146B9F80E00FCF7ED
:10EA600083F9D8B127E0285D062805D92146B9F8F1
:10EA70001600FCF779F970B1285D401E0628DCD23B
:10EA80002146B9F81400FCF76FF90028D5D1385D9C
:10EA9000401C3855D1E707203855CEE7385D0728A8
:10EAA00015D008B1401E3855D74808F0FF010022A4
:10EAB0001A38FCF76AF9285D0D286ED2DFE800F0FD
:10EAC0006D091E3A586E8BA4B8D5F6EFEE003E5590
:10EAD000EAE7385D401E06280BD2CB4800222146CB
:10EAE0001A38FCF752F9385D22460121FFF791FCF4
:10EAF0002EE101212046FFF79BFC29E1385D811EB4
:10EB000005290BD2C048002221461A38FCF73DF9EE
:10EB1000385D22460221FFF77CFC19E1012804D070
:10EB200001212046FFF784FC12E100212046FFF777
:10EB30007FFC0DE1385DC11E04290BD2B2480022D2
:10EB400021461A38FCF721F9385D22460321FFF7E8
:10EB500060FCFDE0022806D0012804D001212046F7
:10EB6000FFF766FCF4E000212046FFF761FCEFE0D0
:10EB7000385D011F03290BD2A348002221461A3811
:10EB8000FCF703F9385D22460421FFF742FCDFE081
:10EB900001212046FFF74CFCDAE0C0E0385D411F60
:10EBA00002290BD29848002221461A38FCF7EDF8CA
:10EBB000385D22460521FFF72CFCC9E0401E0328E2
:10EBC00004D800212046FFF733FCC1E00121204694
:10EBD000FFF72EFCBCE0385D062807D0401E042855
:10EBE0000DD800212046FFF723FCB1E08648002223
:10EBF00021461A38FCF7C9F806203855A8E001214B
:10EC00002046FFF715FCA3E0385D06280BD97E48A7
:10EC1000002221461A38FCF7B8F8385D2246072151
:10EC2000FFF7F7FB94E001212046FFF701FC8FE09E
:10EC3000385D07280DD974484FF000022146A0F135
:10EC40001A00FCF7A2F8385D22460821FFF7E1FB25
:10EC50007EE005D14FF000012046FFF7E9FB77E0A9
:10EC600001212046FFF7E4FB72E0385D08280DD94A
:10EC700065484FF000022146A0F11A00FCF785F824
:10EC8000385D22460921FFF7C4FB61E009D007285F
:10EC900007D001212046FFF7CBFB59E02EE019E019
:10ECA00004E000212046FFF7C3FB51E0385D09284E
:10ECB0000BD95548002221461A38FCF766F8385D12
:10ECC00022460A21FFF7A5FB42E000212046FFF77C
:10ECD000AFFB3DE0385D0A280BD94B4800222146A6
:10ECE0001A38FCF752F8385D22460B21FFF791FBEA
:10ECF0002EE000212046FFF79BFB29E0385D0B2822
:10ED000008D94148002221461A38FCF73EF80C2069
:10ED100038551DE000212046FFF78AFB18E03A48ED
:10ED2000002221461A38FCF730F8385D38B13648F1
:10ED300008F0FF0101221A38FCF727F808E0285DE7
:10ED40003855314808F0FF0100221A38FCF71DF849
:10ED50001AF80400395D884219D02B490120093185
:10ED60000870487088702848012221462438FCF732
:10ED70000CF80A2089F800000220CDE9000602966E
:10ED80000023642221A12448039609F0C2FF385DC4
:10ED900030BB1AF80400DFF87080411EA8F10608A5
:10EDA000A8F1030A06291CD2DFF870B09BF86600B0
:10EDB00048B101222146A8F11800FBF7E6FF9BF8B5
:10EDC000660008F804009BF8670048B10E4801226D
:10EDD00021461C38FBF7D9FF9BF867000AF80400AE
:10EDE0002AE0072828D3DFF834B09BF8660048B142
:10EDF0000548012221461C38FBF7C7FF9BF8660037
:10EE00000AF804000CE00000AC00002053746174A8
:10EE100065537769746368008FAC0008947F0020A5
:10EE20009BF8670040B101222146F948FBF7ADFF8E
:10EE30009BF8670008F8040099F8010000280ED13B
:10EE4000A9F81860A9F81460A9F8166028780728AE
:10EE500000D32E70285D3855012089F8010009B0D3
:10EE6000BDE8F08F2DE9FF4F81B081464D4600246B
:10EE7000DFF8A083DFF898B308F1D6000BF1270B79
:10EE8000A246009084B198F8CD0098F8CE1000EB1F
:10EE90000126049800F00F010398052919D2DFE834
:10EEA00001F00D0F1113170098F8CB0098F8CC1053
:10EEB00000EB0126029801094846EEE7002508E02C
:10EEC000642506E0054604E0322101EB500500E030
:10EED0004508CF4808300555002739460098FBF70C
:10EEE00061FF012807D108EB070090F8B91003294A
:10EEF00001D190F88B511CB17F1CFFB2052FECD3D0
:10EF000098F8D310012902D0022904D006E0C6EBFC
:10EF10000610860002E04FF461604643642206FB5F
:10EF200005F0B0FBF2F0BA4F80B22A3727F8140090
:10EF3000C5F164037343B3FBF2F23B1D23F81420C5
:10EF400088B185B11BF80420012A0CD1A3F142023B
:10EF500001261673621CD2B2FFF722F9A7F1240032
:10EF600006550BF804A037F8140000B11DB9A848E5
:10EF7000801D00F804A0641CE4B2022C82D305B00A
:10EF80006EE72DE9F34F81B00027DFF884A2DFF8A8
:10EF90008892DFF880B20AF11E0A0BEB070000909E
:10EFA00010F8B74F007B072814D002987900005D55
:10EFB000C84000F00300022C0ED24FF0A001A1EBDC
:10EFC00044011BF801604FF0A101A1EB44011BF8C3
:10EFD000018006E00198EEE703D19BF89C609BF866
:10EFE0009D808E49097801290CD19BF8B710012921
:10EFF00001D107B902209BF8B810012902D1012FD5
:10F0000000D1022030B101287ED0022804D003288C
:10F0100001D164E00025CDE07D487D4912302131E9
:10F02000005D095D884235D216B91AF80410E9B1BD
:10F030001AF8041004EB4405494406EB4502114458
:10F0400011F8011C081A4FF47A71FBF78BFE09EBDB
:10F05000450106EB0802114411F8011C90FBF1F583
:10F060004FF47A70854200D90546A3E004EB4405CD
:10F0700008EB4501494411F8011C081A4FF47A7154
:10F08000FBF770FE09EB4501414411F8011C90FBB0
:10F09000F1F5E5E75E492431095D88421DD91AF88A
:10F0A000041004EB44056FF00602494402EB4502EC
:10F0B000895C401A4FF47A71FBF754FE09EB450165
:10F0C000314411F8011CC1F1640190FBF1F5B5F573
:10F0D0007A7F6FD94FF47A756CE000256AE04C486E
:10F0E0004B4912302131005D095D884239D20EB39F
:10F0F0001AF8041004EB4405494406EB4502114498
:10F1000011F8011C081A00E052E04FF47A71FBF785
:10F1100029FE09EB450106EB0802114411F8011C18
:10F1200090FBF1F505F5FA754FF47A70854241D9F7
:10F1300005463FE01AF8041004EB4405494408EB87
:10F140004502114411F8011C081A4FF47A71FBF7BB
:10F1500009FE09EB4501414411F8011C90FBF1F552
:10F16000E0E72B492431095D88421FD91AF80410C1
:10F1700004EB44056FF00602494402EB4502895C4A
:10F18000401A4FF4FA71FBF7EDFD09EB45013144EC
:10F1900011F8011CC1F1640190FBF1F505F5FA7558
:10F1A0004FF47A70854205D9054603E0002501E059
:10F1B0004FF47A75009890F8C300072830D0029871
:10F1C0004021B940005D084000B311481049123099
:10F1D0002131005D095D88423BD2C6B11AF80410A6
:10F1E00004EB4404494406EB4402114411F8011CA9
:10F1F000081A4FF4FA71FBF7B5FD09EB440108EB6F
:10F200000602114411F8011C90FBF1F545E009E0FC
:10F210008E000020947F00209D09002048020020DD
:10F220000020D1E71AF8041004EB4404494408EB29
:10F230004402114411F8011C081A4FF47A71FBF7CB
:10F2400091FD09EB4401414411F8011C90FBF1F5DB
:10F2500023E0F749095D88421ED91AF8041004EB2F
:10F2600044056FF00602494402EB4502895C401AEE
:10F270004FF4FA71FBF776FDA021A1EB44014FF0AA
:10F28000FF321BF8011002EB45024944895CC1F1D1
:10F29000640190FBF1F500E000254FF47A7085429F
:10F2A00000D90546009890F87B0011280DD002285F
:10F2B00017D003281FD004282FD0284622F052F957
:10F2C000DC497A1D01EB821148627F1CFFB2022FDC
:10F2D000FFF463AE9BF8C3000022D749022826D072
:10F2E00027E0680822F03EF90146D24A781D02EB79
:10F2F00080104162E9E705EB85000621B0FBF1F0E3
:10F30000C83022F02FF9CB497A1D01EB82114862F7
:10F31000CA4A9042D9DD4A62D7E7C5F57A7022F031
:10F3200021F9C4497A1D01EB82114862CDE70B88AF
:10F330001BB1032804D1488810B9BE48C0F8642125
:10F340009BF8C400022801D10B8823B1032805D102
:10F350004888002802D1B748C0F8A421BDE8FE8F34
:10F3600030B5B749062813D091F87C10B44A4C1F29
:10F37000642392F85E0392F85D23801A0C2C32D23B
:10F38000DFE804F009111919191919191919222698
:10F3900091F87B10EAE7AB49B1F90010484390FBC4
:10F3A000F3F000B230BDA849B1F90010484390FB1A
:10F3B000F3F000B230BDA04AC91F32F91110484322
:10F3C00090FBF3F000B230BDA048B0F9000030BDB2
:10F3D0009F49098809B2891A4FF47A72514391FB07
:10F3E000F0F000B230BD002030BD2DE9F04F8BB001
:10F3F0000025019597489949914F02789648002A2F
:10F4000006D097F86C20028097F86D00088005E020
:10F4100097F87120028097F8700008800024204639
:10F42000FFF754F8641CE4B2032CF8D38048DFF8EB
:10F4300000A23838AAF1060A007A01280BD197F801
:10F44000A0008AF8000097F8C800C0EB0010810007
:10F45000AAF1320041847A499AF8000001F51C7241
:10F46000734E01F5B0710E36CDE90912DFF8F09157
:10F47000DFF8F0B1A6F12008062828D899F8001086
:10F48000C319C1EBC10202F203129A5C3280D1B1FE
:10F490000999415C059117F8A01F084498F80010DD
:10F4A00010F80B00401A6421FBF75CFC797817F820
:10F4B000A029114411F80B1090FBF1F0C4B2642C98
:10F4C0002ED964242CE00A99415C0591E3E799F870
:10F4D0000010C1EBC102131897F8A120C2F1060277
:10F4E0009B1A3B4493F803313380E9B3811A3944C2
:10F4F00091F8601105915B4998F80020891F405CE4
:10F500006421101AFBF72EFC97F8A01011F80B10CD
:10F51000C1F1640190FBF1F0C4B2642C00D9642401
:10F520004348DFF840A1801F0AF1060A4078062808
:10F5300032D899F8001041B34B49415C7180099968
:10F54000415C039117F89E1F084498F8011010F8C9
:10F550000A00401A6421FBF705FC797817F89E2908
:10F56000114411F80A1000E009E090FBF1F000F0FE
:10F57000FF0BBBF1640F35D94FF0640B32E0811AF9
:10F58000394491F870120591B5E73849415C7180B2
:10F590000A99415C0391D5E799F80010F1B397F807
:10F5A0009F10C1F10601411A394491F82621728059
:10F5B00091F86011039198F8011010F80B00081AE7
:10F5C0006421FBF7CFFB97F89E1011F80A10C1F1E8
:10F5D000640190FBF1F000F0FF0BBBF1640F01D967
:10F5E0004FF0640B12481F49801F0C31807808913E
:10F5F00006284ED899F80010C9B11C493331415C36
:10F60000B18017F89C1F01440898085C98F8021014
:10F61000401A6421FBF7A6FB387800E028E07978EF
:10F620009C3F01440898085CB4FBF0F04DE02CE0EE
:10F63000B20000207C8400203C12002000007A44AC
:10F64000947F0020680200205C00002066020020F9
:10F650006202002042000020D8030020DA030020CC
:10F66000430000209C090020BA8000207382002003
:10F6700097F89F10C1F10601411A394491F8DF2231
:10F68000728091F87012039195E7FC49415CB1805A
:10F69000B7E799F8001041B397F89D10C1F1060142
:10F6A000411A394491F81213B18098F8021010F8F9
:10F6B0000A00081A6421FBF755FB97F89C2008996B
:10F6C000515CC1F1640190FBF1F097F8DB00DFF8C9
:10F6D000B0A3C0B30121002002AA052816DA3B1806
:10F6E00093F8B930032B0AD019E097F89D10C1F1B7
:10F6F0000601411A394491F82013B180D5E7012958
:10F7000002D0012150540AE00021FBE73B1893F896
:10F710007630112B03D1012965D001215054401CB2
:10F7200000B20728D9DB9DF808001AF80000E8B3FA
:10F730009DF809001AF80000C8B3039B5A46194601
:10F740005846FFF78FFB0024DFF834B34FF0010A6F
:10F750000BF1070BCA48005D032861D004286BD069
:10F760000BF804001BF80400214636F81000FBF7E4
:10F77000FBFA0246C24821463238FBF706FB641CFE
:10F78000E4B2072CE6D3BE48BE4E52388079C0B3EF
:10F79000BB48523890F8200001900024381990F8A6
:10F7A000B90001280DD002280BD001E01DE030E0A7
:10F7B000214601A8FBF7F6FA21F0D4FE06EB8411EE
:10F7C0004862641CE4B2052CE8D301210020DFF874
:10F7D000B0B2ABF1380B052860D23A1892F8B920D4
:10F7E000032A48D068E0002198E79DF809001AF83C
:10F7F000000038B15A462046039B0599FFF732FBBB
:10F80000A1E725E0059B224619462046FFF72AFB83
:10F8100099E722465846059B0399FFF723FB92E799
:10F8200098F8000098F80110884202D20BF80450B2
:10F8300098E70BF804A095E798F8000098F80110F5
:10F84000884202D90BF804508CE70BF804A089E732
:10F8500000248B485238B0F820B02BFA04F000F0A6
:10F86000010021F07FFE06EB84114862641CE4B2C3
:10F87000052CF2D3A9E7012908D001211BF80120AA
:10F88000012A05D006EB8012556215E00021F5E74C
:10F8900006EB80134FF07E525A620DE03A1892F850
:10F8A0007620112A08D1C9B100211BF80120012AB4
:10F8B00016D006EB80125562401CC0B207288AD3CE
:10F8C000002404F1B700079002F0EDF803280DD0F2
:10F8D000079802F0E8F8042816D022E00121E4E7B6
:10F8E00006EB80134FF07E525A62E5E798F800006D
:10F8F00098F80110884203D2381980F8B75010E008
:10F90000381980F8B7A00CE098F8000098F80110BA
:10F91000884203D9381980F8B75002E0381980F8C6
:10F92000B7A0641CE4B2022CCBD35548DFF850A139
:10F930005238AAF1060A407980B1062829D0AAF1E6
:10F940001A021178062953D899F80000E0B34E48FE
:10F95000085C8DF8100004F00F0058E0BAF80000C1
:10F96000323000B2AAF800004FF47A71884201DD0B
:10F97000AAF80050BAF80200323800B2AAF8020021
:10F98000002801DAAAF802104FF4FA7009F0CAFF51
:10F990001AE197F8A602042817D0AAF8005097F8A1
:10F9A000A702042817D0AAF80250BAF900104FF4A1
:10F9B0007A70814201DDAAF80000BAF90210814292
:10F9C00001DDAAF80200FFE00BE00620FFF7C8FC0B
:10F9D000AAF80000E3E70720FFF7C2FCAAF802003C
:10F9E000E3E729480E30085C8DF8100020090EE08E
:10F9F00099F80000E0B197F8A100C0F10600081ADC
:10FA0000384490F82D018DF8100004F00F0097F89D
:10FA10009F305178C3F10603CB1A06291AD899F8FA
:10FA200000308BB1184BDB1DC95C8DF8111019E04B
:10FA3000200997F8A130C3F10603C91A394491F897
:10FA40003B118DF81010E2E70C4B3A3BC95C8DF886
:10FA5000111007E099F80010C1B1D91991F83411CB
:10FA60008DF81110917806291BD899F800209AB1C9
:10FA7000024A1A3A895C8DF812101FE0B482002005
:10FA8000CC0000207C840020C1800020D91991F88E
:10FA9000E6128DF81110E5E7B94A895C8DF812106D
:10FAA0000CE099F80020F2B197F89D20C2F106020F
:10FAB000891A394491F806138DF8121004A9FFF73A
:10FAC00060FAB04805210690FBF76CF9B0B197F8E1
:10FAD000620397F86313000200B2084421F02AFD84
:10FAE000C6F85C010DE097F89D20C2F10602891A64
:10FAF000394491F819138DF81210DFE7A248C6F8BF
:10FB00005C0106210698FBF74DF958B197F864039C
:10FB100097F86513000200B2084421F00BFDC6F807
:10FB20009C0102E09848C6F89C01984CA0790128F5
:10FB30004AD197F8B70004A94FF06409095CC1F3F2
:10FB4000011149B101292CD004F13503DA1C022935
:10FB500004D0032927D114E0E58324E018F800102D
:10FB6000125C914203D9881A4000E0831BE0185CC4
:10FB7000814204D2C1F132004000E08313E0E5830A
:10FB800011E018F80010125C914201D9E1830AE0FB
:10FB9000185C814203D2C1F16400E08303E0E58395
:10FBA00001E0A4F81E9007210698FBF7FBF808B1C6
:10FBB000607BE083B4F91E00052801DAE58303E0E9
:10FBC0005F2801DDA4F81E900024DFF8C4813819F5
:10FBD00090F8BE00012802D16E49097861B102286F
:10FBE00002D1B8F8001039B1032802D1B8F80210D8
:10FBF00011B1042804D006E006EB841045622DE024
:10FC000097F8DB1011B105280AD00CE09BF8000032
:10FC1000012823D106EB84114FF07E5048621DE08D
:10FC200097F8DB1011B106280DD017E021465A488D
:10FC3000FBF7B8F89BF80010084021F093FC06EBA6
:10FC4000841148620AE097F8DB00022806D14F4889
:10FC5000807A012802D106EB84104562641CE4B26C
:10FC6000052CB4D30020DFF824914FF07E5899F88A
:10FC700009103A1892F8DC20022A04D101291CD07C
:10FC800006EB80125562401CC0B20528F1D3002457
:10FC90003D4D002006EB841151F82020AA4217D0D8
:10FCA00051F8200010F0FF4F0CD0404514D1012234
:10FCB00021463948FBF75CF80EE006EB8012C2F8EB
:10FCC0002480E0E7002221463348FBF751F803E0A7
:10FCD000401CC0B21028DFD3641CE4B2052CD8D37A
:10FCE00099F80500002817D00524002006EB8411A0
:10FCF00051F82020AA4207D051F8200021F0DEFB65
:10FD0000611F2AF8110003E0401CC0B21028EFD395
:10FD1000641CE4B2072CE8D30BB0BDE8F08F1B489D
:10FD200032300078011F022902D80A30C0B2704771
:10FD3000C11F022902D8C01EC0B27047A0F10A013B
:10FD40000229FAD8C01DC0B2704770B50F4E00210D
:10FD5000308AFBF709F804460A4DD63D95F8A10014
:10FD600000B900240021708AFAF7FEFF28B1A41C14
:10FD7000E4B295F8A00000B90024204670BD000050
:10FD8000AD8200206A80002000007F437A000020BE
:10FD90003C120020420000209E0200200D49086015
:10FDA00070470C49486070470A49886070470949A4
:10FDB0004AF6AA200860704706494CF6CC40086015
:10FDC000704701460020034AD2680A4200D0012051
:10FDD0007047000000300040B448016841F0010164
:10FDE00001604168B24A114041600168B14A114066
:10FDF0000160016821F480210160416821F4FE0165
:10FE000041604FF41F0181607047A8490A6822F4DD
:10FE100080320A600A6822F480220A60B0F5803FCE
:10FE200007D0B0F5802F03D1086840F4A020086007
:10FE30007047086840F4803008607047034600202F
:10FE400059099A4A01290AD002290AD0516A03F0B5
:10FE50001F02012393400B4200D00120704711681C
:10FE6000F5E7116AF3E718B5002000904FF4A0649D
:10FE70003120FFF7E3FF0099491C00910099A1424E
:10FE800001D00028F4D03120FFF7D8FF08B10120BD
:10FE900018BD002018BD854A116821F0F80141EA1B
:10FEA000C000106070478449086070477F4B5A68F3
:10FEB00022F47C1208431043586070477E4908665C
:10FEC00070477A4A516821F003010143516070473D
:10FED0007648406800F00C007047744A516821F081
:10FEE000F001014351607047704A516821F4E061AC
:10FEF0000143516070476D4A516821F4605141EAF5
:10FF0000C00050607047694A002903D0517A01430C
:10FF100051727047517A8143517270476649D831A6
:10FF200008607047614A516821F4404101435160C3
:10FF300070475E49002220310A7001F8202901280B
:10FF400005D0042802D1052081F820007047012047
:10FF500081F82000704759490860704753490A6A80
:10FF600002430A627047554944390860704710B52A
:10FF70004E4A516801F00C01514B002927D0042949
:10FF800027D0082927D00360516801F0F001090942
:10FF90004C4B5C5C0168E1404160546804F4E064EF
:10FFA000240A1C5D21FA04F48460546804F460544B
:10FFB000E40A1B5DD940C160526802F44042920BD2
:10FFC000404B1B1F9A5CB1FBF2F1016110BD036055
:10FFD000DAE70360D8E7516801F47011536803F45D
:10FFE0008033022404EB914133B153689B0307D55E
:10FFF000354B59430160C7E7334B59430160C3E7B1
:020000040801F1
:100000002F4B59430160BFE7284A002903D05169AB
:100010000143516170475169814351617047234ADF
:10002000002903D09169014391617047916981432F
:10003000916170471D4A002903D0D1690143D16104
:100040007047D1698143D1617047184A002903D0B4
:10005000D1680143D1607047D1688143D160704756
:10006000124A002903D011690143116170471169D7
:1000700081431161704711494039086070470E494A
:10008000C86470470949C87170470848416A41F01F
:1000900080714162704701460020044A92680A421A
:1000A00000D001207047014988727047001002405B
:1000B0000000FFF8FFFFF6FE0000424280044242CB
:1000C00000127A00E600002000093D004D4A002998
:1000D00003D011880143118070471188814311803A
:1000E00070474848001D018841F0100101807047A9
:1000F0004448001D018821F01001018070474148EB
:100100001C3000883F491831098840EA0140704797
:1001100000B50246FFF7E5FF3A49100C1831088098
:10012000081D02805DF804EBE2E700B50246FFF728
:10013000D8FF3449C2F3034008310880081D02800B
:100140005DF804EBD4E700B50246FFF7CAFF2D497E
:10015000100C20310880081D02805DF804EBC7E711
:100160002848103000880007010B2648143000880A
:100170000843704770B50024224D2D1D06E0641C15
:10018000E4B2642009F0CEFB1E2C02D82888800639
:10019000F5D570BD70B500241A4D2D1D288820F0AE
:1001A0000800288006E0641CE4B2642009F0BAFB71
:1001B0001E2C02D828880007F5D570BD0146002006
:1001C000104A121D12880A4200D0012070470D49C2
:1001D000091D0A8882430A8070470A49091D098857
:1001E000C2B21140074A1288024202D009B101206E
:1001F0007047002070470349091D0A8882430A801E
:10020000704700000028004010B5FE4988420AD11E
:10021000C41401212046FFF718FF2046BDE8104016
:100220000021FFF712BFB0F1804F0CD0F649884291
:1002300013D101210220FFF713FF0021BDE8104078
:100240000220FFF70DBF01210846FFF709FF00213B
:10025000BDE810400120FFF703BFEC49884209D1F7
:1002600001210420FFF7FCFE0021BDE8104004201E
:10027000FFF7F6BEE649884209D101210820FFF7C1
:10028000EFFE0021BDE810400820FFF7E9BEE1497C
:10029000884209D101211020FFF7E2FE0021BDE8CC
:1002A00010401020FFF7DCBEDB49884209D1012154
:1002B0002020FFF7D5FE0021BDE810402020FFF7E9
:1002C000CFBED64988420AD1441401212046FFF707
:1002D000BCFE2046BDE810400021FFF7B6BED04965
:1002E00088420AD10121CC042046FFF7AEFE204609
:1002F000BDE810400021FFF7A8BECA4988420AD1D4
:1003000001210C052046FFF7A0FE2046BDE8104065
:100310000021FFF79ABEC44988420AD101214C0549
:100320002046FFF792FE2046BDE810400021FFF76F
:100330008CBEBE49884209D101214020FFF790FEC2
:100340000021BDE810404020FFF78ABEB84988422E
:1003500009D101218020FFF783FE0021BDE8104074
:100360008020FFF77DBEB34988420AD18415012160
:100370002046FFF775FE2046BDE810400021FFF73C
:100380006FBEAD4988420AD101210C042046FFF717
:100390005CFE2046BDE810400021FFF756BEA7498D
:1003A00088420AD101214C042046FFF74EFE204628
:1003B000BDE810400021FFF748BEA14988420AD19C
:1003C00001218C042046FFF740FE2046BDE8104086
:1003D0000021FFF73ABE10BD30B50288894C8F4D21
:1003E000A0420DD0A8420BD0B0F1804F08D0864B70
:1003F000984205D0854B984202D0854B984203D154
:1004000022F070034A881A43824B984206D0824BEE
:10041000984203D022F44073CA881A4302808A8823
:1004200082850A880285A0420AD0A84208D0824A62
:10043000904205D0814A904202D0814A904201D137
:10044000097A01860121818230BD30B5028C22F00B
:1004500001020284028C8388048B24F0700424F04F
:1004600003050C882C4322F002020D8915434A88AB
:100470002A43644DA8420BD0684DA84208D06E4D67
:10048000A84205D06D4DA84202D06D4DA8420FD1B3
:1004900022F008054A892A4322F004058A882A4363
:1004A00023F4807323F400738D891D43CB892B4380
:1004B00083800483C9888186028430BD70B5028C34
:1004C00022F010020284028C8388048B24F4E0441E
:1004D00024F440760D884FF6FF7404EA0525354371
:1004E00022F020020E8904EA061616434A8804EA1E
:1004F00002123243434EB04202D0484EB04217D1AE
:1005000022F080024E8904EA0616164326F04006C1
:100510008A8804EA0212324323F4806323F40063DE
:100520008E8904EA86061E43CB8904EA830333439B
:1005300083800583C9880187028470BD70B5028CF1
:1005400022F480720284028C8388848B24F07004ED
:1005500024F003040D88254322F400720E894FF61F
:10056000FF7404EA062616434A8804EA022232434C
:10057000244EB04202D0294EB04217D122F4006678
:100580004A8904EA0222324322F480668A8804EA15
:100590000222324323F4805323F400538E8904EA69
:1005A00006161E43CB8904EA0313334383808583F5
:1005B000C9888187028470BD70B5028C22F4805294
:1005C0000284058C8288838B23F4E04323F44076F5
:1005D0000C884FF6FF7303EA0424344325F40055D6
:1005E0000E8903EA06362E434D8803EA0535354366
:1005F000044EB04202D0094EB04226D122F48046C9
:100600008A891FE0002C01400004004000080040DF
:10061000000C004000100040001400400034014075
:10062000004C0140005001400054014000180040BF
:10063000001C0040002000400040014000440140F8
:100640000048014003EA8212324382808483C988D1
:10065000A0F84010058470BD828B22F44062828332
:10066000828B4FF6FF7303EA01210A4382837047AE
:10067000F0B5048C24F480540484868B048C4FF6EB
:10068000FF7505EA013726F4734605EA0222324374
:1006900005EA03331343F74A90420ED0F64A9042DC
:1006A0000BD0B0F1804F08D0F44A904205D0F44A04
:1006B000904202D0F34A904205D124F400513943CC
:1006C00041F4805104E024F402420A4342F4805190
:1006D00083830184F0BD828B22F00C028283828BA3
:1006E0000A4382837047F0B5048C24F48074048438
:1006F000858B048C4FF6FF7707EA012625F0F3057A
:1007000007EA031313432B43DA4A90420ED0DA4A26
:1007100090420BD0B0F1804F08D0D84A904205D01B
:10072000D74A904202D0D74A904205D124F40071B2
:10073000314341F4807104E024F420620A4342F41E
:10074000807183830184F0BD028B22F440620283B6
:10075000028B4FF6FF7303EA01210A4302837047BD
:10076000F0B5048C24F010040484068B048C4FF63E
:10077000FF7505EA011726F4734605EA0333334390
:1007800005EA02221A43BB4B98420ED0BA4B98425C
:100790000BD0B0F1804F08D0B84B984205D0B84B81
:1007A000984202D0B74B984205D124F0200139433A
:1007B00041F0100104E024F0A0030B4343F01001CA
:1007C00002830184F0BD028B22F00C020283028BB3
:1007D0000A430283704770B5048C24F0010404843A
:1007E000058B048C25F0F3054FF6FF7606EA03131C
:1007F00013432B439F4A90420ED09F4A90420BD006
:10080000B0F1804F08D09D4A904205D09C4A90425A
:1008100002D09C4A904205D124F002020A4342F0E1
:10082000010104E024F00A020A4342F001010383BB
:10083000018470BD70B505460C468E48854209D0CE
:100840008D48854206D0B5F1804F03D08B48854254
:1008500000D08B4820886188A288238958B1042859
:1008600011D0082817D02846FFF702FFE188284654
:10087000BDE87040F0E62846FFF7ADFFE188284666
:10088000BDE870409FE72846FFF76AFFE1882846E9
:10089000BDE8704058E72846FFF725FFE188284665
:1008A000BDE8704017E72DE9F04107460C460025EA
:1008B00001266188002900D10225A288012A00D1E1
:1008C00002262088238988B13846FFF749FFE1884E
:1008D0003846FFF739FF2389324629463846FFF765
:1008E0007AFFE1883846BDE8F0416CE73846FFF70B
:1008F00072FFE1883846FFF766FF238932462946B2
:100900003846FFF72DFFE1883846BDE8F0411BE788
:1009100010B50A884B88CC881A438B8823431A4326
:100920000B891A434B8989891A430A43A0F844204A
:1009300010BD4FF6FF71818000210180C180418090
:10094000017270470021018041808180C180018156
:1009500041818181C1817047002101804180012254
:100960008280C180018170470021018041808180A7
:10097000C1800181418181817047002904D00188B3
:1009800041F0010101807047018821F001010180DF
:100990007047002905D030F8441F41F40041018020
:1009A000704730F8441FC1F30E0101807047002AE0
:1009B00003D082890A438281704782898A43828177
:1009C0007047818270471143A0F848107047002A91
:1009D00003D082890A438281704782898A43828157
:1009E0007047018921F0070101817047028922F0D7
:1009F00070020A430281704700B503461846FFF7AC
:100A0000F5FF188940F00700188100BD70B50D464C
:100A100004461146602D0CD001222046FFF7DBFE74
:100A200029462046FFF7E2FF208940F00700208199
:100A300070BD01222046FFF793FEF1E730B504892F
:100A4000E4B24FF6FF7505EA032313430B43234338
:100A5000038130BD10B504462046FFF7EFFF208923
:100A600020F0070040F0070020F0700040F0700018
:100A7000208110BD002C01400034014000040040E2
:100A800000080040000C004010B504462046FFF767
:100A9000D5FF208940F480402081EAE701858282E9
:100AA0007047028822F070020A430280704770B5D6
:100AB0000589048B068C25F007050D434FF6FC4194
:100AC0000C4040F201110C4326F022064FF6FF7154
:100AD00001EA03111143314305810483018470BD90
:100AE000028B22F070020A4302837047028B22F4C9
:100AF000E0424FF6FF7303EA01211143018370477F
:100B0000828B22F070020A4382837047828B22F428
:100B1000E0424FF6FF7303EA0121114381837047DE
:100B2000002904D0018841F08001018070470188CC
:100B300021F0800101807047002904D0818841F0B4
:100B4000040181807047818821F004018180704711
:100B5000002904D0818841F0080181807047818894
:100B600021F0080181807047002904D0818841F07C
:100B7000010181807047818821F0010181807047E7
:100B8000028B22F008020A4302837047028B22F490
:100B900000624FF6FF7303EA01211143018370479E
:100BA000828B22F008020A4382837047828B22F4F0
:100BB00000624FF6FF7303EA0121114381837047FE
:100BC000028B22F004020A4302837047028B22F454
:100BD00080624FF6FF7303EA0121114301837047DE
:100BE000828B22F004020A4382837047828B22F4B4
:100BF00080624FF6FF7303EA01211143818370473E
:100C0000028B22F080020A4302837047028BC2F3F8
:100C10000E024FF6FF7303EA01211143018370476F
:100C2000828B22F080020A4382837047828BC2F358
:100C30000E024FF6FF7303EA0121114381837047CF
:100C4000028C22F002020A4302847047028C22F0D6
:100C500008020A4302847047028C22F020024FF6F9
:100C6000FF7303EA0111114301847047028C22F0E3
:100C700080024FF6FF7303EA0111114301847047AC
:100C8000028C22F400724FF6FF7303EA0121114334
:100C900001847047028C22F400624FF6FF7303EA6E
:100CA0000121114301847047028C22F400524FF657
:100CB000FF7303EA013111430184704710B501232A
:100CC0008B40048C9C430484038C8A40134303842C
:100CD000CFE610B504238B40048C9C430484038C22
:100CE0008A4013430384C4E630B500F1180301249D
:100CF0008C40058CA5430584002911D008290FD00C
:100D0000091FC1F34E001844016821F4E04101605D
:100D100001684FF6FF7303EA02221143016030BD00
:100D200003EB5100016821F070010160016811437B
:100D3000016030BD002904D0018841F0020101802A
:100D40007047018821F0020101807047002904D01A
:100D5000018841F0040101807047018821F00401FD
:100D600001807047002904D0818841F08001818092
:100D70007047818821F0800181807047028822F0CD
:100D80000802028002880A4302807047828822F0AB
:100D90007002828082880A4382807047028922F032
:100DA0000702028102890A4302817047028922F008
:100DB0008002028102890A43028170478184704760
:100DC00081857047818670470187704781877047AA
:100DD000A0F840107047028822F440720280028816
:100DE0000A4302807047808E7047008F7047808F63
:100DF0007047B0F840007047808C7047008D704796
:100E000002460020128A0A4200D001207047C943DE
:100E10000182704702460020138A0B4092890A40E3
:100E2000002B02D0002A00D001207047C943018264
:100E30007047000010B5E14988420AD101218C03B6
:100E40002046FFF702F92046BDE810400021FFF7D9
:100E5000FCB8DB4988420AD101214C042046FFF747
:100E6000FFF82046BDE810400021FFF7F9B8D5494A
:100E700088420AD101218C042046FFF7F1F8204670
:100E8000BDE810400021FFF7EBB8CF4988420AD1F6
:100E90000121CC042046FFF7E3F82046BDE81040CE
:100EA0000021FFF7DDB8C94988420AD101210C05AC
:100EB0002046FFF7D5F82046BDE810400021FFF797
:100EC000CFB810BD30B585B004460D46208A4CF62B
:100ED000FF710840E98801432182A0894EF6F31191
:100EE0000840A9882A8911436A8902431143A181D4
:100EF000A08A4FF6FF410840A9890143A1826846B4
:100F0000FFF735F8AD48844201D1039800E002981C
:100F1000A189090408D500EBC00101EB0010296884
:100F20004900B0FBF1F007E000EBC00101EB00105D
:100F300029688900B0FBF1F06422B0FBF2F10901ED
:100F40000B096FF018056B4300EB8300A3891D04A8
:100F50004FF0320307D503EBC000B0FBF2F000F016
:100F60000700084306E003EB0010B0FBF2F000F0CE
:100F70000F000843208105B030BD4FF416510160C9
:100F800000218180C18001810C22428181817047D2
:100F900010B5038A4FF2FF0213400A884C8822439F
:100FA0008C88C9880C4322431A43028210BD002159
:100FB000018041808180C1807047002904D08189EF
:100FC00041F4005181817047818921F40051818170
:100FD000704710B540F66A13C1F3421301F01F04C5
:100FE0000121A140012B07D0022B07D014303AB1C8
:100FF00002680A43026010BD0C30F8E71030F6E7D3
:1010000002688A43026010BD002A03D0828A0A4324
:1010100082827047828A8A4382827047028A22F0E3
:101020000F020282028A0A4302827047828922F4F6
:101030000062828182890A4382817047002904D03C
:10104000818941F0020181817047818921F002018B
:1010500081817047028A22F020020282028A0A43BA
:1010600002827047002904D0018A41F48041018244
:101070007047018A21F4804101827047C1F3080161
:10108000818070478088C0F308007047818941F0F3
:10109000010181817047028BD2B20283028B42EA46
:1010A000012101837047028B02F47F420283028B8D
:1010B0000A4302837047002904D0818A41F020014D
:1010C00081827047818A21F0200181827047002946
:1010D00004D0818A41F0100181827047818A21F019
:1010E000100181827047002904D0818A41F00801F3
:1010F00081827047818A21F008018182704700292E
:1011000004D0818941F40041818170478189C1F314
:101110000E0181817047002904D0818A41F4006169
:1011200081827047818A21F4006181827047828ABE
:1011300022F004028282828A0A4382827047002956
:1011400004D0818A41F0020181827047818A21F0B6
:101150000201818270470246002012880A4200D0B4
:10116000012070478A05C9430180704770B500248B
:1011700040F66A12C1F3421301F01F05012606FA78
:1011800005F2012B0CD0022B0DD0838A1340090AE3
:101190008E40008830400BB100B10124204670BD64
:1011A00083891340F3E7038A1340F0E740F66A129D
:1011B0000A0A01219140C94301807047003801406B
:1011C0000044004000480040004C004000500040F7
:1011D00010B50120FEF74FFFBDE810400020FEF7DC
:1011E0004ABF2049086070471E49091F08607047C0
:1011F0001C498431086070471B4A118821F46071D2
:10120000014311807047184A118821F07F01014382
:101210001180704708B5144A2C3A10440090009889
:10122000016008BD08B510492C39084400900098A9
:10123000008808BD0B489C300068C0B270470A485F
:101240000830018841F00101018070470548A03055
:101250000068C0B2704704480830018841F00201BC
:101260000180704704860D422C6C004010B50121AE
:101270000C072046FEF7F4FE2046BDE81040002192
:10128000FEF7EEBE214908627047204908617047A9
:101290001F4A116821F0E0010143116070471B49AA
:1012A000A031086070471A4B1A6822F0030202430B
:1012B0001A601848026842F004020260012905D051
:1012C00020BF016821F004010160704730BFF8E7DA
:1012D0000F48016841F004010160016841F002011A
:1012E00001600C48016841F00401016030BF7047A3
:1012F00001460020064A52680A4200D00120704789
:1013000003490A6842EA80000860704700000E4204
:101310000070004010ED00E0094880470948004790
:10132000FEE7FEE7FEE7FEE7FEE7FEE7FEE7FEE795
:10133000FEE7FEE704480549054A064B70470000F2
:10134000D58300083181000850D8002050DE0020ED
:1013500050DA002050DA00207FB5B24CA088ADF8FA
:101360000C0048258DF80F5002268DF80E6003A959
:101370002068F7F74EFD208AADF808008DF80B5075
:101380008DF80A6002A9E068F7F743FDA08BADF87D
:1013900004008DF807508DF8066001A9A069F7F7E1
:1013A00038FD208DADF800008DF803508DF80260F7
:1013B0006946606AF7F72DFD7FBD70B5994D583DC0
:1013C000B5F85C10A86DF7F77FFD974C18B320783F
:1013D00020F004002070B5F86810686EF7F774FD0F
:1013E000F0B1207820F002002070B5F87410286F5A
:1013F000F7F76AFDC8B1207820F001002070B5F839
:101400008010E86FF7F760FDA0B1207820F00800A9
:101410002070207870BD207840F004002070DAE75A
:10142000207840F002002070DFE7207840F00100D3
:101430002070E4E7207840F008002070E9E72DE90B
:10144000F047012008F04EFAFFF7B7FF044677484F
:101450004480754EDFF8D881093E4FF0000770795F
:101460004FF0010534EA000015D098F87F000328FA
:1014700011D0F5706F48077098F8ED006E49C0EB19
:1014800000104FF6FF7202EA8000088018B10121B7
:101490006A48F7F72DFDF078694B012876D171790C
:1014A00031EA040072D098F87A0002286ED0F77002
:1014B00064480570644A64201070B1716348077015
:1014C000187801280FD072784FF00D0C05204FF0DE
:1014D0000E0962B3012951D002293DD0042960D000
:1014E000082976D169E03079172801D0182803D16E
:1014F00008290AD0042908D001290DD0022908D0D2
:1015000004290CD008290FD10CE01920B0723771D2
:101510005FE01820B07207E01720B07204E01620D8
:10152000B07201E01520B072B07A307151E001293B
:101530004FD002294DD0042902D0082949D105E015
:1015400086F80AC07570B570307042E086F80A906F
:101550007570B57030703CE0B278012A04D0022A70
:1015600005D0032A06D007E00A22B27204E0112255
:10157000B27201E01222B27230702AE0B278012A0F
:1015800005D0022A06D0032A07D008E032E009225B
:10159000B27204E00F22B27201E01022B272307017
:1015A00017E086F80AC07570B278032A02D2521C7E
:1015B000B27000E0B57030700BE086F80A9075707C
:1015C000B278012A02D9521EB27001E00322B27031
:1015D0003070042908D0082906D0022904D0012936
:1015E00002D098F8790028B919480770F571B581CB
:1015F0001848077074710C2C11D1187878B998F8C4
:101600007F0001280BD0032809D0307A411C3172A9
:101610001E2802D91320B0721D70BDE8F087377202
:10162000FBE7000070240308FF0000205A1200208E
:10163000947F00206E00002046000020000801403A
:10164000710000206F00002077000020780000204B
:10165000720000207900002038B5A54C208FADF82D
:10166000000048208DF803006946606BF7F7D1FB56
:10167000218F606BF7F73CFC38BD38B59C4C208F50
:10168000ADF8000010208DF8030003208DF8020053
:101690006946606BF7F7BDFB218F606BF7F728FC9D
:1016A00038BD08B50820ADF8000010208DF8030003
:1016B00003208DF8020069468E48F7F7AAFB08BDA3
:1016C00008B50820ADF8000048208DF803006946F1
:1016D0008848F7F79EFB08BD854A002803D0918D06
:1016E000906AF7F705BC918D906AF7F703BC804AC2
:1016F000002803D0118F506BF7F7FABB118F506B96
:10170000F7F7F8BB7A48018F406BF7F7DDBB7848F5
:10171000818D806AF7F7D8BBF8B5754C0121606AF6
:10172000FEF77DFCA08DADF8000010258DF803506C
:1017300003268DF802606946A06AF7F76AFBA18D5F
:10174000A06AF7F7D5FB0121206BFEF768FC208F1C
:10175000ADF800008DF803508DF802606946606BAB
:10176000F7F757FB218F606BF7F7C2FBF8BD10B599
:10177000FFF783FF0120FFF7BAFF0120FFF7ACFF5F
:10178000042008F0AFF80020FFF7B1FF042008F0B4
:10179000A9F8BDE8104000209EE710B5FFF76DFFE7
:1017A0000020FFF799FF0020FFF7A1FF042008F0B9
:1017B00099F80120FFF790FF0120FFF798FFBDE89F
:1017C0001040042008F08EB810B500240120FFF767
:1017D0008EFFFFF741FF012008F084F80120FFF79A
:1017E0007BFF012008F07EF807E0641CA4B2FA2C0D
:1017F00003D9FFF7D2FF012010BDFFF783FF0028B8
:10180000F3D1FFF769FF002010BD10B50020FFF7EE
:1018100063FFFFF732FF0020FFF769FF022008F0A7
:1018200061F80120FFF758FF022008F05BF8BDE8DF
:101830001040002050E710B50020FFF74DFFFFF7E4
:101840001CFF0120FFF753FF022008F04BF8012096
:10185000FFF742FF022008F045F8BDE810400020E5
:101860003AE770B50546FFF708FF0020FFF734FFA1
:101870000024E809FFF73BFF6806050E022008F088
:1018800031F80120FFF728FF022008F02BF8002094
:10189000FFF722FF022008F025F8641CE4B2082CB0
:1018A000E7D370BD70B506460024FFF7D5FE0025CE
:1018B0000020FFF711FF022008F014F80120FFF7C5
:1018C0000BFF6006040EFFF71DFF08B1641CE4B2B5
:1018D000012008F007F86D1CEDB2082DE8D31EB109
:1018E000FFF793FF204670BDFFF7A5FFFAE7000062
:1018F000182403080008014038B5704CE06B00283C
:1019000015D054F83C0F0121FEF789FB2089ADF872
:10191000000010208DF8030003208DF802006946B6
:101920006068F7F776FA21896068F7F7E1FA38BD61
:10193000624AD16B00290AD020B1B2F84410106C71
:10194000F7F7D6BAB2F84410106CF7F7D3BA70476D
:1019500010B5FFF7E1FEBDE81040CDE710B5044635
:10196000FFF705FF200AA02101EB4000C0B2FFF7FE
:1019700078FFFFF729FFE0B2FFF773FFFFF724FFBF
:10198000FFF7F5FEA120FFF76CFFFFF71DFF00201A
:10199000FFF788FF0446FFF700FF204610BD70B533
:1019A00004460D460020FFF7C3FFFFF7E0FE200AC4
:1019B000A02101EB4000C0B2FFF753FFFFF704FF87
:1019C000E0B2FFF74EFFFFF7FFFE2846FFF749FFA3
:1019D000FFF7FAFEFFF7E1FE0120FFF7A9FFBDE8E0
:1019E0007040052007F09EBF2DE9F04106460D46E8
:1019F0001746002409E0E00025FA00F0C1B23019D2
:101A000080B2FFF7CCFF641CE4B2BC42F3D3BDE864
:101A1000F0812DE9F04102460E460020002497197E
:101A200008E00502381B401E80B2FFF797FF2844EC
:101A3000641CE4B2B442F4D3E9E710B5FF20FFF729
:101A40008DFF55280AD05521FF20FFF7A8FFFF2062
:101A5000FFF784FF552803D0012010BD002010BDE2
:101A6000002010BD70B504460E46154608E020461D
:101A7000641CA4B2FFF772FF06F8010B6D1EADB235
:101A8000002DF4D170BD70B506460D46144606E033
:101A900029783046FFF783FF761CB6B26D1C641EB2
:101AA000A4B2F5D270BD59E7054A1278012A03D0D5
:101AB000B72802D0B82800D071E77047182403086F
:101AC00005010020704730B56423B0FBF3F4E4B2A5
:101AD000B0FBF3F503FB1500132C01D96430C0B241
:101AE00000EB90030724B3FBF4F504FB1533A44D7E
:101AF0001A440D4415F8015C2A4492B2800703D1C0
:101B0000032901D2521E92B2B2FBF4F004FB102062
:101B100030BD810701D0002070476421B0FBF1F295
:101B200001FB120109B1012070474FF4C871B0FBED
:101B3000F1F201FB120008B100207047012070474C
:101B40002DE9F047FEF7DBFA06468E4FB6FBF7F3BA
:101B50008D488E4D0188994233D0038040F2B27493
:101B60004FF4B7784FF4B6790FE02046FFF7D1FF76
:101B700038B1434502D3A3F5B77304E0641CA4B2A3
:101B800005E0A3F26D13641CA4B24B45EDD8AC8004
:101B90000024DFF8EC8108F10C080CE0A888FFF7BE
:101BA000B8FF08B1012C2FD018F80400984204D8CF
:101BB0001B1A641CA4B21C2BF0D2641CAC715B1CFD
:101BC000EB71B6FBF7F007FB10604FF46161B0FBFF
:101BD000F1F22A70B0FBF1F201FB12033C22B3FBDD
:101BE000F2F36B70B0FBF1F301FB1300B0FBF2F109
:101BF00002FB1100A870EA79A979A888FFF763FFB2
:101C000028720020BDE8F0871D2BD6D31D3BD0E7FE
:101C100070B5002401214FF0C050FEF70BFA0420EC
:101C2000FFF700FB45F25005A8423AD00120FFF72C
:101C300029FBFFF7CDFA0120FEF77BF908E0641CD1
:101C4000E4B20A2007F06EFEC82C01D3012070BD5B
:101C50004120FEF7F3F80028F1D0FA2C01D301203F
:101C600070BD4FF48070FEF779F90120FEF77BF923
:101C7000FEF780FAFEF78EFA01210846FEF726FAF3
:101C8000FEF778FAFEF72DFA47F6FF70FEF74DFAE9
:101C9000FEF770FAFEF72CFA29460420FFF7BAFA8D
:101CA00007E0FEF777FA01210846FEF70FFAFEF784
:101CB00061FAFFF707FFFFF743FF002070BD2DE932
:101CC000F05F0646DDF828A0894690460024A6F27B
:101CD000B270822802D30120BDE8F09F40F2B275B5
:101CE0002B4FDFF8B0B008E02846FFF712FF08B12D
:101CF0003C4400E05C446D1CADB2B542F4D3A9F1A4
:101D0000010909F0FF070025DFF87490DFF874B0CF
:101D100009F10C090FE019F8050040F2A32148432E
:101D200004EBC0143046FFF7F4FE10B1012D00D1D2
:101D30005C446D1CADB2BD42EDD3A8F1010840F288
:101D4000A32008FB00F804EBC810C3EB4311C1EB60
:101D5000032100EB0110CAEB0A1100EB81000B9983
:101D6000441801214FF0C050FEF764F90120FFF73D
:101D700089FA2046FEF7CCF9FEF7FCF90020ABE724
:101D8000FE2303088051010006010020B01100204D
:101D90000085E2018033E10170B5FA4B0024C3F8FD
:101DA0008041F94A0125127A042A02D3F74A1560C4
:101DB00001E0C3F888510022C3F88441060602D529
:101DC000C3F88C5101E0C3F88C41C3F8845140063C
:101DD000000E521CD2B2082AEED30020C3F8844170
:101DE0000A0602D5C3F88C5101E0C3F88C41C3F850
:101DF00084514906090E401CC0B20828EED3C3F82E
:101E0000805170BDC0F30722C1B21046C4E730B59F
:101E1000DC4A0023C2F88031DB49097A042902D365
:101E2000DA490B6001E0C2F8883100210124C2F8D0
:101E30008431050602D5C2F88C4101E0C2F88C312C
:101E4000C2F884414006000E491CC9B20829EED3ED
:101E5000C2F8804130BD30B5CA4A0024C2F8804182
:101E6000C9490123097A042902D3C8490B6001E05A
:101E7000C2F888310021C2F88441050602D5C2F8B3
:101E80008C3101E0C2F88C41C2F884314006000E6A
:101E9000491CC9B20829EED3C2F8803130BD2DE902
:101EA000F04381468846C2F30724D5B2C3F3072620
:101EB000DFB22A20FFF7ABFF0020FFF7CCFF484638
:101EC000FFF7C9FF0020FFF7C6FF4046FFF7C3FF3B
:101ED0002B20FFF79CFF2046FFF7BDFF2846FFF7AA
:101EE000BAFF3046FFF7B7FF3846FFF7B4FFBDE84B
:101EF000F0432C208BE72DE9F0410746002240F209
:101F00003F13EF211046FFF7CAFF00254FF4A076DC
:101F100000243846FFF776FF641CF02CF9D36D1CC3
:101F2000B542F5D3BDE8F08100B52820FFF76FFF7B
:101F300010205DF804EB6AE710B51120FFF767FF8A
:101F4000782007F0EFFCBDE8104029205FE770B56E
:101F50008F4C01252560052007F0E4FC0020E0639C
:101F60000A2007F0DFFCE563782007F0DBFC112096
:101F7000FFF74DFF782007F0D5FCCF20FFF747FF94
:101F80000020FFF768FFC320FFF765FF3020FFF751
:101F900062FFED20FFF73BFF6420FFF75CFF0320AB
:101FA000FFF759FF1220FFF756FF8120FFF753FF7D
:101FB000E820FFF72CFF8520FFF74DFF1020FFF7EB
:101FC0004AFF7920FFF747FFCB20FFF720FF39209A
:101FD000FFF741FF2C20FFF73EFF0020FFF73BFFFC
:101FE0003420FFF738FF0220FFF735FFF720FFF717
:101FF0000EFF2020FFF72FFFEA20FFF708FF002049
:10200000FFF729FF0020FFF726FFC020FFF7FFFEA4
:102010002220FFF720FFC120FFF7F9FE1120FFF774
:102020001AFFC520FFF7F3FE3D20FFF714FF202025
:10203000FFF711FFC720FFF7EAFEAA20FFF70BFF0B
:102040003620FFF7E4FEC820FFF705FF3A20FFF730
:10205000DEFE5520FFF7FFFEB120FFF7D8FE00207F
:10206000FFF7F9FE1320FFF7F6FEB620FFF7CFFECD
:102070000A20FFF7F0FEA220FFF7EDFEF620FFF7A3
:10208000C6FE0120FFF7E7FE3020FFF7E4FEF22056
:10209000FFF7BDFE0020FFF7DEFE2620FFF7B7FEAC
:1020A0000120FFF7D8FEE020FFF7B1FE0F20FFF779
:1020B000D2FE3F20FFF7CFFE2F20FFF7CCFE0C20F3
:1020C000FFF7C9FE1020FFF7C6FE0A20FFF7C3FE88
:1020D0005320FFF7C0FED520FFF7BDFE4020FFF7DD
:1020E000BAFE0A20FFF7B7FE1320FFF7B4FE032065
:1020F000FFF7B1FE0820FFF7AEFE0320FFF7ABFEAF
:102100000020FFF7A8FEE120FFF781FE0020FFF787
:10211000A2FE0020FFF79FFE1020FFF79CFE032089
:10212000FFF799FE0F20FFF796FE0520FFF793FEBD
:102130002C20FFF790FEA220FFF78DFE3F20FFF737
:102140008AFE0520FFF787FE0E20FFF784FE0C2095
:10215000FFF781FE3720FFF77EFE3C20FFF77BFE76
:102160000F20FFF778FE1120FFF751FE782007F0CF
:10217000D9FB2920FFF74BFEBDE87040322007F065
:10218000D1BB000000802242947F00209881214230
:102190008081224210B5FB48002101604160C1608E
:1021A000C163A0F5C070F84A127A042A02D3F74836
:1021B000016001E0C0F88811FFF7C9FEBDE81040DA
:1021C00047F6196097E62DE9F05FDDE90A78002807
:1021D0001BD0EF4D18262424203B03EBC30000EB5B
:1021E000400005EB80058819401E00F0FF0C131914
:1021F000C8B25B1E6146FFF752FE7443E01704EB62
:102200005070C0F3CF0900262CE0E24D3026602448
:102210002D2B07D0202B08D0303B03EBC30005EB60
:102220008015E0E705F5B455DDE705F5C655DAE7B5
:1022300000244FEA182A4FEA172B2878E040C007FD
:1022400004D0F9B25846FFF7A7FD04E008F0FF01FB
:102250005046FFF7A1FD641CA4B2082CEDD36D1C01
:10226000761CB6B24E45E3D3BDE8F09F2DE9FC479E
:102270000746DDE90A890C4616461D4609E0B2B25A
:10228000A1B23846CDE90089FFF79DFF37B1173479
:102290006D1C2B78002BF2D1BDE8FC871F34F7E7CB
:1022A00070B51646049A01FB00F4A5B25418184400
:1022B000401EC1B2641ED8B22346FFF7F0FD0024D1
:1022C00007E036F81400C1B2000AFFF765FD641C90
:1022D000A4B2AC42F5D370BD2DE9F041089E069A38
:1022E00001FB00F4A5B254181844401EC1B2641E8C
:1022F000D8B22346FFF7D3FD0024370A05E0F1B238
:102300003846FFF749FD641CA4B2AC42F7D309E696
:102310002DE9FF5FA04F797801297AD19A4991F888
:102320006E200AB1462200E0432291F8C5B00A238C
:102330006426DFF868E22025002441424FF0300A8D
:102340004FF02D0C4FF02E084FF47A79BBF10A0FA5
:1023500026D0002870DB48456FDB90FBF9F1303167
:102360008DF8081090FBF9F109FB110191FBF6F1D2
:1023700030318DF8091090FBF6F106FB110191FB4D
:10238000F3F130318DF80A108DF80B8090FBF3F1EA
:1023900003FB110030308DF80C008DF80D4074E116
:1023A000002858DB48451BDB90FBF9F130318DF8F4
:1023B000081090FBF9F109FB110191FBF6F13031A6
:1023C0008DF8091090FBF6F106FB110090FBF3F07D
:1023D00030308DF80A008DF80B208DF80C4054E158
:1023E000642817DB90FBF6F130318DF8081090FB74
:1023F000F6F106FB110090FBF3F030308DF8090088
:102400008DF80A208DF80B508DF80C508DF80D408A
:102410003BE15EE10A2811DB90FBF3F030308DF8F0
:1024200008008DF809208DF80A508DF80B508DF8B2
:102430000C508DF80D4028E1C4E070E08DF808A044
:102440008DF809208DF80A508DF80B508DF80C503E
:102450008DF80D4019E170451BDC8DF808C091FB2B
:10246000F9F030308DF8090091FBF9F009FB1010FC
:1024700090FBF6F030308DF80A0091FBF6F006FB89
:10248000101090FBF3F030308DF80B008DF80C40FD
:10249000FBE010F1640F14DC8DF808C091FBF6F03E
:1024A00030308DF8090091FBF6F006FB101090FB20
:1024B000F3F030308DF80A008DF80B208DF80C40C9
:1024C000E3E010F10A0F16DC8DF808C091FBF3F081
:1024D00030308DF809008DF80A8091FBF3F003FB92
:1024E000101030308DF80B008DF80C208DF80D4059
:1024F0008DF80E50C9E08DF808C08DF809A08DF850
:102500000A8091FBF3F003FB101030308DF80B00C4
:102510008DF80C208DF80D408DF80E50B5E0642834
:102520001BDB90FBF6F130318DF8081090FBF6F1D3
:1025300006FB110191FBF3F130318DF809108DF894
:102540000A8090FBF3F103FB110030308DF80B0093
:102550008DF80C208DF80D4097E00A2820DB90FBC9
:10256000F3F130318DF808108DF8098090FBF3F10C
:1025700003FB110030308DF80A008DF80C208DF827
:102580000D4082E080812242947F00209881214288
:10259000E8E50308AC250308BA11002018FCFFFF8A
:1025A0008DF808A08DF8098090FBF3F103FB110072
:1025B00030308DF80A008DF80B208DF80C408DF826
:1025C0000D5062E070451BDC8DF808C091FBF9F0FE
:1025D00030308DF8090091FBF9F009FB101090FBE9
:1025E000F6F030308DF80A0091FBF6F006FB101083
:1025F00090FBF3F030308DF80B008DF80C4044E088
:1026000010F1640F14DC8DF808C091FBF6F0303047
:102610008DF8090091FBF6F006FB101090FBF3F02B
:1026200030308DF80A008DF80B208DF80C402CE02E
:1026300010F10A0F16DC8DF808C091FBF3F0303072
:102640008DF809008DF80A8091FBF3F003FB101060
:1026500030308DF80B008DF80C208DF80D408DF882
:102660000E5012E08DF808C08DF809A08DF80A8090
:1026700091FBF3F003FB101030308DF80B008DF858
:102680000C208DF80D408DF80E50FB4E307880B147
:10269000FA48007868B18DF808508DF809508DF827
:1026A0000A508DF80B508DF80C508DF80D408DF8B8
:1026B0000E5047F617604FF6FF71CDE9001002ABE0
:1026C0006C226A210120FFF7D1FD3078002800D16B
:1026D0007C70BDE8FF9F70B586B0E94DA9780129EF
:1026E00041D10021E74B202403AE01EBC0021A4484
:1026F00092F8812352B17254491CC9B20529F4D30E
:1027000093F86F000026012802D010E07454F3E71C
:10271000DD48007858B903F289334F2018706E20D5
:1027200058709E70DC701C715C719C71DC71D74CB0
:10273000207830B1D148007818B1D5A103A81BF09A
:10274000D5FE8DF8116047F617604FF6FF71CDE9A1
:10275000001003AB97226A210120FFF787FD207844
:10276000002800D1AE7006B070BD7FB5C44DE878CA
:10277000002830D0C34890F8A903022803D00128CC
:1027800006D050B10DE0C4A102A81BF0AFFE08E0D6
:10279000C3A102A81BF0AAFE03E0C3A102A81BF07C
:1027A000A5FEC34C207830B1B448007818B1C1A15F
:1027B00002A81BF09BFE47F617604FF6FF71CDE9AC
:1027C000001002ABC2226A210120FFF74FFD2078E2
:1027D000002800D1E8707FBDFEB5B84F38780028DA
:1027E0004BD000203870FDF79AFAB54947F61964C6
:1027F0004FF6FF7509784FF48976C1B3B8B33878CE
:10280000012847D0AF4ACDE90065B6232D21282005
:102810000294FFF745FDAC48017842788078114476
:10282000C14225D1A948007898B3012846D0022892
:102830004ED0032856D0042818D1FDF770FA01288D
:102840005AD0042858D0022860D005285ED003282A
:1028500066D0062864D0002808D19D4ACDE90065DD
:10286000DE232D210F200294FFF71AFDFEBD06E0A6
:10287000984A907901285DD06CE00120B2E7964A31
:10288000CDE90065B6232D2128200294FFF708FD2D
:10289000C1E709E0904ACDE90065B6232D21282043
:1028A0000294FFF7FDFCB6E7894ACDE90065DE2317
:1028B0002D210F200294FFF7F3FCD7E7874ACDE9DB
:1028C0000065DE232D210F200294FFF7E9FCCDE700
:1028D000834ACDE90065DE232D210F200294FFF706
:1028E000DFFCC3E77F4ACDE90065DE232D210F2001
:1028F0000294FFF7D5FCB9E7784ACDE90065DE23FD
:102900002D210F200294FFF7CBFCAFE7744ACDE9ED
:102910000065DE232D210F200294FFF7C1FCA5E7FF
:10292000704ACDE90065DE232D210F200294FFF7C8
:10293000B7FC9BE7D17901290CD0117A012909D084
:10294000CDE90065DE23654A2D210F200294FFF7B3
:10295000A7FC8BE7D17901290ED101280CD0137A7D
:10296000012B09D0CDE90065DE235D4A2D210F2022
:102970000294FFF795FC79E7127A012A0DD101281C
:102980000BD0012909D0CDE90065DE23554A2D2160
:102990000F200294FFF784FC68E7CDE90065DE2391
:1029A0004B4A2D210F200294FFF77AFC5EE72DE9B8
:1029B000FE4FFDF7CAF907464B48DFF8C48001789F
:1029C000B94203D0012188F805100770DFF8B490F0
:1029D0004FF6FF764FF0000A99F8670299F86812EF
:1029E00099F86A22084499F8691247F61964114463
:1029F000C8424FF489753ED0DFF8D8B09BF800008C
:102A000001280DD19BF80110012909D0CDE900560C
:102A10000223364A2D2137200294FFF741FC18E0AB
:102A20009BF8011001290BD1012809D0CDE90056EE
:102A300002232F4A2D2137200294FFF731FC08E0B2
:102A4000CDE90054022300222D2137200294FFF704
:102A500043FC9BF8020001284ED19BF8031001298A
:102A60004AD0CDE900563E23224A2D213720029438
:102A7000FFF716FC23E159E0380000203B0000205E
:102A8000BA110020947F0020370000203900002078
:102A900020202020202020004865617420000000B4
:102AA000436F6F6C200000004175746F20000000C0
:102AB0003A000020202020202000000008010020F3
:102AC00034000020808A0308018200204300002097
:102AD0005867030888090020707C03089E6C03086F
:102AE000E47103082A770308660000209098030821
:102AF000E6AB0308AC4003089BF8031001290BD197
:102B0000012809D0CDE900563E23FD4A2D2137206A
:102B10000294FFF7C5FBD2E0CDE900543E2300222A
:102B20002D2137200294FFF7D7FBC8E099F8B9129E
:102B3000F448012919D098F8041000299AD00068A7
:102B4000002877D0CDE900540223EF4A2D21372009
:102B50000294FFF7A5FBCDE900563E23EB4A2D2159
:102B600037200294FFF79CFBA7E00068C0B198F8FB
:102B70000400002813D0CDE90054022300222D21A7
:102B800037200294FFF7A8FBCDE900563E23DF4A29
:102B90002D2137200294FFF783FB88F804A08EE0F4
:102BA000DFF86CB39BF80000092830D004DC012862
:102BB00007D0042864D117E00A283CD00B285FD145
:102BC0004CE0CDE900560223CF4A2D213720029454
:102BD000FFF766FBCDE900563E23CC4A2D21372076
:102BE0000294FFF75DFB4BE0CDE900560223C64A95
:102BF0002D2137200294FFF753FBCDE900563E23E9
:102C0000BF4A2D2137200294FFF74AFB38E0CDE977
:102C100000560223BF4A2D2137200294FFF740FBC4
:102C2000CDE900563E23B94A2D2137200294FFF703
:102C300037FB25E029E0CDE900560223B54A2D21D6
:102C400037200294FFF72CFBCDE900563E23AC4A17
:102C50002D2137200294FFF723FB11E0CDE900542A
:102C6000022300222D2137200294FFF735FBCDE906
:102C700000543E2300222D2137200294FFF72CFB25
:102C8000A5499BF80000087019E0A448007818B323
:102C900099F87600B0B3CDE9005402239D4A2D2166
:102CA00037200294FFF7FCFACDE900563E23974AFD
:102CB0002D2137200294FFF7F3FA88F804A099F841
:102CC0006B0299F86C12C84268D0DFF8549299F8F8
:102CD000040001282BD039E099F8760098B1CDE9AD
:102CE00000540223884A2D2137200294FFF7D8FA96
:102CF000CDE900563E23824A2D2137200294FFF76A
:102D0000CFFADAE709E0CDE900540223814A2D2108
:102D100037200294FFF7C4FAEAE7CDE90054022312
:102D2000794A2D2137200294FFF7BAFABCE799F8C7
:102D3000051001290AD0CDE900567A23794A2D21C0
:102D400037200294FFF7ACFABDE8FE8F99F8051022
:102D500001290BD1012809D0CDE900567A23724A06
:102D60002D2137200294FFF79BFAEDE7012801D1CE
:102D7000012901D048B941B9CDE900547A23002294
:102D80002D2137200294FFF7A7FA99F80400642850
:102D900008D099F80500642804D0D5E798F8050014
:102DA0000128D1D127B1012F0CD0022F1DD113E062
:102DB000CDE900547A2300222D2137200294FFF719
:102DC0008BFA12E0CDE900567A23574A2D2137209D
:102DD0000294FFF765FA08E0CDE900567A23514ADC
:102DE0002D2137200294FFF75BFA88F805A0ABE7A6
:102DF0001CB547F61964012808D000944BA3C222E1
:102E0000002101200194FFF731FA1CBD009447A373
:102E10006C22002101200194FFF728FA009443A3BB
:102E20009722002101200194FFF720FA1CBD3EB536
:102E300047F619654FF6FF7467208DE831000023CF
:102E40001A462D21EF20FFF747FA92208DE8310036
:102E500000231A462D21EF20FFF73EFABD208DE812
:102E6000310000231A462D21EF20FFF735FA3EBD31
:102E70002DE9FF4764250A2320244FF0000C4FF46E
:102E80007A77202A29D02E264FF0300900297DDBC1
:102E9000B9427CDB91FBF7F030308DF8080091FBF4
:102EA000F7F007FB101090FBF5F030308DF80900BB
:102EB00091FBF5F005FB101090FBF3F030308DF82E
:102EC0000A008DF80B6091FBF3F003FB101030301B
:102ED0008DF80C008DF80D20D3E0B9423FDB91FB5B
:102EE000F7F030308DF8080091FBF7F007FB101079
:102EF00090FBF5F030308DF8090091FBF5F01FE004
:102F0000025403085400002090980308AC400308C2
:102F10003F000020E6AB03083600002043000020FD
:102F20008809002092D203083CBF030820202020FB
:102F30002020202020202020202020200000000011
:102F400005FB101090FBF3F030308DF80A0091FB78
:102F5000F3F003FB101030308DF80B0046E06429CD
:102F60001EDB91FBF7F007FB101090FBF5F0303003
:102F70008DF8080091FBF5F005FB101090FBF3F0C5
:102F800030308DF8090091FBF3F001E07CE034E093
:102F900003FB101030308DF80A008DF80B4025E04F
:102FA0000A2914DB8DF8084091FBF5F005FB1010A1
:102FB00090FBF3F030308DF8090091FBF3F003FB48
:102FC000101030308DF80A008DF80B400EE000290B
:102FD0000CDB8DF8084091FBF3F003FB1010303050
:102FE0008DF809008DF80A408DF80B408DF80C40E3
:102FF0008DF80D408DF80EC0A7E064291BDB91FB16
:10300000F5F030308DF8080091FBF5F005FB10105D
:1030100090FBF3F030308DF809008DF80A6091FBD9
:10302000F3F003FB101030308DF80B008DF80C20FE
:103030008DF80D4025E00A2912DB91FBF3F03030CA
:103040008DF808008DF8096091FBF3F003FB101078
:1030500030308DF80A008DF80C208DF80D4010E00E
:103060008DF808908DF8096091FBF3F003FB1010C8
:1030700030308DF80A008DF80B208DF80C408DF85B
:103080000D408DF80EC060E048424FF02D0811F55C
:103090007A7F24DC8DF8088090FBF7F130318DF8D1
:1030A000091090FBF7F107FB110191FBF5F13031AD
:1030B0008DF80A1090FBF5F105FB110191FBF3F17E
:1030C00030318DF80B108DF80C6090FBF3F103FBA1
:1030D000110030308DF80D008DF80E2033E011F125
:1030E000640F1DDC8DF8088090FBF5F130318DF810
:1030F000091090FBF5F105FB110191FBF3F1303163
:103100008DF80A108DF80B6090FBF3F103FB1100B2
:1031100030308DF80C008DF80D208DF80E4012E047
:103120008DF808808DF809908DF80A6090FBF3F116
:1031300003FB110030308DF80B008DF80C208DF85A
:103140000D408DF80E408DF80FC047F619604FF610
:10315000FF71CDE9001002ABC22200210120FFF770
:1031600085F8BDE8FF877CB50E4647F619654FF632
:10317000FF7403466C2200210120CDE90045FFF7D2
:1031800075F83346972200210120CDE90045FFF76D
:103190006DF87CBD2DE9FE4F05460C4647F61969D2
:1031A0004FF6FF768DE8500208212B46FC4A084670
:1031B000FFF776F8A01C47F6176A80B28DE8410445
:1031C000AB1D002201217120FFF786F804F10800F1
:1031D000CDE9016A87B2AB1C00221C2102200097B6
:1031E000FFF77AF804F12200CDE901691FFA80F8AF
:1031F000EB4A08212B4680320846CDF80080FFF7C5
:103200004FF804F1270080B28DE84104AB1D002285
:1032100001217120FFF760F8CDE9016905F1730321
:10322000CDF8008008219846DE4A0846FFF738F8B6
:10323000DC4A8DE850020821434680320846FFF7F9
:103240002FF8CDE9016A05F1780300221C21012045
:103250000097FFF741F804F128004BF69C6780B215
:103260008DE8C1006B1D002202217320FFF734F8A6
:103270008DE8D0006B1D002202217320FFF72CF88F
:10328000A41DA4B28DE8D0002B46002220210220EC
:10329000FFF722F88DE8D00005F179030022202104
:1032A0000220FFF719F84FE5F0B5BF4D2E27642334
:1032B0000A242026C2EB02122A44002816DA2D2105
:1032C0005172404290FBF3F13031917290FBF3F177
:1032D00003FB110191FBF4F13031D172177390FBB4
:1032E000F4F104FB11003030507358E0DFF8BCC239
:1032F0004FF47A7561444FF0250CA84237DB91F802
:10330000E51002291BD090FBF5F13031517290FB92
:10331000F5F105FB110191FBF3F13031917290FB56
:10332000F3F103FB110191FBF4F13031D17217730A
:1033300090FBF4F104FB1100303050732FE090FB50
:10334000F5F13031517290FBF5F105FB110191FB64
:10335000F3F13031917290FBF3F103FB110090FB1C
:10336000F4F03030D07282F80CC0567317E090FB46
:10337000F3F53035557290FBF3F503FB150393FB22
:10338000F4F330339372D77290FBF4F304FB130021
:103390003030107391F8E500022802D0567396730E
:1033A000F0BD82F80DC0FAE72DE9F05F7F4890F894
:1033B000B812092902D9092180F8B81290F8B81278
:1033C000002973D000243A27DFF8E4814FF00A097E
:1033D0004FF0640A2025744E12E2081990F8BA02E0
:1033E000C01E0E281CD2DFE800F0071E354C647B9F
:1033F00092A9C0FAE7E6E5DA0020C4EB04123244F1
:103400000B1893F8A93163B11354401CC0B20828BB
:10341000F6D31772B8F9000022460021FFF744FFE7
:10342000ECE11554F1E70020C4EB041232440B1810
:1034300093F8B13163B11354401CC0B20828F6D3DD
:103440001772B8F9020022460021FFF72DFFD5E1DF
:103450001554F1E70020C4EB041232440B1893F822
:10346000B93163B11354401CC0B20828F6D31772A7
:10347000B8F9040022460021FFF716FFBEE11554FB
:10348000F1E70020C4EB041232440B1893F8C13169
:103490006BB11354401CC0B20828F6D31772B8F9A8
:1034A000060022460021FFF7FFFEA7E1AEE115541A
:1034B000F0E70020C4EB041232440B1893F8C93132
:1034C00063B11354401CC0B20828F6D31772B8F980
:1034D000080022460021FFF7E7FE8FE11554F1E7CF
:1034E0000020C4EB041232440B1893F8D13163B1BD
:1034F0001354401CC0B20828F6D31772B8F90A005A
:1035000022460021FFF7D0FE78E11554F1E70020B4
:10351000C4EB041232440B1893F8D93163B113543D
:10352000401CC0B20828F6D31772B8F90C00224626
:103530000021FFF7B9FE61E11554F1E70020C4EB6B
:10354000041232440B1893F8E13163B11354401C58
:10355000C0B20828F6D31772B8F90E00224600212F
:10356000FFF7A2FE4AE11554F1E7FCF7EEFBC4EBCE
:1035700004105321315400EB060B74218BF8011019
:1035800061208BF8020067208BF8030065208BF820
:1035900004008BF80570FCF7C2FB00210EE0F4E09C
:1035A000FC0D0408FC0E040810010020947F00208C
:1035B0003C120020B3E074E022E010E0FB4AC0EBD4
:1035C000C00010440BEB0103425C9A71491CC9B264
:1035D0000729F7D38BF80D508BF80E500EE1002021
:1035E000C4EB041232440B1893F8913133B11354E5
:1035F000401CC0B20E28F6D39573FFE01554F7E7D0
:10360000EB498879EB4B401E00EB800003EB400058
:103610004278C4EB041032548A793044521E02EBD3
:10362000820203EB4202927842708A79521E02EBC8
:10363000820203EB4202D2788270C570CA79B2FB73
:10364000F9F230320271CA79B2FBF9F309FB1322A5
:10365000303242712C2282718B884FF47A72B3FB24
:10366000F2F33033C3718B88B3FBF2FC02FB1C32E4
:10367000B2FBFAF2303202728A88B2FBFAF30AFB2A
:103680001322B2FBF9F2303242728988B1FBF9F2AF
:1036900009FB121130318172C57205734573857350
:1036A000ACE0C4EB04105421315430446921417022
:1036B0006D2181706521C1700571BF4909780329A9
:1036C0001FD0BB4A1178B1FBF9F13031417111784B
:1036D000B1FBF9F309FB131130318171C7715178D6
:1036E000B1FBF9F1303101725178B1FBF9F209FB0C
:1036F0001211303141728572C5720573457385733D
:103700007CE04521417172218171C1716F22027289
:1037100041728572C5720573457385736EE0C4EBA3
:1037200004104321315430444F21417032218170C3
:10373000C770A2494FF47A720988914204D3B1FB51
:10374000F2F33033037100E00571B1FBF2F302FBD9
:103750001312B2FBFAF230324271B1FBFAF20AFBF9
:103760001212B2FBF9F230328271B1FBF9F209FBAD
:1037700012113031C1717021017241726D2181725B
:10378000C57205734573857338E0C4EB0410482196
:1037900031543044752141706D2181706921C170AF
:1037A00080F804A04171742181717921C17107727F
:1037B0008349B1F90010B1F57A7F08DB31214172FC
:1037C00030218172C17225210173457315E091FB8F
:1037D000FAF23032427291FBFAF20AFB121292FBB9
:1037E000F9F2303282722E22C27291FBF9F209FB99
:1037F000121130310173252141738573641CE4B2C9
:10380000704991F8B802A0423FF6E7ADBDE8F09FDD
:103810002DE9FC5FFFF7C8FDDFF8A8816A4C6B4D0E
:1038200098F8B812002647F617674FF6FF7B99B94C
:103830000020491EC1EB011129440A5C2254401C9E
:10384000C0B20A28F9D3A672CDE900B75E4BED22CB
:1038500000210120FEF70AFD98F8B802002842D0A6
:10386000DFF86891401EA9F10809C0EB0010421969
:10387000D9F80410501C88421CD80020531A03F1B8
:103880000F0C05E011F8008004F80080401CC0B265
:103890008445F7DC0020A1EB020808E003EB000AF6
:1038A000A24415F800C08AF80FC0401CC0B2804581
:1038B000F4DC06E000200B5C2354401CC0B20A2854
:1038C000F9D30E328A4202D1C9F8045002E0491CF1
:1038D000C9F80410A672CDE900B73B4BED221E21BA
:1038E0000120FEF7C3FCBDE8FC9FF0B587B004469D
:1038F00047F617664FF47847CDE90176ED200023AF
:1039000000901A461E21EF20FEF7E6FC0021274A10
:103910002E4D8C3204A802F11E03083D14B1012C77
:1039200008D00EE095F801C08C4412F80CC000F8E5
:1039300001C006E095F801C08C4413F80CC000F8F3
:1039400001C0491CC9B20A29E8D300248DF81A40E5
:10395000CDE9007604ABED221E210120FEF786FCA6
:103960006878192803D2401C687007B0F0BD6C70ED
:10397000FBE70EB555224FF6FF71002809D0CDE9BF
:103980000021029108218B2300220846FEF7A4FCA7
:103990000EBDCDE9002147F61960029008218B2366
:1039A00000220846FEF798FC0EBD0000E424030840
:1039B000B01100205C1A03081F03002062020020DF
:1039C00066020020947F0020C31100201001002017
:1039D0002DE9F04F87B00D464FF0270B05210491DC
:1039E0005721069105210391972105910521029107
:1039F0004FF47A7A47F619664FF6FF7700287AD1A6
:103A00004FF00A094FF06408002D76DB2C46AFF624
:103A10007473CDE90076202206210120FEF726FCF2
:103A2000554534DB94FBF9F004B2642C0BDB94FBBA
:103A3000F8F03030CDE90076C3B259460020049A40
:103A4000FEF7C1FB07E0CDE90076202359460020B0
:103A5000049AFEF7B8FB94FBF8F008FB104090FBCB
:103A6000F9F0CDE900763030C3B20020039A069910
:103A7000FEF7A9FB94FBF9F009FB1040CDE90076B5
:103A80003030C3B20020029A0599FEF79CFB5545E1
:103A900031DA642D0BDB94FBF8F03030CDE90076A1
:103AA000C3B259460020049AFEF78DFB07E0CDE92A
:103AB0000076202359460020049AFEF784FB94FBED
:103AC000F8F008FB104090FBF9F0CDE900763030BB
:103AD000C3B20020039A0699FEF775FB94FBF9F038
:103AE00009FB1040CDE900763030C3B20020029AC5
:103AF0000599FEF768FB68E0FFE7684204B2642CB2
:103B00002FDB94FBF8F03030CDE90076C3B2594694
:103B10000020049AFEF757FB94FBF8F008FB1040D6
:103B200090FBF9F0CDE900763030C3B20020039A63
:103B30000699FEF748FB94FBF9F009FB1040CDE92C
:103B400000763030C3B20020029A0599FEF73BFBA5
:103B5000CDE9007630A3202206210120FEF786FB66
:103B600033E0CDE90076202359460020049AFEF781
:103B70002AFB94FBF8F008FB104090FBF9F0CDE92C
:103B800000763030C3B20020039A0699FEF71BFB83
:103B900094FBF9F009FB1040CDE900763030C3B258
:103BA0000020029A0599FEF70EFBCDE900761BA3D3
:103BB000202206210120FEF759FBCDE9007616A34D
:103BC000202228210120FEF751FB554503DD00206E
:103BD000FFF7CFFE02E00120FFF7CBFE104C20786C
:103BE00001280DD10F4890F86E0060B1CDE9007644
:103BF0000DA33822D6210120FEF738FB00202070CB
:103C000007B0BDE8F08FCDE9007608A33822D621B1
:103C10000120FEF72BFBF1E72D0000002000000043
:103C2000BA110020947F00204600000043000000ED
:103C300010B5254C01212046FDF7E2F8012803D1FB
:103C400022490A68521C0A602149088841F28832D8
:103C5000904203D20A88521C0A8001E000200880AA
:103C60002046BDE810400121FDF7D1B87FB50446DC
:103C70000D4601211020FCF7DDF9ADF80840ADF844
:103C800004500020ADF80A00ADF806000E4C01A962
:103C90002046FCF7A1FB36218DF8001001218DF89C
:103CA000011003228DF802208DF803106846F4F706
:103CB00038FD012211462046FCF779FE01212046FD
:103CC000FCF75BFE7FBD00000010004040020020BA
:103CD000BA060020FE49097A05290BD2FD4A20B117
:103CE000883291881068F5F703B988329188106896
:103CF000F5F700B9F84A18B102211046F5F7F8B8FF
:103D000002211046F5F7F6B8F149097A05290BD2D8
:103D1000F04A20B1943291881068F5F7E9B89432EE
:103D200091881068F5F7E6B8EB4A18B10121104602
:103D3000F5F7DEB801211046F5F7DCB8E449097A59
:103D400005290BD2E34A20B1A03291881068F5F71B
:103D5000CFB8A03291881068F5F7CCB8DE4A18B118
:103D600010211046F5F7C4B810211046F5F7C2B877
:103D7000D749097A05290BD2D64A20B1AC329188AD
:103D80001068F5F7B5B8AC3291881068F5F7B2B89D
:103D9000D14A18B108211046F5F7AAB808211046F3
:103DA000F5F7A8B8CA49097A05290BD2C94A20B142
:103DB000B83291881068F5F79BB8B83291881068CE
:103DC000F5F798B8C44A18B104211046F5F790B831
:103DD00004211046F5F78EB8BD49097A05290BD2A2
:103DE000BC4A20B1C43291881068F5F781B8C4325A
:103DF00091881068F5F77EB8B74A18B120211046AF
:103E0000F5F776B820211046F5F774B82DE9FC4196
:103E1000F220ADF8040000258DF8075002248DF83B
:103E20000640AE4E01A93046F4F7F3FF0320ADF88B
:103E300004008DF807508DF80640A94F01A93846B7
:103E4000F4F7E7FF2320ADF804008DF807508DF854
:103E50000640DFF8908201A94046F4F7DAFF9C485B
:103E60001025007A052816D21C20ADF804008DF824
:103E700007508DF8064001A94046F4F7CAFFE0203C
:103E8000ADF804008DF807508DF8064001A93046C2
:103E9000F4F7BFFF15E03F20ADF804008DF80750A0
:103EA0008DF8064001A98C48F4F7B3FF0C20ADF85B
:103EB00004008DF807508DF8064001A94046F4F73C
:103EC000A8FF4FF40076ADF800608DF803508DF830
:103ED000024069463846F4F79CFF01213046FCF762
:103EE0009EF8BDE8FC8110B586B04FF40040FCF7A9
:103EF00019F801214802FCF792F8002001908DF892
:103F000008008DF809004FF460210391049001200E
:103F10008DF81400744C01A92046F4F785FC0121AA
:103F20002046F4F7A9FC2046F4F7C9FC2046F4F734
:103F3000CBFC0128FAD02046F4F7CDFC2046F4F75C
:103F4000CFFC0128FAD006B010BD2DE9F047054698
:103F5000042B06D0062B04D0842B05D0862B03D04F
:103F600004E04FF4FA7001E04FF47A70DFF860C1BA
:103F700005F114036344DC7E1B7F04EB032340F252
:103F8000FF345A4FA14203DBFB6418B2BDE8F0874F
:103F900001EB81014E0096FBF0F10CB2CAB1611C3D
:103FA00005EB41016144CA7E097F02EB012305EB69
:103FB00044016144CA7E097F02EB01255D1B00FBC1
:103FC00014636B4393FBF0F000EB01201044F864A2
:103FD00033E005EB4401614411F8312F497802EBDD
:103FE0000122611C05EB4101614491F8315091F8C7
:103FF000328005EB0821A2EB01091DF0B3FA8246DD
:1040000048461DF097FA814630461DF093FA064661
:10401000601C1DF08FFA51461DF0ECFA31461DF080
:10402000BFFB49461DF0E6FA51461DF051F91DF05F
:1040300045FA00EB08202844F864B7F84C0000B2B9
:10404000A4E770B5224C294B0A281FD00A220B285E
:104050002BD0274D231835F9106093F8F73006FB65
:10406000031101EB810149005B1C91FBF3F191FB12
:10407000F2F302FB1313052B00DB0A3191FBF2F381
:1040800025F8103091FBF2F000B270BD587A052887
:1040900000D2998394F86000B3F91C2002FB001150
:1040A000401C91FBF0F09883EEE794F829039C8D77
:1040B00004FB001101EB81014900401C91FBF0F071
:1040C00090FBF2F102FB1101052900DB0A3011E03F
:1040D000947F0020182403080018014000080140C4
:1040E000000C014000100140002401404402002067
:1040F0001412002090FBF2F1998590FBF2F0C3E7D7
:1041000010B512224FF4E164132907D0142932D0DC
:10411000FE4B997C814251DD204610BDFC4B997CC1
:10412000814201DD204610BD521E52B29C5C2144EA
:1041300081421DDD081A64214843995C90FBF1F02F
:10414000042A09DB121F02EBC20101EB021100EB92
:104150008100C0F30E0009E002EBC20101EB021185
:1041600000EB8100C0F5C87040F4004000B210BD03
:10417000002AD9D148E00921E64B5A8A824202DD61
:104180004FF4AF7010BD491E49B233F811402244BC
:10419000824210DD101AC0EB0010400033F81120ED
:1041A00090FBF2F0C1EB011100EB4100C0F30E00F7
:1041B000463000B210BD0029E5D125E0521E52B2B2
:1041C0009C5C214481421DDD081A64214843995CAE
:1041D00090FBF1F0042A09DB121F02EBC20101EB94
:1041E000021100EB8100C0F30E0009E002EBC201F6
:1041F00001EB021100EB8100C0F5C87040F40040F3
:1042000000B210BD002AD9D1C34810BD2DE9F0413C
:104210000746C248B0F92E50B0F93040281B1DF0B7
:1042200089F9BF4E31461DF053F88046C8204443FB
:10423000684200EB800004EBC0001DF07BF93146C2
:104240001DF046F8B74C21461DF0D4F90546384616
:104250001DF088F941461DF0CDF929461CF0CAFF32
:1042600021461DF035F81DF029F900B2BDE8F081B6
:104270002DE9F0471D46AC4E40F2062301FB03F743
:1042800096F878344FF47A784FF0640900283AD0E1
:104290000E2838D063283CD04FF4966A01FB0AFC04
:1042A00040F2FF3A802836D08B2834D0012835D010
:1042B0000B2833D00D2831D0022855D082285ED06B
:1042C000032867D0052865D0072863D0082861D067
:1042D00009285FD00A285DD0832873D0852871D043
:1042E00087286FD088286DD089286BD08A2869D01C
:1042F000042873D0842871D0062870D086286ED008
:104300000C286DD0D5E097FBF8F0434393FBF9F20E
:10431000CFE00A46CDE09CFBFAF2CAE0012816D0B5
:104320000D2819D088B21321FFF7EAFE010402D547
:10433000C0F30E00404296F86E1031B100EBC000A1
:10434000052190FBF1F000F5A0704219B1E088B2B0
:104350000221FFF7D5FEE9E788B21421FFF7D0FE6E
:104360004628E3DA4620E1E708461CF09AFC6F4A4B
:104370006F4B1CF0E9FC1CF065FC024699E0084616
:104380001CF08FFC6B4A6C4B1CF0DEFC1CF05AFCE2
:1043900002468EE0B1F5F17F09DC052805D008283A
:1043A00003D00A2801D0012283E0002281E0032803
:1043B00006D0072804D0092802D0012279E001E0C4
:1043C000002276E04FF4FA7399420CDC852808D07D
:1043D000882806D08A2804D001226AE00FE032E063
:1043E00055E0002265E0994263DD832805D08728E7
:1043F00003D0892801D001225BE0002259E0042883
:1044000002D0842803D004E097FBF8F201E09CFB83
:10441000FAF2534393FBF9F1404A3A3204281278F6
:1044200002D0842807D00CE0042309B20020FFF753
:104430008CFD044605E0842309B20020FFF785FDCA
:104440000446621935E0062802D0862803D004E02D
:1044500097FBF8F201E09CFBFAF2534393FBF9F16E
:104460002E4A3A320628527802D0862807D00CE02D
:10447000062309B20020FFF768FD044605E0862305
:1044800009B20020FFF761FD0446621911E00846F9
:104490001CF007FC294A2A4B1CF056FC1CF0D2FBEE
:1044A0004FF4C871884200DA084680B2FFF7AEFECA
:1044B000024610B26AE5811E0B2910D2DFE801F036
:1044C0000B0F0F0606060606060606001D49401FCE
:1044D00031F9100070471148B0F93E0070470020D4
:1044E00070478008704770B505460C460221284683
:1044F000F4F711FB0523012221462846F4F71EFAA2
:1045000001212846F4F7F3F902211DE0221A0308DD
:10451000351A0308481A0308E883FFFF4402002005
:104520000000204300002041947F002039B4C87669
:10453000BE9FBA3FC1CAA145B6F3BD3F5C8FC2F56D
:10454000285CDF3F3C1200202846F4F7DDFA002803
:10455000DAD02846BDE87040F4F736BA2DE9F047C6
:104560004FF000084FF001090027DFF844A40F21A5
:104570005046FFF7B8FF04B2A044B9F1010F36D09E
:10458000A64200DC2646B6B2A54200DA2C46A5B209
:104590000A2005F0A7F97F1CFFB20C2FE7D3A8EB88
:1045A0000600401B0A21B0FBF1F080B2FFF799FF33
:1045B00001B20A20FFF745FDFE4D95F85F10132963
:1045C0001AD014291DD080B20221FFF799FDFA4CB0
:1045D000E08400EBC001052291FBF2F101F5A0712E
:1045E00009B2218595F86E2082B1E1870FE0A6B26D
:1045F000A5B24FF00009CBE780B21321FFF780FD91
:10460000E5E780B21421FFF77BFDE0E7E087E08F6C
:10461000A4F84000618D0844E087E6480021D530C9
:10462000F6F7C0FB38B195F87B0395F87A1300EBE9
:104630000120A084AAE495F85F00A8B1022816D052
:10464000132814D0042815D0DC49032818D01028CA
:104650001ED0112824D012282FD0421F072A3DD85F
:1046600031F81200A0843FE0E08FA0843CE0E08FAE
:10467000A08439E0208F94F901100844A08433E02D
:10468000B1F90000B4F93E1008444010A0842BE0BA
:10469000B1F90000B1F9021008444010A08423E0F1
:1046A000B1F90000B1F90220B1F904101044084436
:1046B000032190FBF1F0A08416E0B1F90000B1F9FC
:1046C00002201044B1F90420B1F906101144084445
:1046D000C11700EB91708010A08405E0012808D07C
:1046E000152809D0E08FA08495F8A20015280FD0D6
:1046F00019E00888A084F7E795F82703FFF7DBFEA9
:10470000034695F82803FFF7D6FE181AA084EBE7B6
:1047100095F82703FFF7CFFE034695F82803FFF728
:10472000CAFE181AA087B4F92410A548814200DAFD
:10473000A084B4F9241040F6B83081427FF77AAFF4
:10474000A08423E410B50D2828D00ADC0D283DD222
:10475000DFE800F02C242C242C24242424242424DA
:104760003400862812D00EDC83280FD006DC0E28F9
:104770001CD080280AD0822828D107E0842805D0C0
:10478000852823D102E0873804281FD80120FFF7AD
:10479000BBFABDE810400020FFF79CBA0120FFF7EC
:1047A000B3FABDE810400120FFF794BA0020FFF7EC
:1047B000ABFABDE810400120FFF78CBA0020FFF7EC
:1047C000A3FABDE810400020FFF784BA10BD10B571
:1047D00008285DD2DFE800F0040F1A25303B46516F
:1047E0000020FFF7DFFA0020FFF7C2FABDE8104013
:1047F0000020FFF7A3BA0020FFF7D4FA0020FFF74C
:10480000B7FABDE810400120FFF798BA0020FFF783
:10481000C9FA0120FFF7ACFABDE810400020FFF70D
:104820008DBA0020FFF7BEFA0120FFF7A1FABDE81C
:1048300010400120FFF782BA0120FFF7B3FA0020F1
:10484000FFF796FABDE810400020FFF777BA012085
:10485000FFF7A8FA0020FFF78BFABDE8104001200F
:10486000FFF76CBA0120FFF79DFA0120FFF780FAED
:10487000BDE810400020FFF761BA0120FFF792FA6F
:104880000120FFF775FABDE810400120FFF756BA86
:1048900010BD02464749092A08D2DFE802F00705A1
:1048A000080B0E1114171A0091F89E02704791F828
:1048B0009F02704791F8A002704791F8A1027047DB
:1048C00091F8A202704791F8A302704791F8A402F0
:1048D000704791F8A50270472DE9FC5F0024354828
:1048E000DFF8D8B0D430ABF1140B01900120FFF702
:1048F00073FA21460198F6F755FA60B12D4800EB9E
:10490000440090F86B1390F86A0301EB00212B48E8
:1049100020F814108AE0601CC0B2FFF7BAFF062826
:1049200062D04FF000084FF0010A224800EB040962
:1049300099F8E500FFF706FF2046FFF748FF0A2039
:1049400004F0F0FF00270B211948FFF7CCFD80444D
:10495000BAF1010F4ED0854200D80546864200D2FA
:10496000304606460A2004F0BDFF7F1CFFB20C2F24
:10497000E9D3A8EB0500801B0A21B0FBF1F02BF86E
:10498000140099F8E5000C2805D03BF81400FFF757
:10499000A8FD2BF8140099F8E50003281DD0052880
:1049A0001BD0C11F032918D9832816D0852809E0F8
:1049B00000240140947F0020440200203C1200208B
:1049C0000CFEFFFF09D08738032806D93BF91410E5
:1049D0002046FFF736FB2BF8140099F8E500042871
:1049E0000DD084280BD011E0FD48818AFD4820F8C5
:1049F00014101BE0054606464FF0000AB2E7F849DE
:104A00008A7A082A01D2CC7200E08C723BF9141029
:104A100000232246FFF72CFC2BF81400F14938390B
:104A200031F814100144EF4820F81410641CE4B26B
:104A3000082CFFF45BAFEC4E0A213046FFF753FD24
:104A4000DFF89C83A8F80E0098F8020010B1012846
:104A50001BD02FE098F8000007282BD00220F8F791
:104A6000ABFE142004F05EFF0220F8F703FFABF862
:104A700010000020F8F7A0FE322004F053FF0020C1
:104A8000F8F7F8FEA8F8380014E0D549322048318C
:104A9000009001230022081F01F083FAD8F8440097
:104AA0001CF00CFDA8F83800D8F848001CF006FDF2
:104AB000ABF81000CD4890F8D91200297ED040F212
:104AC000DB20FCF7F0FF0002A8F8220040F2DA2019
:104AD000FCF7E9FFB8F822100844A8F82200B8F95A
:104AE00022004FF47A77B84201DDA8F82270B8F9B5
:104AF00022004FF00009002801DAA8F82290B8F946
:104B00002210B8F93800F8F724FFA8F81A00002599
:104B1000002408213046FFF7E6FC0544032004F09A
:104B200001FF641CE4B21E2CF3D31E20B5FBF0F091
:104B30001CF018FD044620461CF0DCFCA8F816000A
:104B4000AB4920461CF056FDAA491CF0C1FBAA49FE
:104B50001CF050FDA9491CF0BBFB1CF0AFFC01464A
:104B60000B20FFF76EFAA8F8160000250024092193
:104B70003046FFF7B8FC0544012004F0D3FE641C66
:104B8000E4B2142CF3D31420B5FBF0F064214843B5
:104B9000000B00EB4000A8F8180001213046FFF799
:104BA000A2FC00B243F6D00148430014A8F832003A
:104BB00004213046FFF797FC00B200E032E043F6F4
:104BC000D00148430014A8F834000C213046FFF708
:104BD0008AFCC0EBC0004000B0FBF7F0A8F8100062
:104BE0000D213046FFF77FFCC0EBC0004000B0FB5A
:104BF000F7F080B2A8F81200B8F810100F2901D809
:104C00000F284BD998F80C000A2802D2401D88F8CA
:104C10000C0098F80C000A2802D3012088F8030041
:104C2000BDE8FC9F90F80001754C70B3BBF9101003
:104C30000920FFF706FA2080B8F820100820FFF7B7
:104C400000FAB8F83610084480B2A8F81E004FF4F5
:104C5000C871884201D2A8F81E1098F802000128F5
:104C600018D098F80000072814D0B8F93810B4F913
:104C70000000F8F756FEA8F822006249B8F82200B2
:104C800009880844A8F8220029E7FFE7BBF81000CC
:104C90002080D1E72088A8F82200EEE798F80C00E1
:104CA00010B1401E88F80C0098F80C000028B7D10D
:104CB00088F80390B4E710B5FFF7A8F8BDE81040F6
:104CC000FFF711B9014600208A1E0B2A0BD2DFE83C
:104CD00002F00B0A0A06060606060606060041480A
:104CE000491F30F9110070473D48B0F93E00704748
:104CF0002DE9F0413A4A002050713A4E01216A3EB6
:104D00003578002D06D173880C2B02D93172517180
:104D100000E03072354B012D93F86E400CD193F8C2
:104D20006C54A54202D03172517100E03072B579F5
:104D30000DB1307200E031722A4F603F3E463D783F
:104D400076882DB90C2E02D93972517100E0387273
:104D5000012D0FD193F86DC4A44502D03972517161
:104D600000E0387297F806C0BCF1000F01D038722D
:104D700000E03972DFF86CC0ACF1560C9CF80070A2
:104D800057B9BCF80280B8F1020F03D98CF80810AB
:104D9000517101E08CF80800012F11D193F86E7465
:104DA000A74203D08CF80810517101E08CF808007C
:104DB0009CF8064014B18CF8080001E08CF808104B
:104DC000DFF820C0ACF1420C64469CF800706488A7
:104DD000E7B90E2C18D08CF80810517116E00000BD
:104DE000440200203C12002000240140947F002057
:104DF00000803B4500F07F450000204100007C42E0
:104E000074000020480000208CF80800012F0FD10A
:104E1000152C03D08CF80810517101E08CF80800B3
:104E20009CF8064014B18CF8080001E08CF80810DA
:104E3000DFF870C164469CF8007064883FB90E2C9E
:104E400003D08CF80810517101E08CF80800012F94
:104E50000FD1152C03D08CF80810517101E08CF89B
:104E600008009CF8064014B18CF8080001E08CF8AA
:104E7000081094793CB993F8B770022F02D0D17121
:104E8000517100E0D071012C07D193F8B840022C89
:104E900002D0D171517100E0D071002D05D193F88D
:104EA000A230B34203D011725171BDE8F08110728B
:104EB000FBE770B5FFF71CFF3B4E96F86A0401282C
:104EC00037D1384C39490A3CA4F11405B4F904002F
:104ED000B5F90430364A984203DA0420087010709D
:104EE00002E0002008701070287818B9A878FFF741
:104EF000E9FEA8802B4D143D287818B9A878FFF753
:104F0000E1FEA880207818B9A078FFF7DBFEA0802A
:104F100096F86B0401280CD1224926480A780AB970
:104F2000428C8A801F490A310A78002A01D1408CBC
:104F3000888070BDF0B51C4C0125002194F86A24CE
:104F40001C48012A0AD001710079012805D11A48AC
:104F50000288428004F89E1F6570F0BD42790AB154
:104F60000171F1E7104BDFF83CC094F86B645A7C98
:104F70009B7CACF11E0C02EB0322BCF904300CF15B
:104F800014079A1AB7F904301EB19A4207DD057169
:104F9000DAE79A4201DD0571D6E70171D4E70171C4
:104FA000D2E70000F0110020947F00204300002091
:104FB00034000020440200205C0000202DE9F04F66
:104FC000A1B001211020FBF72AF801212020FBF7D6
:104FD00026F801210820FBF722F8F84C4FF4005086
:104FE000217A04290BD30121FBF719F801211120A3
:104FF000FBF715F801210220FBF71CF806E0012160
:10500000FBF70DF801211120FBF709F8217AEC4894
:1050100018274FF00308042908D34FF0C001ADF85A
:1050200060104FF03001ADF8201003E04FF47071C4
:10503000ADF840100FD38DF863708DF8628018A919
:10504000F3F7E7FE8DF823708DF8228008A9DD487C
:10505000F3F7DFFE06E08DF843708DF8428010A96B
:10506000F3F7D7FE207A04280BD301210920FAF7A1
:10507000D6FF0121D448F3F75DFF0121D348F3F7B0
:1050800059FFCE4800250224007AD14E4FF0010985
:105090004FF47A7B4FF0700A042824D3ADF858B04F
:1050A000ADF85440ADF85A50ADF8565015A93046F9
:1050B000FBF792F9ADF844A0ADF84690ADF84C403E
:1050C000ADF818B0ADF81440ADF81A50ADF8165060
:1050D00005A9C048FBF780F9ADF804A0ADF806902B
:1050E000ADF80C4011E0ADF838B0ADF83440ADF893
:1050F0003A50ADF836500DA93046FBF76DF9ADF8D2
:1051000024A0ADF82690ADF82C40AC48007A0428D5
:1051100010D311A93046FBF798F911A93046FBF7D7
:10512000CDF901A9AB48FBF790F901A9A948FBF714
:10513000C5F90FE009A93046FBF787F909A9304600
:10514000FBF7BCF909A93046FBF7F8F909A9304685
:10515000FBF732FA08213046FBF712FD08213046F2
:10516000FBF714FD9548007A042808D308219948D4
:10517000FBF706FD08219748FBF708FD0FE0082123
:105180003046FBF7FDFC08213046FBF7FFFC082109
:105190003046FBF705FD08213046FBF707FD0121EE
:1051A0003046FBF7EAFB01213046FBF7F2FB012119
:1051B0000420FAF73FFF8148007A042807D3012131
:1051C0000220FAF737FF01218248FBF7D6FB0121C5
:1051D0002120FAF724FF01210803F3F7ABFE4FF477
:1051E000E040ADF880008DF883708DF8828020A9B2
:1051F0007948F3F70EFEADF878B0ADF87440ADF82D
:105200007A50ADF87650754D1DA92846FBF7E4F8A5
:10521000ADF864A0ADF86690ADF86C4019A92846C9
:10522000FBF713F919A92846FBF748F919A92846ED
:10523000FBF784F908212846FBF7A2FC0821284641
:10524000FBF7A4FC08212846FBF7AAFC012128460D
:10525000FBF793FB21B0BDE8F08F0B461146012B05
:1052600007D0022B07D0032B07D0042B07D1FBF765
:10527000AFBDFBF7A7BDFBF7A7BDFBF7A7BD704709
:1052800030B403464D4A534C5148127A062B2CD267
:10529000DFE803F02B1922030E26042A04D320464C
:1052A0000A4630BC0121D8E70A4630BC0321D4E7C6
:1052B000042A04D320460A4630BC0221CDE70A4620
:1052C00030BC0421C9E7464A9182D38A5B1CD38251
:1052D0000A4630BC0121C0E70A4630BC0221BCE7C7
:1052E0000A4630BC01213D48B7E730BC70473B4B14
:1052F000002804D04FF47A7203211846ADE700224B
:1053000003211846A9E7354B002804D04FF47A72E0
:1053100002211846A1E70022022118469DE72DE947
:10532000F84F83462F48421C02F1010A00789AF890
:1053300000101278BBF1080F6DD2DFE80BF06C049F
:105340000F1B27335561002500F0010601F0010411
:1053500002F00107A8464FF001095CE00125C0F307
:105360004006C1F34004C2F340074FF002084FF07B
:10537000030950E00225C0F38006C1F38004C2F3A4
:1053800080074FF004084FF0050944E00325C0F3FF
:10539000C006C1F3C004C2F3C0074FF006084FF0C7
:1053A000070938E00425C0F30016C1F30014C2F366
:1053B00000174FF008084FF009092CE0947F0020F7
:1053C00000100140000C01400004300000081A00E9
:1053D0000034014000040040001401400008004077
:1053E000608800209E0200200525C0F34016C1F30E
:1053F0004014C2F340174FF00A084FF00B090AE0BF
:105400000625C0F38016C1F38014C2F380174FF055
:105410000C084FF00D09B74245D1FF4841460089BD
:10542000F5F7A2FC0090A6B100200099884220D098
:105430008EB10022F84841460830F5F7A6FCF64840
:10544000F649009A0A3042B1294491F84211415577
:1054500007E00120E9E70122ECE7294491F849112E
:105460004155405D28B1EC48012249460830F5F726
:105470008CFCE94D49462889F5F776FC002812D1C5
:1054800085F801B007B90124BBF1080F0BD2DFE8A2
:105490000BF00A040C131A21282F9AF8000064F369
:1054A00000008AF80000BDE8F88F9AF8000064F365
:1054B00041008AF80000F6E79AF8000064F38200E1
:1054C0008AF80000EFE79AF8000064F3C3008AF856
:1054D0000000E8E79AF8000064F304108AF800007E
:1054E000E1E79AF8000064F345108AF80000DAE773
:1054F0009AF8000064F386108AF80000D3E72DE9DB
:10550000F84FC748DFF81C830078002823D0012417
:10551000DFF804A34FF000090AF1040AAAF101061A
:10552000F51EAF1C2046FFF7FAFE6878002877D0FA
:10553000012803D09AF80010CA0772D03878317861
:10554000401C60F3000131709AF8000020F0010067
:105550008AF80000CDE0B8F90000C82815DA4FF449
:105560007A710120FFF78CFE00210220FFF788FEF0
:1055700000210320FFF784FE00210420FFF780FEB6
:1055800000210520FFF77CFE61E0B0F5C87F15DA49
:1055900000210120FFF774FE4FF47A710220FFF71B
:1055A0006FFE00210320FFF76BFE00210420FFF7B0
:1055B00067FE00210520FFF763FE48E0B0F5167F87
:1055C00015DA00210120FFF75BFE00210220FFF722
:1055D00057FE4FF47A710320FFF752FE002104209A
:1055E000FFF74EFE00210520FFF74AFE2FE0B0F541
:1055F000487F17DA00210120FFF742FE0021022038
:10560000FFF73EFE00210320FFF73AFE4FF47A71C8
:105610000420FFF735FE00210520FFF731FE16E0DC
:1056200069E027E000210120FFF72AFE0021022087
:10563000FFF726FE00210320FFF722FE00210420B1
:10564000FFF71EFE4FF47A710520FFF719FE764C26
:10565000B8F8002002212046FFF7FFFDB8F802202D
:1056600003212046FFF7F9FDBDE8F84F4FF4FA702B
:1056700004F058B9022801D08A070BD5387832785F
:105680004010401C60F34102327021F002008AF8A1
:1056900000002EE0032801D04A070BD53878327875
:1056A0008010401C60F38202327021F004008AF8FE
:1056B00000001EE0042801D00A070BD538783278A4
:1056C000C010401C60F3C302327021F008008AF859
:1056D00000000EE0052801D0C8060AD538783278D7
:1056E0000011401C60F30412327021F010008AF89F
:1056F000000085F80190641CE4B2062CFFF412AFA0
:10570000DFF818A1DFF824B10AF1D6009AF86A1080
:105710000090062917D0002421460098F5F742FB97
:1057200078B30AEB040090F8B900032831D0214681
:105730003F48F5F737FB28B3002237482146C01C05
:10574000F5F716FB25E03B48007838B12878C0070C
:105750000DD0E9880120FFF793FD7BE000210120B7
:10576000FFF78EFD287800F0FE00287072E04FF4FD
:105770007A710120FFF784FD297841F00101297039
:1057800068E001E00122D8E72C482B4900EB8410A7
:10579000C1619BF80000012820D19AF85302022829
:1057A00002D001280ED014E021462548F5F7FAFA78
:1057B00030B1002218482146C01CF5F7D9FA08E09C
:1057C0000122F7E72CB98AF8D6900021D620FCF701
:1057D0006BF9042C02D103208BF80000641CE4B2A6
:1057E000052C99D396F80090164809F00101018024
:1057F0000024124850F824001BF07CFE1149A21C22
:1058000021F81200641CE4B2092CF2D35FEAC970DB
:1058100030D00021012017E09C020020947F00205E
:105820007F000020C6000020000800406200002029
:10583000FA8200204300002000007F437C84002087
:10584000E88100205A120020FFF71AFD287800F0A6
:10585000FE0028703078800723D4287880071BD476
:105860004FF47A710220FFF70BFD297841F0020115
:1058700029701EE02878C00704D0E9880120FFF7CE
:10588000FFFCE7E74FF47A710120FFF7F9FC297874
:1058900041F001012970DDE7E9880220FFF7F0FC03
:1058A00007E000210220FFF7EBFC287800F0FD0064
:1058B00028703078400711D42878400709D44FF475
:1058C0007A710320FFF7DCFC297841F0040129708C
:1058D0000CE0E9880320FFF7D3FC07E00021032058
:1058E000FFF7CEFC287800F0FB0028703078000726
:1058F00011D42878000709D44FF47A710420FFF7F7
:10590000BFFC297841F0080129700CE0E9880420E7
:10591000FFF7B6FC07E000210420FFF7B1FC287870
:1059200000F0F70028703078C00611D42878C0063F
:1059300009D44FF47A710520FFF7A2FC287840F0D3
:10594000100028700CE0E9880520FFF799FC07E0BB
:1059500000210520FFF794FC287800F0EF00287064
:105960009BF8000001280DD19AF85302022809D1B2
:10597000012205210098F5F7FBF901220621009884
:10598000F5F7F6F905210098F5F70CFA80B39BF8C6
:105990000000012803D19AF85302022811D09AF886
:1059A000620300029AF86313084400B29AF87B106D
:1059B00079B111290DD082B202215848FFF74DFC70
:1059C00026E09AF8560200029AF85512084400B2EE
:1059D000ECE7012805D0002202215048FFF73DFCEA
:1059E00016E04FF47A7202214C48FFF736FC0FE0C4
:1059F000FFE79AF87B00A8B101281ED004281CD02C
:105A000011280FD0B8F8002002214448FFF725FCE8
:105A100006210098F5F7C6F9F0B39BF800000128BD
:105A200024D027E03878800603D50120FFF76BFCEF
:105A3000EEE70020FFF767FCEAE79AF86A0401281E
:105A40000DD19AF86F04B8F9001000EB8002B1EBA9
:105A5000420F04DA00EB80004000A8F80000B8F81C
:105A6000002002212D48FFF7F8FBD1E79AF85302F6
:105A7000022816D09AF8640300029AF865130844C5
:105A800000B29AF87C1091B19AF87B1011290ED0CF
:105A900082B20321214800E01AE0BDE8F84FFFF789
:105AA000DCBB9AF857020102084400B2E9E701287A
:105AB00006D0BDE8F84F002203211848FFF7CDBB00
:105AC000BDE8F84F4FF47A7203211448FFF7C5BBC5
:105AD0009AF87C0068B1012818D0042816D0112843
:105AE00007D0B8F80220BDE8F84F03210B48FFF7B4
:105AF000B4BB3878400604D5BDE8F84F0120FFF765
:105B0000F6BBBDE8F84F0020FFF7F1BBB8F8022064
:105B1000BDE8F84F03210148FFF79FBB0008004094
:105B200010B5FBF7AAFD0120FBF7E1FD012003F012
:105B3000D9FE0120FBF7D0FD012003F0D3FE0020A9
:105B4000FBF7D5FD0A2003F0CDFE0020FBF7C4FDD6
:105B5000BDE810400A2003F0C5BE10B5FBF78DFD6F
:105B60000020FBF7B9FD012003F0BCFE0020FBF78D
:105B7000BEFD012003F0B6FE0120FBF7ADFD0A20BB
:105B800003F0B0FE0120FBF7B2FDBDE810400A2093
:105B900003F0A8BE70B50546FBF76FFD80242C42CC
:105BA00003D10020FBF7A3FD02E00120FBF79FFDDE
:105BB000052003F097FE0120FBF78EFD052003F082
:105BC00091FE0020FBF788FD012003F08BFE6408A6
:105BD000002CE4D1BDE87040FBF7F6BD70B50025A0
:105BE000FBF76EFD642407E0641EE4B201D20420DA
:105BF00070BD642003F076FEFBF789FD0028F3D02A
:105C0000284670BD2DE9F04105460E461746002096
:105C100028700120FBF76BFDFBF71EFD802401209F
:105C2000FBF75AFD012003F05DFE3846FFF7D6FF73
:105C30008046032003F056FEFBF733FDFBF762FDC1
:105C400010B12878204328700020FBF745FD012083
:105C500003F048FE6408002CE1D1FBF70EFDBEB155
:105C60000120FBF744FD012003F03CFE0120FBF77F
:105C700033FD052003F036FE0020FBF72DFD01204B
:105C8000FBF735FD142003F02DFE4046BDE8F08102
:105C90000020FBF72CFDE6E710B5FFF741FF0020E1
:105CA000FFF778FF002803D1BDE81040062071E718
:105CB00010BD0000F9494000087040F00100487034
:105CC0007047F7E7FFF749BF70B50546FF2000238F
:105CD00040F2311410E0EA5C50400822060603D579
:105CE00084EA4000C0B201E04006000E521ED2B26B
:105CF000002AF3D15B1CDBB28B42ECD370BD10B534
:105D00001446FFF7E1FFA04201D0022010BD0020A1
:105D100010BD7CB504460D46002101A8FFF772FFB7
:105D200028B9002211460DF10500FFF76BFF20B9DD
:105D3000002229466846FFF765FF28B99DF8002034
:105D4000022101A8FFF7DBFF9DF805109DF8042054
:105D500041EA022121807CBD10B5FFF7E1FECF486A
:105D60004078BDE81040FFF715BF70B50446200A23
:105D7000FFF710FF0546E0B2FFF70CFF284370BDA8
:105D800010B5FFF7CDFEC5480078BDE81040FFF71D
:105D900001BFF8B50646FFF7F3FF05464FF45E5026
:105DA000FFF7E3FF40EA050414B9FFF7D5FF044607
:105DB0002CB9642200216846FFF7ABFF044634B9D2
:105DC000002201210DF10200FFF7A3FF0446FFF7B7
:105DD00079FF34B9BDF80200BDF8001040EA014077
:105DE00030602046F8BD70B50546FFF7C9FF044690
:105DF00024B94FF22D30FFF7B8FF044614B9FFF76E
:105E0000ABFF04462CB9002201212846FFF781FF91
:105E10000446FFF757FF204670BD10B5FFF7B0FFEF
:105E2000044624B943F24100FFF79FFF0446FFF701
:105E300049FF204610BD10B51BF094FB98491BF09C
:105E4000D9FB98491BF0D6FBBDE8104096491BF0E2
:105E50003FBA10B51BF086FB94491BF0CBFB914970
:105E60001BF0C8FB90491BF033FABDE81040904985
:105E70001BF096BC2DE9FC410746884616461D4698
:105E8000FFF77EFF0446200005D196B1012E0AD00F
:105E9000022E02D0802494B120E042F21640FFF797
:105EA00064FF0446F7E742F20B40FFF75EFF04464B
:105EB000F1E74FF41050FFF758FF0446EBE74FF4BB
:105EC0007A7606E0FFF748FF04462CB1304603F02F
:105ED00009FD6D1EEDB2F5D205B9042464B90022A6
:105EE000114601A8FFF715FF05460022012168466B
:105EF000FFF70FFF40EA0504FFF7E4FE54B9BDF8D1
:105F00000400FFF7A6FF3860BDF80000FFF793FF1D
:105F1000C8F800002046BDE8FC812DE9FC4106469A
:105F20000F4615469846FFF72BFF04462CB995B14E
:105F3000012D0AD0022D02D0802494B114E042F643
:105F40001040FFF712FF0446F7E742F60D40FFF757
:105F50000CFF0446F1E742F60640FFF706FF044651
:105F6000EBE7FFF7F9FE04462CB94246002101A8F1
:105F7000FFF7CFFE04462CB9002201216846FFF747
:105F8000C8FE0446FFF79EFE4CB9BDF80400FFF7BB
:105F900060FF3060BDF80000FFF74DFF386020461D
:105FA000B9E730B4029C002B04D0012B05D080202F
:105FB00030BC7047234630BCAFE7234630BC59E7BE
:105FC00070B505460E46FFF7DBFE04462CB97DB3DF
:105FD000012D2ED0022D04D08024FFF773FE204621
:105FE00070BD052E22D2DFE806F003090F151B0055
:105FF00042F22F00FFF7B9FE0446EEE742F22D1001
:10600000FFF7B3FE0446E8E742F22B20FFF7ADFEB0
:106010000446E2E742F22930FFF7A7FE0446DCE738
:1060200042F22A70FFF7A1FE0446D6E78024D4E7A7
:1060300026E0052E22D2DFE806F003090F151B002B
:1060400042F22400FFF791FE0446C6E742F2261012
:10605000FFF78BFE0446C0E742F22020FFF785FEE3
:106060000446BAE742F22230FFF77FFE0446B4E767
:1060700042F22170FFF779FE0446AEE78024ACE7D8
:10608000052E2FD2DFE806F003161C22280042F26C
:106090003200FFF76AFE04469FE70000AE020020D0
:1060A0000000C8420000204100FF7F4700002F434E
:1060B0000000E14342F23010FFF757FE04468CE740
:1060C00042F23620FFF751FE044686E742F23430B2
:1060D000FFF74BFE044680E742F23770FFF745FEBC
:1060E00004467AE7802478E77CB505460E46FFF73C
:1060F00047FE044624B94FF46040FFF736FE0446DD
:1061000014B9FFF729FE04462CB90022114601A854
:10611000FFF7FFFD04462CB9002201216846FFF776
:10612000F8FD04464CB9BDF80400FFF792FE286064
:10613000BDF80000FFF77FFE3060FFF7C3FD20468B
:106140007CBD10B5FFF71CFE044624B943F26D0078
:10615000FFF70BFE0446FFF7B5FD204610BD10B556
:10616000FFF70EFE044624B943F26600FFF7FDFD7B
:106170000446FFF7A7FD204610BD70B5FFF700FEEF
:10618000054643F2A200FFF7F0FD40EA0504FFF7E1
:1061900099FD1CB94CF2503003F0A4FB204670BDB1
:1061A00010B5244C4FF080502060234803F09AFB38
:1061B000A0142060BDE810404CF2503003F092BBB8
:1061C00038B5010A8DF800108DF8010002216846EB
:1061D000FFF77AFD04469DF80000FFF7DBFC18B9D5
:1061E0009DF80100FFF7D6FC002802D12046FFF7FA
:1061F000D1FC38BD10B511491AF0FCFF10491BF055
:1062000067F810491BF0F6F91BF074F980B210BD65
:1062100010B50D491BF05CF80A491BF0EBF91BF0B7
:1062200069F980B210BD034808380068C0F38020C7
:1062300070470000100C0140A086010000003442AD
:1062400000002F4300FF7F470000C842F0B503461F
:106250000025084600260A2A01D00670F0BD002B52
:106260001DD005DA4FF02D0200F8012BC3F1000319
:1062700042F210724FF00A0793FBF2F454EA050C55
:1062800006D004F1300500F8015B04FB1233012550
:1062900092FBF7F2002AEFDC06700846F0BD3022D0
:1062A000027046700846F0BD0FB430B585B00546A3
:1062B0000AA800900EE05C2914D025292CD0521C8D
:1062C00028460992FAF7DAFE80212846FAF743FFBA
:1062D0000028F9D0099A11780029ECD105B030BC1A
:1062E0005DF814FB521C099210786E280CD07228AD
:1062F00002D0521C0992E7E70D212846FAF7BEFEAC
:106300000998401C0990DFE70A212846FAF7B6FEF3
:106310000998401C0990D7E7521C0992107864280C
:1063200019D0732802D0521C0992CDE7009810C8EA
:10633000009009E02846FAF7A1FE80212846FAF7E6
:106340000AFF0028F9D0641C21780029F2D10998AD
:10635000401C0990B8E7009808C800900A2201A9DB
:106360001846FFF773FF01AC09E02846FAF786FEEE
:1063700080212846FAF7EFFE0028F9D0641C217826
:106380000029F2D10998401C09909DE708B54FF407
:10639000A060F2F7C1F934208DF8000000208DF8DC
:1063A00001008DF8020001208DF803006846F2F725
:1063B000B8F908BD10B586B00121C804F9F73AFE56
:1063C00001211020F9F72BFE4FF48060ADF8140086
:1063D00018208DF8170003208DF81600FD4C05A934
:1063E0002046F2F716FDE114ADF8141004218DF8E3
:1063F000171005A92046F2F70CFD4FF4E13001908B
:106400000020ADF80800ADF80A00ADF80C00ADF8BA
:1064100010000C20ADF80E00EF4C01A92046FAF751
:1064200051FD012240F225512046FAF7D2FD01220A
:1064300040F224412046FAF7CCFDFFF7A7FF0121E7
:106440002046FAF7BAFD06B010BD08B510208DF849
:10645000030003208DF8020001212020F9F7DFFD61
:106460000420ADF800006946DC48F2F7D2FC08BD14
:1064700010B5FFF7EAFFFFF79DFF01F0E5FCBDE86F
:1064800010400421D548F2F733BD10B5D34C042198
:106490002046F2F72FFD4FF4FA7003F043FA20463E
:1064A000BDE810400421F2F723BD2DE9F047064670
:1064B0000D4691461F46DFF82883B8F800046FF3B5
:1064C0000E00A8F800040024DFF80CA30BE0315DF7
:1064D0005046FAF7D3FD80215046FAF73CFE0028DB
:1064E000F9D0641CA4B2BC42F1D3B8F800046FF335
:1064F0000E00A8F8000498F8010420F0800088F845
:106500000104002404E0322003F00CFAF9F74FFCF8
:1065100098F80104000604D42046641CA4B20A289A
:10652000F1D3B8F800140020C1F30E0108F80100FF
:1065300085B1B9F1000F0DD02946A94817F0C4FF65
:1065400028B94946A64817F0BFFF002800D001200F
:10655000BDE8F0873DB12946A14817F0B5FF0028F6
:10656000F6D00120F4E749469D4817F0ADFF00281A
:10657000EED00120ECE72DE9F0410D4690461E4695
:10658000024698A19448FFF78FFE55EA080012D002
:10659000934FB7F800046FF30E00A7F8000497F8C4
:1065A000010420F0800087F8010400243220B6FBAB
:1065B000F0F086B207E00120BDE8F081322003F060
:1065C000B1F9F9F7F4FB97F80104000604D420466A
:1065D000641CA4B2B042F1D3B7F800140020C1F398
:1065E0000E0178547DB1B8F1000F0CD029467C48DB
:1065F00017F06AFF28B94146794817F065FF00286F
:10660000DAD00120D8E73DB12946754817F05CFF84
:106610000028D1D00120CFE74146714817F054FF40
:106620000028C9D00120C7E770B5002404216B48B9
:10663000F2F75EFC4FF47A7003F074F94FF4FA75D8
:106640000CE02B46002269A169A0FFF794FF08B176
:10665000022070BDFFF719FF641CE4B20A2CF0D3CE
:1066600001D0012070BD002070BD40F6C413002889
:1066700005D0012807D0022809D0002070475DA26C
:106680005AA15FA077E75BA258A160A073E759A267
:1066900056A161A06FE700B59FB00B46024661A10D
:1066A00001A8F2F799FC41F2883300224FA101A81A
:1066B000FFF761FF1FB000BD00B59FB00B4602465B
:1066C0005DA101A8F2F788FC41F28833002247A1BE
:1066D00001A8FFF750FFEDE72DE9F041CEB06421AE
:1066E00035A817F0E7FF0024594D13AE281906EB23
:1066F000840190F86A000A22FFF7A8FD641CE4B246
:10670000042CF3D300240FAF281907EB840190F871
:106710006E000A22FFF79AFD641CE4B2042CF3D346
:1067200000240DF12C08281908EB840190F8720060
:106730000A22FFF78BFD641CE4B2042CF3D312A8E9
:1067400011A9CDE9081010AACDE906720EA80DA96D
:10675000CDE9041016A815A90CAACDE90010CDE9C1
:106760000282331D13AA3BA135A8F2F735FC35AAE6
:1067700043A117A8F2F730FC4FF47A6300221BA163
:1067800017A8FFF7F8FE4EB016E700B59FB00B460E
:10679000009202463FA101A8F2F71EFC4FF47A7363
:1067A000002212A101A8FFF7E6FE83E700B585B03D
:1067B000002801D0012200E000223CA16846F2F747
:1067C0000BFC4FF4FA73002208A16846FFF7D3FED2
:1067D00005B000BD00100140004C00400014014015
:1067E0007812002025730D0A000000004F4B0000B6
:1067F000415400006E6F206368616E6765000000A1
:1068000041542B43574D4F44453D310041542B4398
:10681000574D4F44453D320041542B43574D4F4453
:10682000453D330041542B43574A41503D22257387
:10683000222C22257322000041542B43574A4150F9
:106840005F4445463D222573222C222573220000F9
:10685000AB2200202225732E25732E25732E25733F
:10686000222C2225732E25732E25732E2573222C80
:106870002225732E25732E25732E257322000000EA
:1068800041542B4349505354415F4445463D257381
:106890000000000041542B43575341503D222573C3
:1068A000222C222573222C312C25640041542B43A9
:1068B00049504D55583D256400000000F0B5B9B071
:1068C00004460F4615461E46642120A817F0F2FE26
:1068D00014B1012C0FD107E03B46F9A2F9A120A881
:1068E0000095F2F779FB06E03B46FAA2F5A120A855
:1068F0000095F2F771FB052E06D220AB3246F6A1C9
:1069000002A8F2F769FB04E020AAF8A102A8F2F7B6
:1069100063FB4FF47A63F9A2AFF2301102A8FFF7DC
:106920002AFE39B0F0BD2DE9F041BAB08046409F53
:106930000E4615461C46642121A817F0BBFECDE982
:1069400000654346E3A2F1A121A80294F2F744FBBB
:10695000052F06D221AB3A46DFA103A8F2F73CFB94
:1069600004E021AAE1A103A8F2F736FB4FF47A6311
:10697000E2A2AFF2881103A8FFF7FDFD3AB01BE6D3
:1069800010B59EB04FF4FA7400280ED00B460122C9
:10699000E3A16846F2F720FB23460022AFF2B411D0
:1069A0006846FFF7E8FD1EB010BD0B460022DCA1D3
:1069B0006846F2F711FB23460022AFF2D011684679
:1069C000FFF7D9FDEFE710B54FF4FA730022AFF2ED
:1069D000E411D8A0FFF7CFFDD8B1DAA1DC4817F059
:1069E00073FD08B1022010BDDAA1D94817F06CFD83
:1069F00008B1032010BDDAA1D54817F065FD08B134
:106A0000042010BDD9A1D24817F05EFD08B10520C1
:106A100010BD062010BD10B500244FF4FA730022FB
:106A2000AFF23821C3A0FFF7A6FD00282DD0D2A1D8
:106A3000C74817F049FD00B10124D3A1C44817F09D
:106A400043FD10B144F0020401E024F00204D2A19D
:106A5000BF4817F039FD10B144F0040401E024F000
:106A60000404D1A1BA4817F02FFD10B144F0080476
:106A700001E024F00804D0A1B54817F025FD10B1BD
:106A800044F0100401E024F01004204610BD2DE96C
:106A9000FC410646C8230022AFF2B021CAA0FFF78E
:106AA0006AFD00250024CCA1A94817F00DFD18B1FE
:106AB0000B3000226F4602E00020BDE8FC81815CC3
:106AC0003A2902D0052D0DD00EE0022C06D19DF8FA
:106AD00001109DF8003001EB031171556D1CEDB2F2
:106AE000002413E0222915D0A1F13003092B04D88A
:106AF0002146641CE4B27B5408E0A1F16103052B3C
:106B000004D857392346641CE4B2F954521CD2B25B
:106B1000282AD4D3022C06D19DF801009DF800103C
:106B200000EB01107055B049C88A401CC882012092
:106B3000C3E710B592B041790279C3788478CDE982
:106B40000221CDE9004343780278A8A105A8F2F715
:106B500043FA4FF47A730022AFF2703105A8FFF7C1
:106B60000AFD12B010BDF8B54FF4FA730022AFF26F
:106B70008431A8A0FFF7FFFC0024AAA1744817F0F5
:106B8000A3FC18B10C300021A94D08E0A9A1704860
:106B900017F09AFC08B10220F8BD0020F8BD425C55
:106BA000222A0CD023462B44641CE4B29A72491C5E
:106BB000C9B23C29F3D328B11530002104E00844C0
:106BC000401CF8E70020F8BD425C2C2A1CD0491C70
:106BD000C9B20529F8D3002100226C46835C63B159
:106BE0002D2B14D0303B092B03D80E46491CC9B2BB
:106BF000A355521CD2B2052AF0D3012909D002298B
:106C00000BD0032913D020E00844401CE3E7002107
:106C1000EFE79DF80000287217E09DF800009DF84E
:106C2000011000EB800001EB400028720DE09DF8A0
:106C30000010642041439DF8010000EB800001EB4F
:106C400040009DF80210084428720120F8BD2DE98B
:106C5000FE4380460E4617464FF4FA794B46002213
:106C6000AFF2784175A0FFF786FC0025002476A1DD
:106C7000374817F029FC10B1C21D002006E10020A2
:106C8000BDE8FE83115C2E2902D0032D15D0F3E060
:106C9000012C04D0022C06D0032C0FD0E6E09DF886
:106CA00008107155E2E09DF808109DF8093001EBDD
:106CB000810103EB41017155D8E0DBE0C8E0000041
:106CC00054435000222573222C222573222C257335
:106CD000000000005544500041542B434950535488
:106CE0004152543D25642C257300000041542B4330
:106CF000495053544152543D25730000414C524574
:106D0000415920434F4E4E454354000022257322E3
:106D10002C222573222C25642C25642C256400004C
:106D200041542B4349505345525645523D25642CFE
:106D30002573000041542B4349505354415455533B
:106D4000000000005354415455533A320D0A0000DC
:106D5000781200205354415455533A330D0A000021
:106D60005354415455533A340D0A0000535441547E
:106D700055533A350D0A00002B43495053544154A2
:106D800055533A302C0000002B4349505354415482
:106D900055533A312C0000002B4349505354415471
:106DA00055533A322C0000002B4349505354415460
:106DB00055533A332C0000002B434950535441544F
:106DC00055533A342C00000041542B43495053543E
:106DD000414D41433F0000002B4349505354414D26
:106DE00041433A22000000006088002041542B43B8
:106DF00049505354414D41435F4445463D22257817
:106E00003A25783A25783A25783A25783A2578222D
:106E10000000000041542B43574A41505F435552F4
:106E20003F0000002B43574A41505F4355523A0000
:106E3000AB220020627573790000000041542B439F
:106E4000494653520000000053544149502C22003F
:106E50009DF8083064214B439DF8091001EB810136
:106E600003EB41019DF80A30194471556D1CEDB2D8
:106E7000002409E022290CD0303923460DF1080CFA
:106E8000641CE4B20CF80310401CC0B2B842FFF41A
:106E9000F9AE012C04D0022C06D0032C0ED01BE03E
:106EA0009DF80800705517E09DF808009DF809103E
:106EB00000EB800001EB400070550DE09DF80810DC
:106EC000642041439DF8090000EB800001EB400085
:106ED0009DF80A10084470554B460022AFF2F46149
:106EE000AFF21C10FFF747FB00250024AFF218118A
:106EF000FE4817F0E9FA20B100F10B0300206E46BE
:106F00002BE00020BCE6195C3A2902D0052D0ED0FA
:106F10000FE0022C07D19DF801109DF8002001EB35
:106F2000021108F805106D1CEDB2002413E02229AF
:106F300015D0A1F13002092A04D82146641CE4B21C
:106F4000725408E0A1F16102052A04D8573922469B
:106F5000641CE4B2B154401CC0B2B842D3D3022C7A
:106F600007D19DF801009DF8001000EB011008F812
:106F70000500FFF7F8FD012082E62DE9FF470746EF
:106F80004FF47A730022AFF29C71D9A0FFF7F3FAA5
:106F900000250024A0468DF80E808DF80D808DF818
:106FA0000C80D7A1D14817F08FFA20B1431D0020E3
:106FB00002AA03AE03E0002004B0BDE8F087195C2C
:106FC0002E2907D0032D01D3222934D0022C28D911
:106FD0000020F1E7012C04D0022C06D0032C0ED0A7
:106FE0001BE09DF80C10515517E09DF80C109DF812
:106FF0000D4001EB810104EB410151550DE09DF87D
:107000000C4064214C439DF80D1001EB810104EB11
:1070100041019DF80E40214451556D1CEDB20024F4
:1070200005E03039A446641CE4B206F80C10401C9C
:10703000C0B22828C3D3012C04D0022C06D0032CC4
:107040000ED01BE09DF80C00505517E09DF80C0089
:107050009DF80D1000EB800001EB400050550DE055
:107060009DF80C10642041439DF80D0000EB80005A
:1070700001EB40009DF80E1008445055DFF888924F
:10708000E7B19DF8080099F86A10884211D19DF87F
:10709000090099F86B1088420BD19DF80A0099F805
:1070A0006C10884205D19DF80B0099F86D1088424C
:1070B00007D00298C9F86A0002207DE70298C9F853
:1070C0006A00002500248DF80E808DF80D808DF863
:1070D0000C808EA1854817F0F7F920B100F10A0362
:1070E000002001AA01E0002066E7195C2E2907D0E4
:1070F000032D01D3222934D0022C28D900205BE7AC
:10710000012C04D0022C06D0032C0ED01BE09DF8DD
:107110000C10515517E09DF80C109DF80D4001EB37
:10712000810104EB410151550DE09DF80C406421B3
:107130004C439DF80D1001EB810104EB41019DF8DA
:107140000E40214451556D1CEDB2002405E030394C
:10715000A446641CE4B206F80C10401CC0B22828F7
:10716000C3D3012C04D0022C06D0032C0ED01BE07C
:107170009DF80C00505517E09DF80C009DF80D107F
:1071800000EB800001EB400050550DE09DF80C1025
:10719000642041439DF80D0000EB800001EB4000AE
:1071A0009DF80E1008445055E7B19DF8040099F879
:1071B0007210884211D19DF8050099F87310884229
:1071C0000BD19DF8060099F87410884205D19DF8FE
:1071D000070099F87510884207D00198C9F8720025
:1071E0000220E9E60198C9F87200002500248DF814
:1071F0000E808DF80D808DF80C8047A13B4817F06C
:1072000063F920B100F10A0300206A4601E0002082
:10721000D2E6195C2E2907D0032D01D3222934D0C0
:10722000022C28D90020C7E6012C04D0022C06D05D
:10723000032C0ED01BE09DF80C10515517E09DF863
:107240000C109DF80D4001EB810104EB41015155FB
:107250000DE09DF80C4064214C439DF80D1001EBAE
:10726000810104EB41019DF80E40214451556D1CF4
:10727000EDB2002405E03039A446641CE4B206F8FF
:107280000C10401CC0B22828C3D3012C04D0022CFF
:1072900006D0032C0ED01BE09DF80C00505517E0D3
:1072A0009DF80C009DF80D1000EB800001EB4000F4
:1072B00050550DE09DF80C10642041439DF80D00E1
:1072C00000EB800001EB40009DF80E100844505583
:1072D00047B39DF8000099F86E1088422FD19DF8B1
:1072E000010099F86F10884229D11CE07812002023
:1072F00041542B4349505354415F4355523F000082
:107300003A69703A22000000AB2200203A676174AB
:10731000657761793A2200003A6E65746D61736B2E
:107320003A22000010E09DF8020099F8701088429F
:1073300005D19DF8030099F87110884207D0009894
:10734000C9F86E00022037E60098C9F86E000120E7
:1073500032E610B54FF4FA7423460022AFF67431CA
:10736000CEA0FFF708F940B12346D0A2AFF6843192
:10737000BDE81040CEA0FFF7FEB8002010BD10B54C
:107380004FF47A7002F0CEFACCA1CD48FEF78CFF14
:10739000BDE810404FF4FA7002F0C4BA70B514465C
:1073A000ADF5167D0E461A46002540F226218C4288
:1073B00003D900200DF5167D70BD38B13246AFF20D
:1073C000C861BF48FEF770FF012520E0052A05D2FD
:1073D0002346BCA16846F1F7FFFD04E02246BEA1AA
:1073E0006846F1F7F9FD684617F0A4F881B211B1CB
:1073F000B1F5077F01D90020DCE7684600F06FFD9A
:10740000022002F08FFAA1B2304600F068FD284653
:10741000D0E700B59FB0642106A817F04BF906AA83
:10742000B1A101A8F1F7D8FD4FF47A630022AFF6BD
:10743000444101A8FFF79FF81FB000BD2DE9F047B8
:1074400081460027DFF8B482B8F800046FF30E001D
:10745000A8F8000498F8010420F0800088F80104DE
:1074600040F20241404617F003F900240026A44DE3
:107470003DE0022002F056FA2978182904D0192993
:1074800013D0162918D030E0FFF726F968B39D48CD
:107490009D4902780A7042784A7082788A70C07872
:1074A000C870FEF7F2FF2E701FE0FFF7B2FFE0B1E9
:1074B000FEF7EBFF2E7018E04FF4FA730022AFF6E0
:1074C000D44192A0FFF757F800B12E708E484021AA
:1074D000603817F0CDF88C482021203817F0C8F814
:1074E0008D490120487109F0F5FDF8F760FC98F826
:1074F0000104000604D42046641CA4B26428B8D356
:10750000B8F80004C0F30E0008F80060B9F1000FED
:1075100001D07A4F05E081A1784816F0D5FF00B17F
:10752000764F384649E570B5027A2C2A01D0002002
:1075300070BD827A3A2A10D1437A303B092B0CD89D
:107540009BB2002205E08418E47A01F8014B521C3A
:1075500092B29A42F7D3184670BDC37A6FF02F05E6
:107560003A2B03D0047B3A2C1AD03EE0437A303BCE
:10757000092B3AD8302A38D3392A36D803EB83037B
:1075800005EB43031A4493B2002205E08418247BE0
:1075900001F8014B521C92B29A42F7D3184670BDC3
:1075A000447A303C092C20D8302A1ED3392A1CD8E2
:1075B000302B1AD3392B18D804EBC406303A06EB1B
:1075C000041402EB820203EB840305EB42021A442B
:1075D00093B2002205E08418647B01F8014B521C31
:1075E00092B29A42F7D3184670BD002070BD10B514
:1075F000044640214B4817F03BF84A4914B1012C8E
:1076000003D004E06520088001E0672008801D2089
:107610004880454802788A804278CA8082780A8108
:10762000C2784A8109228A818379CB81364A1478CB
:107630000C8254784C8294788C82D478CC8232F844
:10764000684C0C8370244C83007A88833748006828
:10765000C0F3072444EA00244C8481F82430030C4E
:107660001B0243EA1060A1F83900002081F83B00BA
:1076700032F8662C8A8781F83E0081F83F002C4959
:107680000120087010BD0B0A037041700021817049
:10769000C170110A017142717047000041542B43BF
:1076A00049504D4F44453D31000000003E00000070
:1076B00041542B43495053454E4400002B2B2B0083
:1076C000004C004041542B43495053454E443D2506
:1076D000642C25640D0A000041542B434950534546
:1076E0004E443D25640D0A0041542B435744484302
:1076F000505F4445463D312C310000007812002097
:107700001F030020F28400201523002041542B5237
:107710004553544F52450000810400202B495044EA
:10772000000000007A160020947F00200C0000204A
:10773000B302002070B50024FD4D4FF4FA76FFF738
:1077400042F9A871401E032808D3304602F0EAF837
:10775000F8F72DFB641CE4B20A2CF0D3A8790328B7
:1077600007D13346BDE870400022F2A1F2A0FEF737
:1077700002BF70BD70B500244FF47A7504E0F8F7CD
:1077800016FB642002F0CEF82B460022E9A1EEA001
:10779000FEF7F1FE002804D12046641CE4B2142850
:1077A000EDD370BD10B5002404E0F8F700FB6420B1
:1077B00002F0B8F864230022DEA1E6A0FEF7DBFEAB
:1077C000002804D12046641CE4B21428EDD310BD77
:1077D00010B5002404E0F8F7EAFA642002F0A2F8F9
:1077E00064230022D3A1DFA0FEF7C5FE002804D148
:1077F0002046641CE4B21428EDD310BD2DE9F041FD
:10780000DC4D00242C71CA4EB07901284CD0307860
:1078100050B12C704FF4FA730022C6A1D1A0FEF72C
:10782000AAFEC82002F07EF83078012839D170789D
:107830004FF47A7701280ED1FEF74EFF384602F05A
:1078400071F83B46CCA2BBA1CDA0FEF794FEC820A8
:1078500002F068F82C710020FEF707FFC82002F044
:1078600061F8B3494A31A1F14000FEF714FF00244A
:107870004FF480663D460FE00020FFF7DFFD014634
:107880003246C14816F075FEAAA1C04816F01CFE8B
:1078900038B9284602F046F82046641CE4B20528B0
:1078A000EAD3BDE8F04145E7BDE8F08110B5B14C41
:1078B0006079012805D1FFF7A1FFF1F7C9FB00208E
:1078C000607110BD8EB014200990AA4C002525705F
:1078D0006571974F0420F87178884FF6FF7800287B
:1078E00001D0404502D14FF4FB7078809048B97ABE
:1078F0000A300D90FF2906D1F87AFF2803D14021E4
:107900000D9816F0B5FE8A4897F84A104A300C9048
:10791000FF2907D197F84B00FF2803D120210C98AD
:1079200016F0A6FE6571B88808B1404502D14BF645
:10793000C020B8807E480A2207A94088FEF786FC4E
:10794000FEF796FD4FF4FA67384601F0EBFFFEF7BD
:107950009CFD384601F0E6FFFEF766FE814674485E
:10796000012776300B90B9F1020F02D0763887717B
:1079700055E040F26550FAF796F88DF81400442867
:1079800042D018208DF81500FE208DF81600804A90
:10799000107828B9517819B9917809B9D17891B38B
:1079A000FF2808D15178FF2905D19178FF2902D10C
:1079B000D178FF292BD0D178102903D210318DF83E
:1079C000171001E08DF817109178102903D21031AB
:1079D0008DF8181001E08DF818105178102903D295
:1079E00010318DF8191001E08DF81910102803D20C
:1079F00010308DF81A0001E08DF81A000DF1150015
:107A0000FFF797F8A77002E00B98FFF740F8484897
:107A1000052181710020FEF728FEFFF7EFFEDFF859
:107A200068A1052001F07EFFF8F7C1F9B9F1020F56
:107A30000BD1A078012808D10B98FFF728F8A57082
:107A4000442140F26550F9F7AAFFB9F1020FE8D1DD
:107A5000DFF8DC8098F80600022855D0012853D0C2
:107A60004C49088D401C088598F8010038B988F801
:107A70006A5088F86B5088F86C5088F86D50207800
:107A800040B94FF4FA7300222AA132A0FEF773FD29
:107A900000B12770207898B34FF0000BFEF793FFEA
:107AA00088F80600642001F03DFFF8F780F998F8A7
:107AB0000600032806D958460BF1010B1FFA8BFB71
:107AC000C828EBD3BBF1C80F02D3FFF797FEA8E796
:107AD00088F8005040210D9816F0CAFD20210C981E
:107AE00016F0C6FD2C48477109F0F4FA4FF4FA730A
:107AF000002210A11BA0FEF73EFD642001F012FF42
:107B0000C82001F00FFF8CE7207980B14FF4806B23
:107B10005946224816F0ACFD59461B4816F0A8FD00
:107B20000020FFF78BFC01465A46174838E04FE02B
:107B3000AB2200204F4B000041542B434950434C93
:107B40004F53453D3500000041542B524553544F8F
:107B50005245000041542B43575354415254534D06
:107B60004152540041542B435753544F50534D41AD
:107B700052540000B0020020726561647900000078
:107B800041542B5253540000C31600207812002099
:107B9000947F00206088002081040020AB1E00201C
:107BA00016F0E7FC9AF80700303800F0FF0BD249D6
:107BB000A1F5FD60FFF7B7FC0246100077D0ABF1EE
:107BC0000200022874D8CC490878EE2872D080E0F0
:107BD0002822CA490B98FFF73AF860B198F86A0072
:107BE00040B998F86B0028B998F86C0010B998F86B
:107BF0006D00E0B127710020FFF7BFF94FF4FA7B69
:107C00005B460022AFF2D401BDA0FEF7B4FC012018
:107C1000FEF7CCFDF8F7CBF85B460022AFF2EC01A3
:107C2000AFF2EC00FEF7A7FC4FF0000B03E025716C
:107C3000E1E7F8F7BCF80095B8F8041002230A460B
:107C4000B3A0FEF770FE30B958460BF1010B1FFAD6
:107C50008BFB0528EDD34FF0000840F2D24B01E03A
:107C6000F8F7A5F8594602230A46A9A00097FEF79F
:107C70005AFE30B9404608F101081FFA88F8052875
:107C8000EED34FF0000801E0F8F791F809AA07A930
:107C90000120FEF775FE00287FF419AF404608F179
:107CA00001081FFA88F80528BFF411AFECE733E0AC
:107CB00033E0FFE7487810280BD1887848B9C878B6
:107CC00038B9087928B9487918B9887908B9C879CC
:107CD00038B1934A8879927990420CD0FF2807D026
:107CE0008EE07F210B20F9F7DFFEF1F7B1F987E095
:107CF000C879192810D08049052007F091FE228903
:107D000042B19AF8070087493038C3B20020FFF724
:107D100045FB2581FFF7CAFD72E0BBF1000F03D0E0
:107D2000BBF1010F1CD06BE00023734902A8009740
:107D30000DF033F80246501EB0F5FF7F60D80123E6
:107D40006D4902A80EF07BFFE288EAB39AF80700BB
:107D500075493038C3B20020FFF720FBE5804FE0C3
:107D60006549087864284BD1E770002098F86A309C
:107D700098F86BC098F86CB098F86D10C2F3850E47
:107D80000A9112E05C4901EB80014A789A420AD1DB
:107D90008A78624507D1CA785A4504D10A790A9986
:107DA0008A4200D1E570401CC0B27045EAD3E07849
:107DB00050B10020FFF71BFC5C498D77CD7781F82F
:107DC000205081F8215000E01AE00020544A01EBD5
:107DD000000C131893F848338CF82530401CC0B2BF
:107DE0001428F4D311F83E0F40F0020008709AF8FE
:107DF000070040223038C3B24C490020FFF7CEFACA
:107E00006420B6FBF0F100FB116068B9FEF7ABFE31
:107E100020B165706078032804D005E06078401CCC
:107E20006070F7E788F806703046761CB6B2B0F599
:107E3000967F7FF64CAE00260120FFF79EF80228C1
:107E40007FF445AE2571ECE510B58CB00121022020
:107E5000F8F7DAF8364C2046F0F77EFE4FF416704D
:107E600004901020039000210B91244A12320292B8
:107E7000089180220692202009902E4801900791B7
:107E8000059180140A9001A92046F0F7DCFE0CB0A1
:107E900010BD70B50446274D01222D1F80212846B4
:107EA000F9F7B2F82146224C2046F0F70DFF0121E8
:107EB0002046F0F7F2FE204E3046F0F70AFF002889
:107EC000FAD03046F0F714FF00212046F0F7E5FE27
:107ED0002846BDE8704000228021F9F795B810B51A
:107EE0000C46014605482246123016F042FB204659
:107EF000FFF7CFFF10BD0000AB1E002015230020B0
:107F000041542B4349504D4F44453D300000000043
:107F10003235352E3235352E3235352E3235350067
:107F2000947F0020B71C0020C31A00207A1600207E
:107F300058040240044C00400000021008B5002123
:107F400042F2B112684600F03EFB024669466220EA
:107F500000F0FBFB00B2002804D14FF47A7000F06F
:107F600074FE002008BDFEB506460D4614460021ED
:107F70004EF60542684600F026FB0246694662203E
:107F800000F0E3FB00B2002815D10622694662200A
:107F900000F0A1FB00B200280DD1684600F024FDDE
:107FA00030806E46B01C00F01FFD2880301D00F0B0
:107FB0001BFD20800020FEBD7CB50C4615466A46A0
:107FC00001A9FFF7D0FF002810D1BDF8040045F249
:107FD0007351FF4A484302EB50302060BDF8000067
:107FE00043F2D4014843400B286000207CBD08B513
:107FF000002143F68672684600F0E5FA02466946BB
:10800000622000F0A2FB00B2002803D1F14800F08A
:108010001CFE002008BD38B50446002142F218328B
:10802000684600F0D0FA02466946622000F08DFBF7
:1080300000B2002810D14FF47A7000F006FE022240
:108040006946622000F047FB00B2002804D1684670
:1080500000F0CAFC2080002038BD38B504466846D0
:10806000FFF7D9FF002807D1BDF8000045F2735192
:108070004843400B2060002038BD1CB50446002159
:1080800042F21D42684600F09EFA014622466846CA
:1080900000F0C7FA82B26946622000F056FB00B2D7
:1080A000002804D14FF47A7000F0CFFD00201CBDF1
:1080B00045F6DE714843000CDFE738B50446002181
:1080C00042F22232684600F07EFA02466946622099
:1080D00000F03BFB00B2002810D14FF47A7000F0A2
:1080E000B4FD02226946622000F0F5FA00B20028D1
:1080F00004D1684600F078FC2080002038BD1CB513
:108100000446002142F22742684600F05CFA01462C
:108110002246684600F085FA82B26946622000F085
:1081200014FB00B2002804D14FF47A7000F08DFDEA
:1081300000201CBD1CB5044600214FF46042684677
:1081400000F041FA01462246684600F06AFA82B21F
:108150006946622000F0F9FA00B2002804D14FF419
:108160007A7000F072FD00201CBD7CB505460C46FF
:10817000002143F22F62684600F025FA01462A46A4
:10818000684600F04EFA82B26946622000F0DDFADD
:1081900000B200280FD1904800F057FD0222694636
:1081A000622000F098FA00B2002804D1684600F07E
:1081B0001BFC208000207CBD38B50446002142F223
:1081C0001332684600F0FFF902466946622000F06B
:1081D000BCFA00B2002810D14FF47A7000F035FDDF
:1081E00002226946622000F076FA00B2002804D12B
:1081F000684600F0F9FB2080002038BD1CB504461D
:10820000002142F21642684600F0DDF9014622469E
:10821000684600F006FA82B26946622000F095FADC
:1082200000B2002804D14FF47A7000F00EFD002057
:108230001CBD08B5002142F2AC12684600F0C3F93B
:1082400002466946622000F080FA00B208BD38B5E7
:10825000044600214EF2B842684600F0B4F90246E6
:108260006946622000F071FA00B2002810D14FF484
:108270007A7000F0EAFC02226946622000F02BFAD4
:1082800000B2002804D1684600F0AEFB2080002038
:1082900038BD08B5002143F21562684600F093F935
:1082A00002466946622000F050FA00B2002803D16D
:1082B0004A4800F0CAFC002008BDFEB506460D463F
:1082C0001446002143F28262684600F07CF90246BF
:1082D0006946622000F039FA00B2002819D14FF443
:1082E0007A7000F0B2FC06226946622000F0F3F9D1
:1082F00000B200280DD1684600F076FB30806E4653
:10830000B01C00F071FB2880301D00F06DFB208058
:108310000020FEBD38B50446002143F239626846AC
:1083200000F051F902466946622000F00EFA00B2F0
:1083300000280FD12A4800F088FC022269466220FA
:1083400000F0C9F900B2002804D1684600F04CFBE7
:108350002080002038BD08B5002143F23262684613
:1083600000F031F902466946622000F0EEF900B2F1
:10837000002803D1194800F068FC002008BD08B5AA
:10838000002143F24662684600F01DF90246694644
:10839000622000F0DAF900B2002804D144F620602F
:1083A00000F053FC002008BD08B5002142F29D12E8
:1083B000684600F008F902466946622000F0C5F9F7
:1083C00000B2002803D1074800F03FFC002008BDA0
:1083D0003850FFFF20A10700801A060000350C006E
:1083E00080969800404B4C0008B5002142F296124E
:1083F000684600F0E8F802466946622000F0A5F9F8
:1084000000B20028E3D14CF2503000F01EFC0020F6
:10841000DDE708B5002143F2E062684600F0D3F8DA
:1084200002466946622000F090F900B20028CED1E1
:108430004FF47A7000F009FC0020C8E708B500216D
:1084400043F2F662684600F0BEF8024669466220D2
:1084500000F07BF944F6206000F0F7FB0020B6E75F
:108460003EB5FFF7EBFFFFF7C2FDFFF788FF2C4992
:10847000002008706A4601A902A8FFF71EFF294CD8
:10848000072500B92570FFF759FD002800D1257098
:108490003EBD3EB523480078072825D1204C224D0B
:1084A0002078012821D06A4601A902A8FFF784FD9F
:1084B000002819D1BDF80800002815D000996424BF
:1084C00091FBF4F18AB2019991FBF4F189B2F2F7D0
:1084D000F7FBBDF808002884019890FBF4F068844D
:1084E000009890FBF4F0A8843EBDE88B401CE88324
:1084F000FFF77DFD4FF47A75284601F013FA0C4A18
:108500000A491088FFF731FE284601F00BFAFFF701
:1085100015FD41F2883001F005FA002020703EBDC3
:10852000BA02002044020020608800203A030020A4
:108530003C03002070B50546FF200023312410E0E5
:10854000EA5C50400822060603D584EA4000C0B227
:1085500001E04006000E521ED2B2002AF3D15B1C8D
:108560009BB28B42ECD370BD10B51446FFF7E2FF0F
:10857000A04201D0012010BD002010BD2DE9F04126
:10858000054617469846080A28700220697000249C
:1085900015E037F814100A0A411C89B22A5417F85A
:1085A00014004A1C96B26854A819801E0221FFF7D5
:1085B000C1FF0146701C80B2A955641CE4B2444559
:1085C000E7D3BDE8F08110B5140A4B1C9BB24454AC
:1085D000591C89B2C254084610BD70B504461546F0
:1085E0002A0E481C80B262542A0C411C8EB22254BE
:1085F000A019801E0221FFF79DFFA055761CB1B285
:108600002A0A481C80B26254411C8EB22554A0191B
:10861000801E0221FFF78EFFA055761CB0B270BD00
:10862000DBE730B50446130A481C80B26354411C92
:108630008DB222546019801E0221FFF77BFF605526
:108640006D1CA8B230BD92B2EBE770B5044615467A
:108650002A0E481C80B262542A0C411C8EB222544D
:10866000A019801E0221FFF765FFA055761CB1B24C
:108670002A0A481C80B26254411C8EB22554A019AB
:10868000801E0221FFF756FFA055761CB0B270BDC8
:108690002DE9F04105460846174698465FEAC8713D
:1086A00001D004208DE7002412E03A5D411C89B21C
:1086B0002A5438194278481C86B26A54A819801E78
:1086C0000221FFF737FFA855761CB0B2A41CA4B254
:1086D0004445EAD375E72DE9F0410D46510801EB19
:1086E00041011FFA81F8D10701D0042069E7424611
:1086F000294600F04CF80028F8D10024002615E0A7
:108700002819074682780221FFF72EFF20B1094A77
:10871000D18D491CD18554E7295D701C80B2A955C3
:108720007A78411C8EB22A54E41CA4B24445E7D3A3
:10873000002046E76088002010B5F9F792F8F9F7B5
:1087400043F840B210BDF9F7ADB82DE9F041044649
:108750000E461746F9F70BF86006000EFFF7ECFF20
:108760000546280001D0BDE8F081002409E0305D15
:10877000FFF7E2FF054615B1F9F70FF803E0641CB7
:10878000A4B2BC42F3D3F9F708F82846EBE72DE989
:10879000F04104460D461646F8F7E9FF012000EBCC
:1087A0004400C0B2FFF7C8FF04461CB1F8F7F5FF5C
:1087B0002046D8E70024771E09E0BC4201DA0120F8
:1087C00000E00020FFF7BFFF2855641CA4B2B442AC
:1087D000F3D3F8F7E2FF0020C5E710B5814C07E0BE
:1087E00000F02FFA08B1002010BD0A2000F02DFA89
:1087F000641EF5D1601E10BD70B5064607244FF00B
:10880000FF3500F00AFA26FA04F0C00702D000F0A3
:10881000DBF901E000F0E9F9052000F016FA00F0BC
:10882000C7F9052000F011FAFFF7D7FF08B1284675
:1088300070BD641E64B2002CE3DA00F0EEF900F0C3
:10884000C3F9052000F001FA00F0B2F9052000F0AC
:10885000FCF9FFF7C2FF08B1284670BD00F0D9F956
:1088600008B1012400E0002400F0D7F9204670BDD3
:1088700070B50646002500F0A7F90724052000F092
:10888000E4F900F095F9FFF7A8FF08B1FF2070BDEB
:1088900000F0BFF908B1012100E00021A140294307
:1088A000CDB200F0BAF9641E64B2002CE6DA16B15B
:1088B00000F09BF901E000F087F9052000F0C5F910
:1088C00000F076F9052000F0C0F9FFF786FF08B147
:1088D000FF2070BD00F0A1F900F076F9284670BDC8
:1088E00010B500F065F9FFF778FF10B14FF0FF30D9
:1088F00010BD00F07AF9052000F0A7F900F08DF91D
:10890000052000F0A2F9002010BD10B500F06DF9AF
:10891000052000F09AF900F04BF9052000F095F9D8
:1089200000F052F9BDE81040052000F08EB92DE9A5
:10893000F04104460E461746FFF7D2FF002806D145
:108940006006000EFFF758FF0546280000D00AE732
:10895000002409E0305DFFF74FFF054615B1FFF732
:10896000D4FF03E0641CA4B2BC42F3D3FFF7CDFFF5
:108970002846F8E62DE9F04104460D461646FFF775
:10898000AFFF00280AD1012000EB4400C0B2FFF77E
:1089900033FF04461CB1FFF7B8FF2046E3E600248E
:1089A000771E09E0BC4201DA012000E00020FFF759
:1089B0005FFF2855641CA4B2B442F3D3FFF7A5FFB0
:1089C0000020D0E610B500F00AF900F0F1F8BDE89B
:1089D000104000F0F9B810B500F0EAF8BDE810401A
:1089E00000F0F2B8F04902004178007841EA002036
:1089F0007047C178027841EA0261427880781204B7
:108A000042EA002008437047F3E770B50546FF20AF
:108A10000023312410E0EA5C50400822060603D50A
:108A200084EA4000C0B201E04006000E521ED2B2FD
:108A3000002AF3D15B1C9BB28B42ECD370BD10B506
:108A40001446FFF7E2FFA04202D04FF0FF3010BD06
:108A5000002010BD08B506200090012269460020C4
:108A6000FFF765FF08BD2DE9F0410546174698461A
:108A7000080A287002206970002415E037F81410E5
:108A80000A0A411C89B22A5417F814004A1C96B2EB
:108A90006854A819801E0221FFF7B7FF0146701C19
:108AA00080B2A955641CE4B24445E7D3BDE8F08127
:108AB0002DE9F04391B00F4602EB42011FFA81F815
:108AC00001AE42463146FFF755FF002818D1002479
:108AD000002512E03019814682780221FFF7AFFFAE
:108AE00000280DD1315D681C80B2795599F80120BC
:108AF000411C8DB23A54E41CA4B24445EAD3002090
:108B000011B0BDE8F08370B50C4615462A462146E3
:108B1000FFF7CEFF00280DD109E004EB40035978A0
:108B20001A7841EA022124F81010401CC0B2A84271
:108B3000F3D3002070BD38B5044600231A466846BA
:108B4000FFF791FF022269462046FFF7F0FE38BD8D
:108B500010B588B00446DBB26846FFF784FF0246D2
:108B600069462046FFF7E3FE08B010BDF8B506469B
:108B7000069F14461D4600231A466846FFF773FFFA
:108B8000022269463046FFF7D2FE002808D114B110
:108B9000204600F05AF83A4629463046FFF7B3FF20
:108BA000F8BD08B5009313460022FFF7DFFF08BDAC
:108BB00008B50820ADF8000004208DF803006946D0
:108BC0002348F0F726F908BD08B50420ADF80000E9
:108BD0008DF8030069461E48F0F71BF908BD10B573
:108BE000FFF7F2FFBDE81040E2E738B50420ADF82A
:108BF000000010208DF8030003208DF80200144CB3
:108C000069462046F0F705F904212046F0F772F98D
:108C100038BD04210E48F0F757B938B50820ADF833
:108C2000000010208DF8030003208DF80200084C8E
:108C300069462046F0F7EDF808212046F0F75AF98A
:108C400038BD08210248F0F73FB900F04BBE0000E4
:108C50000008014070B50024F74D04EB840005EBDB
:108C6000800000F0F9FB641C052CF6D3F248643058
:108C700000F0F2FBF048783000F0EEFBEE488C306C
:108C800000F0EAFBEC48A03000F0E6FBEA48B43024
:108C900000F0E2FBE849E948643141631431816343
:108CA00070BD70B504461546102204F1340015F06D
:108CB00028FD002084F84300052D00D30425E5623B
:108CC000201D00F0D4FB04F1180000F0D0FB24615B
:108CD000C5F10500A061646270BD70B506460D4621
:108CE000442000F04FFC044644B1B60045B128468C
:108CF000206348B1A522314615F0B2FC204670BD74
:108D0000304600F03FFCF3E7204600F091FC0024E1
:108D1000F4E72DE9FF4F81B08246DDE90E68109936
:108D200017469B463846FFF7D8FF0446C34DECB3C1
:108D3000216B781E01EB800020F007090097324676
:108D40002046119B0299FFF7ACFF5A465146484610
:108D500000F0C8FB2060B8F1000F01D0C8F8004057
:108D600000F0EBFBA868401CA860286810B1A86957
:108D700038B10BE02C60A868012807D1FFF76AFF23
:108D800004E02868C06AB04200D82C60E06A296913
:108D9000884200D92861E96A491CE9626969884208
:108DA00000D9686100EB8001A34800E008E000EB17
:108DB0008100211D00F05EFB012400F0C6FB01E0F4
:108DC0004FF0FF34012C07D1A86928B12868C06A88
:108DD000B04201D200F0ABFB05B02046BDE8F08FF9
:108DE00070B5054600F0A9FB944E3068854200D16D
:108DF0000025FDB12C46201D00F062FBA06A18B1D1
:108E000004F1180000F05CFB8B48211DA03000F03D
:108E100031FB7068401C7060F06A401CF06200F02A
:108E200094FBB069002807D0002D05D1BDE8704043
:108E300000F07DBB3468DEE770BD70B57F4DE8693A
:108E4000002803D0286A401C286270BDE868401CD6
:108E5000E860E8684FF0FF3670B9686BA96B69632A
:108E6000A863A86A401CA862686B0068A0B1686B20
:108E7000C068C06840682863E868296B8842E4D30A
:108E8000686B006850B1686BC068C4686068E96866
:108E9000814205D2286370BD2E63EDE72E6370BD5D
:108EA000201D00F00DFBA06A18B104F1180000F0BD
:108EB00007FBE06A6969884200D968615E4900EB96
:108EC000800001EB8000211D00F0D4FAD8E72DE9E5
:108ED000F041002700F031FB584EF069401EF06170
:108EE000F069E8BBB068D8B30025DFF84C8108F121
:108EF0008C081CE0D8F80C00C46804F1180000F0DD
:108F0000DFFA201D00F0DCFAE06A7169884200D9BE
:108F10007061494900EB800001EB8000211D00F0E9
:108F2000A9FAE06A3168C96A884200D30125D8F8F5
:108F300000000028DED1306A28B908E0FFF77DFF85
:108F4000306A401E3062306A0028F7D10125012DB9
:108F500002D0706A012806D101270020706200E06B
:108F600001E000F0E4FA00F0F0FA3846BDE8F081E4
:108F700070B50446314D28684460E868844206D2E2
:108F80002968A86B091DBDE8704000F081BA296806
:108F9000686B091D00F07CFA286B844200D22C63B8
:108FA00070BD2648C169491CC161704770B5034650
:108FB0000C460022FFF7F5FF186804441F49CD68EE
:108FC000A84206D9A0420AD9C868844207D901221A
:108FD00005E0A04202D8C868844200D901221C6082
:108FE00032B10868001D00F06BFA2046FFF7C0FFA1
:108FF000FFF76DFF002803D1BDE8704000F097BA7D
:1090000070BD10B502460020002A0DD0FFF7C9FF41
:109010000A48C1688C180068001D00F051FA20460B
:10902000FFF7A6FFFFF753FF002803D1BDE810406C
:1090300000F07DBA10BD000080250020BC02002099
:1090400010B5044600F079FA0CB9F7480468E46AF0
:1090500000F07BFA2046EDE72DE9F04106460D468B
:109060000027052D00D3042500F067FADFF8B88348
:10907000D8F80000864200D1002646B13446E06AA6
:10908000A8422AD0854205D936B1012704E0D8F894
:109090000040F4E706B90127E562C5F10501A161C9
:1090A000E24D00EB8000616905EB8000814210D148
:1090B000201D00F005FAE06AD8F81410884201D9A2
:1090C000C8F8140000EB800005EB8000211D00F0C3
:1090D000D1F9012F01D100F02AFABDE8F04100F0EA
:1090E00034BAD149C869002802D0012048627047CB
:1090F000CE4A02E04869401E4861486900EB8000A2
:1091000052F820000028F5D0486900EB800002EBFF
:10911000800042685268426000F108039A4201D11F
:10912000526842604068C0680860704770B5054684
:1091300000F003FABC4E3068854200D10025C5B16D
:109140002C46201D00F0BCF9A06A18B104F11800EB
:1091500000F0B6F9B548211DB43000F08BF900F0ED
:10916000F4F9002D0FD1B06928B1BDE8704000F0CE
:10917000DEB93468E5E7AD48B4300068B1688842CC
:1091800002D10020306070BDBDE87040A9E7002129
:10919000A64B4269B4339A4206D1806AA3F12802F1
:1091A000904201D000B901210846704770B50446CD
:1091B000002C25D09C4D2868844221D000F0BDF9B8
:1091C0002046FFF7E4FF012816D1201D00F078F9B2
:1091D000E06A6969884200D96861944900EB8000BF
:1091E00001EB8000211D00F045F9E06A2968C96A99
:1091F000884201D300F09BF9BDE8704000F0A5B9AA
:1092000070BD70B5044600252046FFF7C0FF012859
:1092100008D1854EF06938B1844804F118018C30CA
:1092200000F028F9284670BDE06A3168C96A8842B2
:1092300001D3012500E00025201D00F041F9E06A7E
:109240007169884200D97061784900EB800001EBB8
:109250008000211D00F00EF9E4E710B50446206BF4
:1092600000F0E6F92046BDE8104000F0E1B970B525
:109270006D4D686800281FD0FFF793FE6B4EA03637
:109280003068B8B10024FFF722FE002C14D100F0A2
:1092900054F9F068C468201D00F012F9A868401E57
:1092A000A8606868401E686000F04FF92046BDE87D
:1092B0007040D2E70124E6E770BD5C4CFFF7D7FFB2
:1092C00020680128FAD900F032F9F7E71FB5002429
:1092D0000094019402942346642255A156480394B5
:1092E000FFF717FD012809D1EEF7EEFF4E480121E7
:1092F0008161C460BDE81F4000F005B91FBD10B515
:10930000EEF7E2FF484900208861BDE8104000F018
:109310000DB910B500F011F94348C46800F015F913
:10932000204687E610B5EEF7CFFF3F48C468EEF75A
:10933000D2FF20467EE63C488068704770B50D46F7
:10934000394C2168183100F0A3F82068001D00F0A6
:10935000B7F8681C04D0E0682844BDE8704007E610
:109360002168BDE870403148091DB43000F082B872
:1093700070B5C068C46804F11800064600F0A0F893
:10938000294DEA695AB1294831468C3000F072F80B
:10939000E06A2968C96A884212D3012070BD201D85
:1093A00000F08EF8E06A6969884200D968611F4957
:1093B00000EB800001EB8000211D00F05BF8E7E787
:1093C000002070BD18498A6A0260C9684160704710
:1093D00070B504460D4600F0B0F82868411C0AD06C
:1093E000114B21689A6A914207D06168DA6891420C
:1093F00003D8012410E000240EE06268D968891ABD
:10940000814208D2D968891A401A28602046FFF79D
:10941000D9FF002400E0012400F097F8204670BD39
:109420000149012048627047BC02002080250020CD
:1094300049444C4500000000BB9201080548816981
:10944000002903D0C06918B10220ECE70020EAE748
:109450000120E8E7BC02002000F1080141604FF064
:10946000FF328260C160016100210160704700210C
:1094700001617047426853684B6043688B60536872
:1094800099605160416008610168491C0160704742
:1094900010B50B685A1C02D000F1080202E0026904
:1094A00004E05268546824689C42FAD953684B60BF
:1094B00099608A60516008610168491C016010BDB3
:1094C000D0E901219160D0E90112516001694A6837
:1094D000824201D182684A60002202610868401E0F
:1094E0000860704720384FF08073C36181610021AC
:1094F000416140F8202970474FF0E0201E4941614A
:1095000007210161704710B51C48016841F47F01D3
:109510000160016841F07F410160FFF7EDFF1849EC
:1095200000200860EEF7A8FE002010BD7047134928
:109530004FF080501C390860704710B5EEF7C4FE3C
:109540000F480168491C016010BD0D490868401EA4
:109550000860002801D1EEF7BEBE704710B507497C
:109560004FF080501C390860EEF7AEFEFFF765FC47
:10957000BDE81040EEF7AFBE3F19010020ED00E05E
:10958000F80200202DE9F04104460025FFF709FD0F
:10959000384E06F10801706801F1080360B93648D9
:1095A0000860002048604FF4A0425A6018603248BA
:1095B00042600360012070603CB11034600704D049
:1095C00004F00700C0F108000444601E44F6FF7276
:1095D000904228D2274A0832096801E00A4601462B
:1095E0004868A04202D208680028F7D199421AD0F0
:1095F00015681035086810604868001B20280ED9CF
:109600000B1958604C605C681A48083000E010463E
:1096100002685768A742FAD302681A600360486874
:109620003168081A3060FFF752FC2846BDE8F08127
:1096300010B5002818D010380446FFF7B2FC606857
:109640000C49083100E011460A6853688342FAD396
:10965000086820600C600748616802681144016076
:10966000BDE81040FFF733BC10BD024800687047EA
:1096700070470000FC02002048260020704770B5AB
:109680000446874D40212846F7F765FD0028F9D0AC
:10969000A1B22846F7F7F2FC204670BDF0B587B0BE
:1096A0000546012144F20400F6F7B9FC7C4E304631
:1096B000F7F7C0FB7015ADF8180003208DF81A00FD
:1096C00018208DF81B00774F06A93846EFF7A1FB4D
:1096D0003015ADF8180048208DF81B0006A9384653
:1096E000EFF797FBB415ADF8184010208DF81B006C
:1096F00006A93846EFF78DFB21463846EFF7F8FB11
:1097000025208DF8040000248DF805408DF80640D2
:1097100001208DF8070001A8EFF703F80295ADF8D6
:109720000C40ADF80E40ADF81040ADF814400C20E0
:10973000ADF8120002A93046F7F7C4FB012240F24F
:1097400025513046F7F745FC01213046F7F735FC47
:1097500007B0F0BD70B586B0054601210820F6F7C8
:109760005EFC01218804F6F765FC4F4E3046F7F7A2
:1097700061FB3015ADF8140003208DF81600182099
:109780008DF81700494C05A92046EFF742FBE0147D
:10979000ADF8140048208DF8170005A92046EFF712
:1097A00038FB27208DF8000000248DF801408DF84B
:1097B000024001208DF803006846EEF7B2FF0195E4
:1097C000ADF808407014ADF80A00ADF80C40ADF8E3
:1097D00010400C20ADF80E0001A93046F7F772FBDF
:1097E000012240F225513046F7F7F3FB01213046C4
:1097F000F7F7E3FB06B070BD70B586B005460121F2
:109800001020F6F70CFC01212020F6F708FC0121BE
:109810000805F6F70FFC264E3046F7F70BFBB014A1
:10982000ADF8140003208DF8160018208DF81700ED
:1098300005A92048EFF7EDFA0420ADF81400482000
:109840008DF8170005A91C48EFF7E3FA35208DF8CD
:10985000000000248DF801408DF8024001208DF8B1
:1098600003006846EEF75DFF0195ADF808407014FF
:10987000ADF80A00ADF80C40ADF810400C20ADF882
:109880000E0001A93046F7F71DFB012240F22551D9
:109890003046F7F79EFB01213046F7F78EFBA9E72C
:1098A000003801400008014000480040000C014021
:1098B0000050004000100140001401404FF0E02132
:1098C0000A6922F004020A61224AC00810704FF4AB
:1098D0007A735843012353804861086940F00100BE
:1098E000086170472DE9F04100244FF0E0277E69C0
:1098F0000546184800784543FFF71FFEBA69B96965
:109900009142FCD003D2A2EB0100044403E0A6EB99
:109910000100104404440A46AC42F0D3BDE8F041D3
:10992000FFF713BE70B50446FFF788FD60B1094D1F
:109930006888844203D3B4FBF0F0FFF762FB6888C9
:10994000B4FBF0F100FB11444FF47A706043BDE8C2
:109950007040C7E714030020F849FF200870F84959
:1099600008707047F74900200860F7494873487647
:10997000012240F22551F548F7F72BBB10B5F24C08
:10998000E07B801EC1B2F24806F090F8F049E27B1D
:10999000E37B0A4412F8012C194411F8021C02EB73
:1099A0000121814201D1012010BD002010BD2DE90F
:1099B000F05FDFF8988340F225514046F7F7D6FB79
:1099C000DFF890A301270026DFF88C93DE4C0128F6
:1099D00029D040F2277529464046F7F7C7FB0128F2
:1099E00055D18AF8077099F80610032901D000298B
:1099F0004DD1E28CE08B824273D340214046F7F791
:109A0000AAFB0028F9D040214046F7F7ABFB002223
:109A100029464046F7F7DDFAE684FFF7A3FFBDE8E5
:109A2000F05F0DF0A9B98AF8087099F806100329BB
:109A30000AD000292BD14046F7F724FBC1B2BDE87C
:109A4000F05FC6480DF0B4B8607BC14DDC2807D28A
:109A50004046F7F717FB617B4A1C6273685401E0CC
:109A6000FFF780FF607B01280DD0607B042810D0B9
:109A7000607B07281CD0607BDFF8E4824FF003098D
:109A8000062841D043E05020E073207EE075BDE819
:109A9000F09FE878A97800EB01200A28F7D16878D0
:109AA0000628F4D10C20E073207E0830E075EEE744
:109AB0006878032816D0062814D010281DD02978DD
:109AC0005529E4D1FF28E2D1A8780128DFD16879AF
:109AD0000028DCD1A8790028D9D127700520607032
:109AE000D5E769E0E878A97800EB01200A28CED014
:109AF0000820E073207EE075C9E7A87900F109012C
:109B0000E1730830E075C2E76878192828D0607BD7
:109B1000E17B8842BBD16878032803D0062801D0B6
:109B20001028B4D12878DFF83CB2FF2803D09BF886
:109B3000061088423DD1FFF721FFB0B3A07801287D
:109B400024D08AF808709BF8D80030B18649C0EB61
:109B500000108000088085480670E67500201DE032
:109B6000A08B002893D1607A002890D0607BE073AE
:109B7000E67584F81990002004E0295C08F80010CC
:109B8000401CC0B2E17B8842F7D380E7BDE8F05FBC
:109B9000E8E6295C08F80010401CC0B2E17B88426E
:109BA000F7D384F81990277271E7FFE7BDE8F05FFB
:109BB000D8E6BDE8F05FD5E6501CE0846C48815CD7
:109BC0004046F7F75BFABDE8F05F0DF0D5B870B529
:109BD000684D40F225512846F7F7C8FA664CB8B1EF
:109BE0002846F7F74FFAC2B2B4F8000440F2FF314A
:109BF000C0F30E0088420BD2B4F80004B4F800346D
